:1000000000800020BD010000899B00004D9B000086
:100010004D9B00004D9B00004D9B00004D9B000040
:100020004D9B00004D9B00004D9B0000899B0000F4
:10003000899B00004D9B0000899B00003D9B0000B8
:10004000899B0000899B0000899B0000899B000020
:10005000899B0000899B0000899B0000899B000010
:10006000899B0000899B0000899B0000899B000000
:10007000899B0000899B0000899B0000899B0000F0
:10008000899B0000899B0000899B0000899B0000E0
:10009000899B0000899B0000899B0000899B0000D0
:1000A00099950000899B0000899B0000899B0000B6
:1000B000899B0000899B0000899B0000899B0000B0
:1000C000899B0000899B0000899B0000899B0000A0
:1000D000899B0000899B0000899B0000899B000090
:1000E000899B0000899B0000899B0000899B000080
:1000F000899B000025A60000899B0000FDC200002E
:10010000899B000079C80000899B0000899B000042
:10011000899B0000899B0000899B0000899B00004F
:10012000899B0000899B0000899B0000899B00003F
:10013000899B0000899B0000899B0000899B00002F
:10014000899B0000899B0000899B0000899B00001F
:10015000899B0000899B0000899B0000899B00000F
:10016000899B00000DA90000899B0000899B00006D
:10017000899B0000899B0000899B0000899B0000EF
:10018000899B0000899B0000899B0000899B0000DF
:10019000899B000025690000899B0000899B000065
:1001A000899B0000899B0000899B0000899B0000BF
:1001B000899B0000899B000019B60000574B4CF248
:1001C000205210B51A804DF628121A8000BF00BFC9
:1001D00009F0DEFC524B4FF010621A60514A9A60EF
:1001E000514ADA60A3F53043203B1A6812F480725A
:1001F00004D14E490A604FF4A8521A604C4B1A7849
:10020000110703D51A7842F008021A70494B4A4C7C
:100210004A482A221A704A4A00239918A14203D256
:10022000195899500433F8E7464B474900228B424E
:1002300002D243F8042BFAE74448454900235A58B0
:100240001A500433B3F5DE7FF9D1424B424A802184
:1002500003F8011B9342FBD1404B3C4A1A60404BD0
:100260008A221A70A3F5805324225A70A0221A7091
:100270009A799207FCD59A79D406FCD4394A9379B5
:1002800003F00C03082B374BF9D103221A714022DB
:100290005A719A799006FCD5324A9179314B4906C8
:1002A000FBD5314A314911600221516020221A7078
:1002B0009A7902F00C020C2AFAD12D4B2D4A1A60C1
:1002C0002D4B2E4A1A6000225A60072243F8042C54
:1002D0002B4AC3F80C2D62B609F044FE134B1B6881
:1002E000DA0705D5274809F003FD274B274A1A608E
:1002F000274B1B785B0609D5234C244A236893427D
:1003000004D1204809F0F4FC002323600DF01EFD09
:1003100009F044FC0BF076FCFEE700BF0E20054020
:1003200030800440823F04000100002B14D00340C1
:1003300002D0074000E00740E8ABFF1F4005010086
:100340006097FF1FE8ABFF1F6CD9FF1F0092FF1FD4
:100350000000000000E400E05FE400E008ED00E0E1
:100360000050064000400640448004400000030165
:1003700004800440C010050014E000E0FF76010096
:100380000000202063D1545B1CE00340A5C3945AB5
:1003900000F00740FFFFFFFFFFFFFFFFFFFFFFFF32
:1003A000FFFFFFFFFFFFFFFFFFFFFFFFFFFFFFFF5D
:1003B000FFFFFFFFFFFFFFFFFFFFFFFFFFFFFFFF4D
:1003C000FFFFFFFFFFFFFFFFFFFFFFFFFFFFFFFF3D
:1003D000FFFFFFFFFFFFFFFFFFFFFFFFFFFFFFFF2D
:1003E000FFFFFFFFFFFFFFFFFFFFFFFFFFFFFFFF1D
:1003F000FFFFFFFFFFFFFFFFFFFFFFFFFFFFFFFF0D
:10040000FFFFFFFFFFFFFFFFFFFFFFFFDEF9FFFF23
:1004100010B5054C237833B9044B13B10448AFF33E
:1004200000800123237010BDE8ABFF1F0000000017
:100430004005010008B5064B1BB106480649AFF35D
:1004400000800648036813B1054B03B1984708BD07
:100450000000000040050100ECABFF1FE8ABFF1FF0
:100460000000000038B5074C074DC4F8B05204F541
:10047000327008F0ADF8204640F8185B08F0A8F894
:1004800038BD00BF68BCFF1F9000010070B5084E6A
:1004900006F62804A6F52676064D44F8185C204694
:1004A00008F096F8A4F52C74B442F6D170BD00BFE4
:1004B000B4AEFF1F9000010008B5224B1B7813B1AA
:1004C000012B13D008BD204B1968204B1B68194421
:1004D0001F4B19601F4806F013FA0122194B1A70BE
:1004E0001D4814211D4A06F011FB08BD184B1A685F
:1004F000164909680A441A60194B1B7823B1194B35
:100500001B689A4204DA0AE0164B1B689A4206DC22
:10051000144B1A680E4B1A6002220A4B1A700D48CF
:100520000B4B196806F0ECF9064B1B78012B05D133
:1005300009481421094A06F0E9FA08BD0022014BD6
:100540001A7008BD71ADFF1F7C9AFF1F6CADFF1FB5
:1005500078ACFF1F9CC2FF1F88ADFF1FB9040000CD
:1005600004C6FF1F14A1FF1F00B583B0374B1B78D3
:1005700043B10022364B1A703648374B196806F0E3
:10058000DFFA5FE0354B1B78012B1AD013B1022B39
:1005900036D057E0324B187809F0DEFB002851D1F5
:1005A000304B1B680093009A2F4B1A602948142186
:1005B0002E4A06F0ABFA284B18600122274B1A701E
:1005C00040E0274B187809F0C7FB58BB244B5B78F9
:1005D00063B327E01F481421244A06F097FA1E4B04
:1005E00018602FE001221A4B1A7002221B4B1A705E
:1005F000184864211D4A06F089FA174B186021E05B
:10060000174B187809F0A8FB012803D10022104BE2
:100610001A7017E00F486421144A06F077FA0E4B5F
:1006200018600FE000220A4B1A700BE00D4B1B689C
:100630000193019A0C4B1B68D21A40F2DB539A4289
:10064000C8D9CFE703B05DF804FB00BF8FBBFF1F25
:1006500084C2FF1F88ADFF1F58BAFF1FC8C1FF1F0C
:1006600088C4FF1F20D6FF1FF4C5FF1F69050000C7
:100670000F4B03604172026100230372C36039B102
:100680001946026942F823100133427A9A42F8DC93
:10069000084B1A680AB9186004E053690BB11A468E
:1006A000FBE75061002343618380C380704700BF34
:1006B00040F30000B0D7FF1F144B036004234372C4
:1006C00000F12803036100230372C3601946026925
:1006D00042F823100133427A9342F8DB0C4B1A683C
:1006E0000AB9186004E053690BB11A46FBE7506180
:1006F000002343618380C380064B03604FF4803343
:100700008361C36103624362704700BF40F300002E
:10071000B0D7FF1F7000010010B504460F4B0360F7
:100720000023437203610372C3600D4B1A680AB958
:10073000186004E053690BB11A46FBE754610023CB
:100740006361A380E3802046064B40F8183B07F026
:100750002FFF204606F040FD204610BD40F300006C
:10076000B0D7FF1F9000010010B5124B5B7B13B98F
:10077000114B5B7B4BB1114B5B7B33B1104B5B7B04
:100780001BB101220F4B1A7010BD00220D4B1A70C5
:100790000D4B1B7863B10D4C20460BF019F8236804
:1007A0005B6820460A492622984720460BF010F83D
:1007B00010BD00BF68A0FF1F649AFF1F98A0FF1F15
:1007C000589FFF1F80C5FF1F639AFF1FE4D7FF1FBD
:1007D00060F3000010B5174B5B7B9BB10122164BF9
:1007E0001A70164B1B781BB3154C23685B682046A8
:1007F00014491C22984720460AF0EAFF20460AF0D6
:10080000E7FF10BD00220C4B1A700C4B1B787BB11C
:100810000B4C20460AF0DCFF23685B6820460A493F
:100820002E22984720460AF0D3FF20460AF0D0FF38
:1008300010BD00BF18A1FF1F8EBBFF1F639AFF1FD3
:10084000E4D7FF1F88F30000A8F30000F8B50746BF
:10085000224B1B78002B3FD0214803685B6821495D
:100860000E229847204A4FF42C7303FB07F3D41849
:1008700004F2832402F524761E44194D2B681B686C
:10088000284614F8011F9847B442F7D1144C236846
:100890005B682046154910229847204639460A22AF
:1008A00000230AF0A5FF23685B6820461049062252
:1008B00098474FF42C720C4B02FB07372046B7F8D1
:1008C000AA120AF0D1FF23685B6820460949012279
:1008D000984720460AF07CFFF8BD00BF639AFF1FCF
:1008E000E4D7FF1FD8F3000068BCFF1FE8F3000047
:1008F000FCF3000004F40000F8B50746224B1B7817
:10090000002B3FD0214803685B6821490E2298479D
:10091000204A4FF42C7303FB07F3D41804F283240A
:1009200002F524761E44194D2B681B68284614F8DE
:10093000011F9847B442F7D1144C23685B682046E6
:1009400015490C229847204639460A2200230AF00E
:100950004FFF23685B6820461049062298474FF4F2
:100960002C720C4B02FB07372046B7F8AA120AF08C
:100970007BFF23685B68204609490122984720468F
:100980000AF026FFF8BD00BF639AFF1FE4D7FF1FE0
:10099000D8F30000B4AEFF1F08F40000FCF3000021
:1009A00004F40000F8B50746224B1B78002B3FD01B
:1009B000214803685B6821490E229847204A4FF47A
:1009C0002C7303FB07F3D41804F2832402F5247676
:1009D0001E44194D2B681B68284614F8011F9847C0
:1009E000B442F7D1144C23685B68204615490C22A9
:1009F0009847204639460A2200230AF0F9FE236868
:100A00005B6820461049062298474FF42C720C4B25
:100A100002FB07372046B7F8AA120AF025FF236821
:100A20005B68204609490122984720460AF0D0FE1B
:100A3000F8BD00BF639AFF1FE4D7FF1F18F4000042
:100A4000B4AEFF1F08F40000FCF3000004F4000043
:100A500038B50546124B1B7803B3124C23685B680C
:100A600020461149072298472046691C0AF0FCFEDF
:100A700023685B6820460D490A2298470C4B03EB1C
:100A800005152046A9890AF0EFFE23685B68204619
:100A900008490322984720460AF09AFE38BD00BF55
:100AA000639AFF1FE4D7FF1F28F4000030F4000012
:100AB0008CC5FF1F3CF4000010B50446092804D87B
:100AC000054803681B6830219847034821460A22DD
:100AD00000230AF08DFE10BDE4D7FF1FF8B5274BA9
:100AE000A3FB00239B0B264DA5FB03246409C4EB49
:100AF0000414A3EB8404234BA3FB00239B09A5FB55
:100B000003256D09C5EB0515A3EB85054FF47A7236
:100B100002FB13000CF0A2FE1B490CF0A7FF0646D7
:100B200000210DF0A1F840B130464FF07C510CF09F
:100B3000E1FD0DF0ADF8074607E030464FF07C517F
:100B40000CF0D6FD0DF0A4F80746E0B2FFF7B4FFB5
:100B50000E4C23680E4E5B682046314601229847B2
:100B6000E8B2FFF7A9FF23685B68204631460122FF
:100B70009847F8B2FFF7A0FFF8BD00BF73B2E74592
:100B800089888888D34D621000002041E4D7FF1F78
:100B900040F40000F8B53225094C0A4F01262368BD
:100BA0005B6820463946324698476B1E13F0FF05B6
:100BB000F5D103480AF00CFE0AF0B8FBF8BD00BFFF
:100BC000E4D7FF1F44F4000010B584B0164C204653
:100BD0000AF0FEFDFFF7DEFF23685B68204613493D
:100BE000122298472046124B19780A2200230AF055
:100BF000FFFD20460AF0ECFD23685B6820460D49A6
:100C00001222984768460C490AF0D0FF20466946F0
:100C10000AF0B8FD20460AF0DBFDFFF7BBFF68468F
:100C20000AF078FF04B010BDE4D7FF1F48F40000BD
:100C3000FA9AFF1F5CF4000070F40000F8B532254A
:100C4000094C0A4F012623685B6820463946324624
:100C500098476B1E13F0FF05F5D103480AF0B8FD65
:100C60000AF064FBF8BD00BFE4D7FF1F64F5000085
:100C700008B5034803685B6802490122984708BD2C
:100C8000E4D7FF1FECF7000038B5054630B100246B
:100C9000FFF7EEFF0134E4B2AC42F9D138BD00BF3A
:100CA00070B506460024124D2B681B682846315D3E
:100CB000984701340D2CF7D10620FFF7E5FF737B31
:100CC00063B13069FFF70AFF0620FFF7DDFF084830
:100CD000317D0A2200230AF08BFD05E004480368F9
:100CE0005B6804490122984701480AF071FD70BD14
:100CF000E4D7FF1F44F4000038B5154C20460AF035
:100D000067FDFFF747FF23685B68204611490F2204
:100D1000984720460AF05CFDFFF73CFF23685B68BC
:100D200020460D492822984720460AF051FDFFF73A
:100D300031FF0A4D2C1F05F5CA7554F8040FFFF753
:100D4000AFFFAC42F9D102480AF042FD38BD00BF06
:100D5000E4D7FF1F80F4000090F40000A4C2FF1F3E
:100D600008B530B1064803685B6806490322984716
:100D700008BD034803685B6803490222984708BD21
:100D8000E4D7FF1FCCF40000D0F4000008B5FFF753
:100D9000E7FF02480AF01CFD08BD00BFE4D7FF1FB3
:100DA00030B4002308481946012502241954C218FA
:100DB00051709170D57014710533962BF6D10022C5
:100DC000024B1A7030BC704768BAFF1F84C4FF1F03
:100DD00038B5274C23685B68204626490722984788
:100DE00020460AF0F5FC23685B68204622490F2262
:100DF0009847224D286822490CF084FD0CF06EFFC4
:100E0000C1B220460A2200230AF0F2FC20460AF072
:100E1000DFFC23685B6820461A49102298476868FF
:100E200017490CF06FFD0CF059FFC1B220460A22A1
:100E300000230AF0DDFC20460AF0CAFC23685B6848
:100E40002046114916229847A8680D490CF05AFD12
:100E50000CF044FFC1B220460A2200230AF0C8FC6D
:100E600020460AF0B5FC20460AF0B2FC38BD00BFAF
:100E7000E4D7FF1FE4F40000ECF400004098FF1FEB
:100E80000000C842FCF4000010F500002DE9F84312
:100E90002A4C23685B68204629490F229847204640
:100EA0000AF096FC00260125DFF8AC90DFF8AC8054
:100EB00023685B6820464946072298472046294612
:100EC0000AF0D2FC23685B68204641460522984719
:100ED0001C4F2046B95B0AF0C7FC23685B682046BC
:100EE0001949052298473744204679880AF0BCFC06
:100EF00023685B6820461549092298473879FFF72F
:100F00002FFF20460AF064FC01351036072DCFD1A3
:100F10000A4C23685B6820460D49112298472046F9
:100F20000C4B19780A2200230AF062FC20460AF0D2
:100F30004FFC20460AF04CFCBDE8F883E4D7FF1FC5
:100F400028F500008CC5FF1F40F5000048F50000A3
:100F500054F50000FF9AFF1F28F4000038F5000048
:100F60002DE9F843002601251D4CDFF88490DFF8B9
:100F7000848023685B6820464946062298472046BD
:100F800029460AF071FC23685B68204641460D2221
:100F90009847144F2046B95B0AF066FC23685B68EB
:100FA00020461149102298473744204679880AF094
:100FB0005BFC23685B6820460C4911229847204659
:100FC000B9880AF051FC20460AF002FC01350636C9
:100FD000042DCED102480AF0FBFBBDE8F88300BF28
:100FE000E4D7FF1F74ADFF1F80F5000094F50000EB
:100FF00068F5000070F5000010B582B03C4C236825
:101000005B6820463B491822984720460AF0E0FBDF
:1010100023685B682046384921229847374B187867
:10102000FFF7B4FE23685B682046354925229847C0
:10103000344B1868B8B10CF00DFC33490CF016FDB8
:101040000CF044F802460B460121009120460AF0BC
:1010500017FC23685B6820462C49082298472046E5
:101060000AF0B6FB09E0224C23685B682046284959
:101070000322984720460AF0ABFB1D4803685B68D3
:10108000244918229847244B1B7853B1184C2368E5
:101090005B68204621490C22984720460AF098FBBD
:1010A00009E0134C23685B6820461D4909229847D4
:1010B00020460AF08DFB0E4C23685B6820461949D8
:1010C0000F2298472046184B19780A2200230AF06D
:1010D0008FFB23685B68204614490122984720460D
:1010E0000AF076FB20460AF073FB02B010BD00BF89
:1010F000E4D7FF1FA8F50000C4F5000055BAFF1F94
:10110000E8F5000004C5FF1F00606A4710F6000004
:101110001CF6000020F60000F89AFF1F3CF60000C5
:101120004CF6000058F60000F99AFF1FE0F40000AA
:1011300038B53D4C23685B6820463C490E229847F1
:1011400020460AF045FB23685B6820463849102298
:101150009847384B1878FFF719FE23685B682046DC
:101160003549102298472046344B19880AF07CFBF9
:101170002368334D5B682046294603229847204662
:101180000AF026FB23685B6820462E491022984708
:1011900020462D4B19880AF067FB23685B682046C0
:1011A00029460322984720460AF012FB23685B6811
:1011B000204626490C2298472046254B19780A22BA
:1011C00000230AF015FB23685B68204621490C22A6
:1011D00098472046204B19680AF046FB23685B6855
:1011E00020461E490622984720461D4B19780A22A0
:1011F00000230AF0FDFA23685B68204619490B2298
:1012000098472046184B19680AF02EFB23685B6844
:10121000204616490422984720460AF0D9FA20466B
:101220000AF0D6FA38BD00BFE4D7FF1F68F6000009
:1012300078F6000004C6FF1F8CF600007EC5FF1F75
:101240003CF40000A0F60000F8C5FF1FB4F6000053
:1012500010A1FF1FC4F600007C9AFF1FD4F6000007
:10126000629AFF1FDCF6000014A1FF1FE8F60000E1
:1012700070B50D4614460138062800F2BD80DFE83F
:1012800000F0040B12192D5594005C4803685B684C
:101290005B490C22984770BD584803685B68594900
:1012A0000B22984770BD554803685B6856490D226C
:1012B000984770BD514C23685B682046534907220C
:1012C0009847204629460A2200230AF091FA23680B
:1012D0005B6820464E490522984770BD474E3368EB
:1012E0005B6830464B490C229847304629460A2213
:1012F00000230AF07DFA022C0AD0032C0FD0012C17
:101300007AD1304633685B6843490622984770BDFE
:101310003A4803685B6841490522984770BD3748E1
:1013200003685B683E490722984770BD334E3368B7
:101330005B6830463B4906229847304629460A22D8
:1013400000230AF055FA013C052C55D8DFE804F0DB
:10135000030A11181F26294803685B6832490322D3
:10136000984770BD254803685B6830490422984758
:1013700070BD224803685B6829490722984770BD01
:101380001E4803685B682A490F22984770BD1B48B6
:1013900003685B6827491022984770BD17480368A7
:1013A0005B6825490622984770BD144E33685B6818
:1013B000304622490B229847304629460A2200230C
:1013C0000AF016FA022C0AD0032C0FD0012C13D1EC
:1013D000304633685B681A490522984770BD074854
:1013E00003685B680D490522984770BD0348036890
:1013F0005B6814490722984770BD00BFE4D7FF1F00
:10140000F0F6000000F700000CF700001CF70000E9
:1014100024F700002CF700003CF7000044F7000020
:101420004CF7000068F5000054F7000058F7000082
:1014300060F7000070F7000084F700008CF70000F0
:1014400098F70000A0F700002DE9F8435A4C2368F4
:101450005B68204659490D22984720460AF0B8F9A2
:10146000574D0126DFF89091DFF8908123685B6883
:101470002046494608229847204631460AF0F4F9AA
:1014800023685B6820464146022298472F466B7DC1
:1014900093B123685B6820464A4908229847204652
:1014A000697A0A2200230AF0A3F923685B682046C0
:1014B00045490B22984727E023685B68204643494B
:1014C00011229847AB7D012B0AD013B1022B0ED00D
:1014D00014E023685B6820463D490422984713E0E6
:1014E00023685B6820463B490C2298470CE0236840
:1014F0005B68204638490D22984705E023685B6801
:101500002046364907229847FB792BB123685B6850
:10151000204633491322984720460AF059F90136EC
:101520001835062EA2D1244C20460AF051F9236822
:101530005B6820462B491022984720460AF048F95C
:10154000294B1B78002B32D00025DFF8AC80274FC9
:1015500023685B68204641460822984705EB8503CF
:10156000FE182046F95C0A2200230AF041F923689C
:101570005B6820461E4905229847204671780A225A
:1015800000230AF035F923685B68204619490322D5
:101590009847B078F1783279FFF76AFE20460AF072
:1015A00017F90135EDB2104B1B78AB42D0D8024889
:1015B0000AF00EF9BDE8F883E4D7FF1FA8F7000092
:1015C00088C4FF1FC4F70000D0F70000DCF700005C
:1015D000F0F70000F8F7000008F8000018F8000025
:1015E00020F8000034F8000084C4FF1F68BAFF1F11
:1015F00048F8000078F40000B8F7000000F400009C
:1016000070B5054610B1441EE4B200E000244B1E44
:10161000052B00F22581DFE813F0060028004A00C0
:101620008800B200FF002C208E4B00FB043005F038
:101630000DF88D4B1B78002B00F012818B4C23682A
:101640005B6820468A4906229847204629460A2296
:1016500000230AF0CDF823685B6820468549032201
:10166000984720460AF0B4F870BD2C207D4B00FB53
:10167000043004F0F5FF7C4B1B78002B00F0F08069
:101680007A4C23685B6820467949062298472046B1
:1016900029460A2200230AF0ABF823685B6820463B
:1016A00075490422984720460AF092F870BD2C2212
:1016B0006C4B02FB0434204604F080FF6A4B1B781D
:1016C000002B00F0CD80204604F03AFFB0B1674C0B
:1016D00023685B68204666490622984720462946CB
:1016E0000A2200230AF084F823685B6820466349D5
:1016F0000A22984720460AF06BF870BD5B4C2368BD
:101700005B6820465A4906229847204629460A2205
:1017100000230AF06DF823685B68204658490B22C5
:10172000984720460AF054F870BD564B62001119D4
:1017300003EB41010B462C204A4A00FB0420498858
:101740009A8804F0C5FF484B1B78002B00F0888076
:10175000464C23685B682046454906229847204648
:1017600029460A2200230AF043F823685B682046D2
:1017700045490F22984720460AF02AF870BD2C26CA
:10178000384B06FB0436304604F026FF18B13046CD
:1017900004F054FF0AE03B4B6200111903EB4101D6
:1017A0000B46304649889A8804F092FF2E4B1B78EE
:1017B000002B55D0304604F00FFFB0B12B4C2368FE
:1017C0005B6820462A4906229847204629460A2275
:1017D00000230AF00DF823685B6820462A490F228F
:1017E0009847204609F0F4FF70BD204C23685B68E1
:1017F00020461F4906229847204629460A220023F0
:1018000009F0F6FF23685B68204620490E229847BE
:10181000204609F0DDFF70BD04EB44022C20114B83
:1018200000FB0430174B33F8121004F001FF0E4B8D
:101830001B78ABB10D4C23685B6820460C4906222F
:101840009847204629460A22002309F0D1FF236841
:101850005B6820460E4906229847204609F0B8FFEB
:1018600070BD00BFCCC1FF1F639AFF1FE4D7FF1FED
:1018700068F5000050F8000054F800005CF8000023
:1018800068F8000074ADFF1F74F8000084F80000D1
:1018900094F800002DE9F843144E06F1080406F10F
:1018A00080094FF00208002540F2DC5714F8080CBC
:1018B000414608F05FFA04F8075C24F8067C24F837
:1018C000047C04F8025C357204F8015C0323737233
:1018D00086F80A80F560A560257301236373A573FC
:1018E000183618344C45E1D1BDE8F88388C4FF1F91
:1018F00010B50F4C20780F49042208F07BFA207EA7
:101900000D49042208F076FA94F830000B490422BD
:1019100008F070FA94F848000949042208F06AFABD
:1019200094F860000749042208F064FA10BD00BF73
:1019300088C4FF1FF9190000051A0000111A0000E1
:101940001D1A0000291A000008B5134B1878222828
:1019500028BFFF2008F082F90F4B187E222828BFED
:10196000FF2008F07BF90C4B93F83000222828BFA9
:10197000FF2008F073F9084B93F84800222828BF8D
:10198000FF2008F06BF9044B93F86000222828BF71
:10199000FF2008F063F908BD88C4FF1F70B5044636
:1019A00008F0A8FA054604EB4402114B03EBC2030E
:1019B0009B79DBB90E4B13F8320008F0CDF950B12A
:1019C00004EB44020A4B03EBC203DD6074B901224D
:1019D000084B1A7070BD064B6200101903EBC00073
:1019E000C668AE1B8680C5600122827170BD00BFD3
:1019F00088C4FF1F8FBBFF1F08B50020FFF7CEFF75
:101A000008BD00BF08B50120FFF7C8FF08BD00BF33
:101A100008B50220FFF7C2FF08BD00BF08B50320CC
:101A2000FFF7BCFF08BD00BF08B50420FFF7B6FFF5
:101A300008BD00BF10B5104B1B78012B03D073B14C
:101A4000022B04D012E00D4804F000FE0EE00B4C17
:101A5000204604F005FE204604F05CFE06E0074C3C
:101A6000204604F0FDFD204604F04CFE024B1A789F
:101A7000034B1A7010BD00BF00C5FF1F60BBFF1FE6
:101A8000FDBBFF1F2DE9F04182B0234B1B68009383
:101A9000009A224B1B68D31A642B3AD91E4B1B6841
:101AA0000193019A1D4B1A6008F024FA4FF080420E
:101AB0001B4B1A6072B61B4E06F110023346883675
:101AC0000024194D4FF00208A4461969411AA94291
:101AD00009D90134E4B212F80F1C012904BF02F83D
:101AE0000F8C83F814C018321833B242EDD162B6AD
:101AF0004FF080420D4B1A60052C02D102220C4B94
:101B00001A700B4B1A780B4B1B789A4201D0FFF7D7
:101B100091FF02B0BDE8F08120D6FF1F50BAFF1F31
:101B200088E100E088C4FF1FA086010008E100E012
:101B300000C5FF1FFDBBFF1F2DE9F00F82B08046DF
:101B400000EB40025D4B03EBC2035F8893F8099002
:101B5000C7F57A75002DB8BF6D424E46B9F1010F39
:101B60004BDD0022012342F20F719446A9F10204D9
:101B7000DFF858B1DFF858A15148CDF80480042CA3
:101B80002FD8DFE804F0030C151D26004D49114441
:101B9000B1F90210C91B0029B8BF494221E04A49E6
:101BA0001144B1F90210C91B0029B8BF494218E01D
:101BB0008118B1F90210C91B0029B8BF494210E0D1
:101BC0000AEB0201B1F90210C91B0029B8BF494252
:101BD00007E00BEB0201B1F90210C91B0029B8BFE5
:101BE0004942A942BCBF5FFA83FC0D460133023271
:101BF000B342C4DBDDF8048001E04FF0000C0CF1CF
:101C0000010C5FFA8CF008EB48082C4B03EBC8087A
:101C100098F80730002B4DD0A9F10209B9F1040F53
:101C200048D8DFE809F003080E182200012814BF85
:101C3000012002203EE0012825D0032808BF012012
:101C400038E0012821D0022821D0032821D00428FF
:101C500008BF01202EE001281DD002281DD0042835
:101C60001DD0052808BF012024E0012819D0022832
:101C700019D0032819D0042819D0052819D006280E
:101C800008BF012016E0032014E0042012E0032026
:101C900010E002200EE005200CE004200AE0022003
:101CA00008E0062006E0052004E0042002E003200E
:101CB00000E0022002B0BDE8F00F704788C4FF1FAB
:101CC00080FD000048F300004CF3000054F30000D6
:101CD00088FD000042780378134482781344C27868
:101CE0001344007903F07F03984214BF00200120C1
:101CF000704700BF08B50138052820D8DFE800F09C
:101D000003070C11161B0E4808F088F908BD44F6AD
:101D1000206008F083F908BD42F2107008F07EF9E7
:101D200008BD41F2883008F079F908BD40F28360BF
:101D300008F074F908BD40F6055008F06FF908BDC9
:101D40008038010008B50648064B196804F0D8FD34
:101D50000548064B1988064A04F0D8FE08BD00BFA6
:101D60009CC2FF1F7C9AFF1F88ADFF1F7EC5FF1F0F
:101D7000B904000010B51E4B1B78DBB11D4B186871
:101D80001D4B1B68C01A0BF069FD04461B4B1888DD
:101D90000BF060FD1A490BF069FE014620460BF07E
:101DA00065FE4FF07C510BF0A5FC0BF071FF154B5D
:101DB000186010BD104B18680E4B1B68C01A0BF052
:101DC0004DFD04460D4B18880BF044FD0C490BF0FB
:101DD0004DFE014620460BF049FE4FF07C510BF0C2
:101DE00089FC0BF055FF4042064B186010BD00BF48
:101DF00004C6FF1F14A1FF1F7C9AFF1FF8C5FF1F19
:101E00000000A0416CADFF1F38B5254B18780BF0D2
:101E100021FD24490BF06CFC23490BF073FD0546B2
:101E2000224B18780BF016FD1E490BF061FC1E4981
:101E30000BF068FD04461E4B1B78C3B128461D49B4
:101E40000BF058FC4FF07C510BF054FC0BF020FFD2
:101E5000194B1860204619490BF04CFC4FF07C518F
:101E60000BF048FC0BF014FF154B186038BD2846EA
:101E700012490BF03FFC4FF07C510BF03BFC0BF098
:101E800007FF0D4B186020460A490BF033FC4FF05A
:101E90007C510BF02FFC0BF0FBFE094B186038BD9A
:101EA00010A1FF1F0000C8420000A040629AFF1F5F
:101EB00004C6FF1F00007A447C9AFF1F0000FA440A
:101EC00014A1FF1F70B5FEF76BFF4F4B0021597532
:101ED00001229A7583F87510022183F876104B4B16
:101EE00019705A709A70597103209871D97198724B
:101EF000DA7204251D735A73D873197405245C743F
:101F00009974D974187558759C75D9751A765D765B
:101F10009A760724DC761A775A779D77D87783F8F4
:101F2000204083F8211083F82220394B1C70394A55
:101F300040F2DC5313804FF47A6151804FF4FA641D
:101F4000148241F28833538240F6B83010844FF443
:101F5000FA5555844FF47A7515865486A2F84000D8
:101F6000A2F84210A2F8503041F27073A2F8523039
:101F7000131D02F1080102F16400002201F8042C93
:101F800001F8032C5A601A81103310318342F5D1C5
:101F90001922214B1A70214B4FF07C521A605A6063
:101FA0009A601F4C0126267005221E4B1A701E4B8C
:101FB0001E225A809A801A801A815A81DA80DA8128
:101FC0001A829A810025194B1D70C822184B1A805D
:101FD0004FF44872174B1A806423174A1370174A3C
:101FE00013704FF4FA62164B1A604FF47A72154B65
:101FF0001A60FFF709FFFFF7BDFE134B1E70134A6F
:10200000134B1A60257070BD88C4FF1F68BAFF1F8C
:1020100084C4FF1F8CC5FF1FFF9AFF1F4098FF1F3E
:10202000F89AFF1FF99AFF1F74ADFF1F04C6FF1F28
:102030007EC5FF1FF8C5FF1F10A1FF1F629AFF1F7B
:102040007C9AFF1F14A1FF1F55BAFF1FC0D40100C7
:1020500004C5FF1F2DE9F04F85B0AA4FAA4EAB4D26
:102060004FF05008CDF80080A94C04F116030193FD
:1020700038463146A74A2B4604F012FACDF80080C4
:1020800004F12E03019338463146A34A2B4604F04F
:1020900007FACDF8008004F1460301933846314633
:1020A0009E4A2B4604F0FCF9CDF8008004F15E0353
:1020B0000193384631469A4A2B4604F0F1F9CDF89F
:1020C000008004F17603019338463146954A2B4649
:1020D00004F0E6F904F17801234600209A7D02B16C
:1020E000587518338B42F9D1DFF818828E4F874E1E
:1020F0004FF05009CDF80090854DEB1D01934046FF
:1021000039468A4A334604F08BF9CDF8009005F140
:102110001F03019340463946854A334604F080F94F
:10212000CDF8009005F13703019340463946814AC6
:10213000334604F075F9CDF8009005F14F03019393
:10214000404639467C4A334604F06AF9CDF800909F
:1021500005F16703019340463946784A334604F057
:102160005FF96B7D53B1CDF8009005F10903019340
:1021700040467349734A334604F092F9644B93F82E
:102180002D304BB1502300936F4B01935D486C4948
:102190006E4A5E4B04F084F95D4B93F845304BB1C9
:1021A000502300936A4B019356486549694A574B3F
:1021B00004F076F9564B93F85D304BB15023009301
:1021C000654B01934F485E49644A504B04F068F9EF
:1021D0004F4B93F875304BB150230093604B0193F4
:1021E000484857495F4A494B04F05AF9FEF7D8FD71
:1021F000A1460B254FF0010ADFF888B1DFF8048112
:10220000594F4E4699F81530002B4AD099F80930AD
:10221000002B46D0002400230393601980B202A94A
:102220000A2207F009FD02465023009303AB0193F5
:1022300040463946354B04F067F968B34B4B1B7881
:102240001E2B29D84A4803EB8301421800F801A04D
:10225000611C51700398ABFB00C1490B5FFA81FE12
:1022600082F802E089B2DFF820C10CFB0101DFF83F
:102270001CC1ACFB01C1C1F347111171CEEB0E1EA5
:1022800000EB0E1001EB810EC1EBCE0100EB8101E2
:10229000D1700133354A13700134E4B2737AA3422A
:1022A000B9D80AF1010A5FFA8AFA09F118090A3560
:1022B000ADB2BAF1060FA4D1124D2E4F134C5026D9
:1022C0000096DFF8CC80CDF80480284639462A4AAB
:1022D000234604F009F9009608F102030193284609
:1022E0003946264A234604F0FFF8009608F1040315
:1022F000019328463946224A234604F091F8009675
:1023000048E000BF28C5FF1F9CF8000018BCFF1F55
:1023100088C4FF1FACF80000B8F80000C4F8000043
:10232000D0F80000DCF80000E8F80000FCF800003D
:1023300008F9000014F9000020F900002CF9000051
:1023400038F900004CF90000A9C4FF1F54F900003F
:10235000C1C4FF1F5CF90000D9C4FF1F64F900006D
:10236000F1C4FF1F6CF9000074F9000084C4FF1F62
:1023700068BAFF1F8CF900009CF90000A4F9000066
:10238000ACF900005917B7D1F0D8FFFF1F85EB510A
:102390008CC5FF1F08F11003019328463946A24A55
:1023A000234604F0A1F8009608F112030193284691
:1023B00039469E4A234604F097F8009608F1140324
:1023C0000193284639469A4A234604F029F8009694
:1023D00008F12003019328463946964A234604F023
:1023E00083F8009608F12203019328463946924A61
:1023F000234604F079F8009608F124030193284657
:1024000039468E4A234604F00BF8009608F1300353
:102410000193284639468A4A234604F065F8009617
:1024200008F13203019328463946864A234604F0D0
:102430005BF8009608F13403019328463946824A36
:10244000234603F0EDFF009608F140030193284670
:1024500039467E4A234604F047F8009608F14203C5
:102460000193284639467A4A234604F03DF80096FF
:1024700008F14403019328463946764A234603F07F
:10248000CFFF009608EB0603019328463946724AAF
:10249000234604F029F8009608F1520301932846D8
:1024A00039466E4A234604F01FF8009608F154039B
:1024B0000193284639466A4A234603F0B1FF009645
:1024C000684B019328463946674A234603F0E8FFE4
:1024D00004ABFF2203F8042D0096019328466349BC
:1024E000634A234603F0DCFF9DF80C00FF2809D067
:1024F0006428A8BF64200BF0ADF95E490BF0B6FA72
:102500005D4B186004ABFF2203F8042D50220092AB
:1025100001935A4855495A4A5A4B03F0C1FF9DF856
:102520000C00FF2809D06428A8BF64200BF092F9A2
:1025300050490BF09BFA504B586004ABFF2203F854
:10254000042D5022009201934C4848494E4A4D4B6D
:1025500003F0A6FF9DF80C00FF2809D06428A8BF4F
:1025600064200BF077F943490BF080FA424B9860F6
:10257000FF238DF80C30414D444F424C50260096BD
:10258000DFF82C81CDF8048028463946404A23469E
:1025900003F0AAFF009608F102030193284639468A
:1025A0003C4A234603F0A0FF009608F10403019380
:1025B00028463946384A234603F096FF009608F12C
:1025C0000603019328463946344A234603F08CFF1C
:1025D000009608F10803019328463946304A2346FD
:1025E00003F082FF009608F10A030193284639465A
:1025F0002C4A234603F078FF009608F10C03019360
:1026000028463946284A234603F06EFF009608F113
:102610000E03019328463946244A234603F064FFFB
:10262000009608F1100345E0B4F90000BCF9000081
:10263000C4F90000CCF90000D4F90000DCF9000076
:10264000E4F90000ECF90000F4F90000FCF90000E6
:1026500004FA00000CFA000014FA00001CFA000052
:1026600024FA0000FF9AFF1F2CFA000038FA00003D
:1026700040FA00000000C8424098FF1F28C5FF1F15
:1026800048FA000018BCFF1F50FA000058FA00007A
:1026900060FA00006CFA000078FA000084FA00008A
:1026A00090FA00009CFA0000A8FA0000B4FA0000BA
:1026B00074ADFF1F0193284639463A4A234603F07A
:1026C00013FF394F0096394B019328463946384A53
:1026D000234603F0A5FE0096364B01932846394663
:1026E000354A234603F000FF0096344B01932846F9
:1026F0003946334A234603F0F7FE0096314B0193E7
:1027000028463946304A234603F0CAFE00962F4B2E
:102710000193284639462E4A234603F0C1FEFFF7AF
:1027200073FBFFF727FB2B482B4B196804F0E8F8E5
:102730002A4F00962A4B019328463946294A2346B8
:1027400003F06EFE0096284B019328463946274A2F
:10275000234603F0D9FE264F0096264B01932846C8
:102760003946254A234603F05BFE0096234E019628
:1027700028463946224A234603F092FE30780BF071
:1027800069F820490BF072F91F490BF0BBF84FF0C4
:102790007C510AF0AFFF0BF07BFA1C4B187005B0B0
:1027A000BDE8F08FC0FA0000CCFA000004C6FF1F9D
:1027B000D4FA00007EC5FF1FE4FA0000F8C5FF1F31
:1027C000F0FA000010A1FF1FFCFA0000629AFF1F40
:1027D00008FB00009CC2FF1F14A1FF1F40FA00006D
:1027E00055BAFF1F14FB000004C5FF1F20FB0000AB
:1027F0002CFB0000F89AFF1F38FB0000F99AFF1F1E
:1028000048FB00000000C84200007F434DA0FF1FAE
:10281000054B1B781BB90122034B1A70704700222D
:10282000014B1A70704700BF5DBAFF1F2DE9F04FD2
:1028300083B00546894617469846467B002E00F031
:102840008480444B1878DFF824B18BF80000424CA8
:102850004FF42C7A0AFB004004F0D4FC9BF800C033
:102860000AFB0C4E0EF521740FCD0FC495E8030042
:1028700084E8030001228EF89C228EF89D928EF847
:10288000AE8247B10CEB8C0C344800EBCC003449E1
:1028900004F052FA08E00CEB8C0C304800EBCC0052
:1028A0003049012204F048FADFF8C08098F80000AF
:1028B000294C4FF42C7505FB00F02118084601F552
:1028C000217104F0CBFC98F80000274B1B680093A3
:1028D000009B05FB0044C4F8A032B4F8AA320133CF
:1028E000A4F8AA3284F8AC02FDF7B0FFFFF790FF1E
:1028F0005FB3184B1A78184B05FB023004F038FF11
:10290000054610B3134C237803EB8303134800EB05
:10291000C3001349002204F00FFA2378124A126808
:102920000192019A4FF42C700B4900FB031302F53E
:10293000C872C3F8A42203F52A71012283F8A822E1
:10294000002283F89D228A712E46304603B0BDE8EE
:10295000F08F00BF5DBAFF1F68BCFF1FE8ACFF1F10
:1029600016B703005D74D10520D6FF1F64BAFF1FA0
:1029700008B50B4600210122FFF758FF08BD00BF34
:1029800008B50B4601210A46FFF750FF08BD00BFFE
:1029900008B50B4600210A46FFF748FF08BD00BFF7
:1029A00000B583B0074B1878074B1B78013B0093A9
:1029B0000021FF220B4609F09FF8C0B203B05DF87A
:1029C00004FB00BF65BAFF1F90BBFF1F10B5064C8C
:1029D000204604F017FC04F52C7004F013FC0022D0
:1029E000024B1A7010BD00BF68BCFF1F5DBAFF1F0D
:1029F00008B50023034A1370034A1370FFF7E6FF7C
:102A000008BD00BF81C5FF1F80C5FF1F08B50B4B68
:102A10001B78012B11D10A4B1B6873B1094A11684D
:102A2000002903DD084804F0FDF808BD06481946F2
:102A3000064A04F06BF8034B186008BD70C2FF1F14
:102A400004C5FF1F00C6FF1F88ADFF1F152B000028
:102A500010B5074B1B78012B09D1064B1B6833B10E
:102A6000054C0648216804F06BF80023236010BD74
:102A700070C2FF1F04C5FF1F00C6FF1F88ADFF1FE8
:102A800010B5174A137817490B701070834225D080
:102A9000022B01D1FFF7DCFF114B1B78022B01D178
:102AA000FFF7B4FF0E4B1B78012B09D10E4C2368A6
:102AB0005B6820460D490C229847204608F088FEA6
:102AC000074B1B78082B09D1074C23685B6820460D
:102AD00007490F229847204608F07AFE10BD00BF34
:102AE00081C5FF1FFBC5FF1FE4D7FF1F58FB000078
:102AF00068FB000008B5054B1B782BB1044B1B7815
:102B000013B90120FFF7BCFF08BD00BF80C5FF1F40
:102B100081C5FF1F08B5044B1B7813F0F70F02D0D7
:102B20000820FFF7ADFF08BD81C5FF1F08B5194B91
:102B30001870194B1B78012B0DD1184B1B783BB328
:102B4000174B1B7853B1174B1B783BB903281FD980
:102B5000FFF7D0FF08BD114B1B78CBB1114B1B7891
:102B6000012B15D9082B13D028B1022B10D103202B
:102B7000FFF786FF08BD052B03D10720FFF780FF75
:102B800008BD033BDBB2012B02D80620FFF778FF1C
:102B900008BD00BF65BAFF1F70C2FF1F80C5FF1FC1
:102BA00055BAFF1F81C5FF1F2DE9F04F89B0804640
:102BB0000591029203939DF848200492437B019370
:102BC000002B00F0BB805F4B1B78002B00F0AE8029
:102BD0000024214622465C4F5A4D002A41D14FF431
:102BE0002C7303FB047393F89C32002B39D14FF400
:102BF0002C7A0AFB04FA07EB0A09484604F002FBA8
:102C000009F52176C646BEE80F000FC69EE8030010
:102C100086E803004FF0010B89F89CB2029A89F80C
:102C20009D22039A89F89E22002289F89F22049B04
:102C300089F8AE32484609F5217104F00FFB434A8A
:102C400013680693069BC9F8A032B9F8AA325B4410
:102C5000A9F8AA3289F8AC422046FDF74DFE21467C
:102C60005A460134E4B22B78A342B6D8002A53D195
:102C7000344B1B78002B5CD00024334F314D002A9D
:102C800044D14FF42C7303FB047393F8980298F823
:102C9000143098423AD24FF42C7B0BFB04FB07EB29
:102CA0000B06304604F0AEFA06F5217EC446BCE8B9
:102CB0000F00AEE80F009CE803008EE803004FF021
:102CC000010A86F89CA2029A86F89D22039A86F849
:102CD0009E22002286F89F22049B86F8AE32304660
:102CE00006F5217104F0BAFA184A13680793079B96
:102CF000C6F8A032B6F8AA325344A6F8AA3286F82B
:102D0000AC422046FDF7F8FD214652460134E4B2BC
:102D10002B78A342B3D87AB14FF42C720A4B02FB42
:102D20000131D1F8AA32059A136007E0002301931C
:102D300004E00022019201E000230193019809B010
:102D4000BDE8F08F249FFF1FB4AEFF1F20D6FF1FEA
:102D500000B585B00023009303A91A46FFF724FFAE
:102D600005B05DF804FB00BF00B585B0009103A974
:102D700000221346FFF718FF05B05DF804FB00BF03
:102D800000B585B00B460022009203A90122FFF78F
:102D90000BFF05B05DF804FB10B582B0144600933C
:102DA00001222346FFF700FF02B010BD00B583B03B
:102DB000009200221346FFF7F7FE03B05DF804FB14
:102DC00038B504460D464FF42C70134B00FB04300D
:102DD00004F018FA114B1B785BB955B14FF42C7203
:102DE0000D4B02FB043393F89C3213B12046FDF7E0
:102DF000D9FD4FF42C70084B00FB0430002380F801
:102E00009C3280F89D3280F89E3280F89F3280F8A4
:102E1000AE3280F8A83238BDB4AEFF1F84C2FF1FA7
:102E200038B500242546E0B22946FFF7C9FF013432
:102E3000042CF8D138BD00BF2DE9F04389B0BA4B5E
:102E40001B78002B00F0BD810024B84DB84F2646FA
:102E50004FF42C7303FB045393F89C32002B00F0C7
:102E6000A9814FF42C7808FB0458404604F080FCFC
:102E7000002840F09F81AF4B1B680093009AD8F860
:102E8000A032D31A042B40F2958198F8AE32013B60
:102E90000A2B00F22881DFE813F00B004F008D00B1
:102EA000B600C000E900F3001C0178007F00860036
:102EB000A14B1B789BB997F86D3083B14FF42C7EF2
:102EC0000EFB045E0EF5217E07F1600CBCE80F00DE
:102ED000AEE80F009CE803008EE803000FE04FF41B
:102EE0002C7E0EFB065E0EF5217E07F1180CBCE869
:102EF0000F00AEE80F009CE803008EE803004FF4DB
:102F00002C7303FB06F6A919404601F5217104F064
:102F1000A5F9884B1B680193019B2E44C6F8A0328B
:102F2000012386F89D32002386F89E3286F8AE3261
:102F30002046FDF7E1FC3DE14FF42C7303FB04F662
:102F400005EB060909F5217E07F1A80CBCE80F0086
:102F5000AEE80F009CE803008EE80300404609F548
:102F6000217104F07BF9734B1B680293029BC9F833
:102F7000A032012389F89D32002389F89E3289F816
:102F8000AE322046FDF7B8FC14E100216B4B1970FE
:102F90002046FFF715FF0DE10021684B59702046D0
:102FA000FFF70EFF06E10021644B99702046FFF702
:102FB00007FFFFE04FF42C7303FB04F605EB060953
:102FC00009F5217E07F1F00CBCE80F00AEE80F0018
:102FD0009CE803008EE80300404609F5217104F0E7
:102FE0003DF9544B1B680393039BC9F8A03201239E
:102FF00089F89D32002389F89E3289F8AE32204646
:10300000FDF77AFCD6E000234D4A13704D4A137049
:1030100020460121FFF7D4FECCE04FF42C7303FBD4
:1030200004F605EB060909F5217E07F59C7CBCE852
:103030000F00AEE80F009CE803008EE80300404656
:1030400009F5217104F00AF93A4B1B680493049BBB
:10305000C9F8A032012389F89D32002389F89E32F5
:1030600089F8AE322046FDF747FCA3E00023344A3E
:103070005370344A537020460121FFF7A1FE99E0B6
:103080004FF42C7303FB04F605EB060909F5217ECA
:1030900007F5C07CBCE80F00AEE80F009CE8030019
:1030A0008EE80300404609F5217104F0D7F8214B62
:1030B0001B680593059BC9F8A032012389F89D324E
:1030C000002389F89E3289F8AE322046FDF714FCC1
:1030D00070E000231A4A93701A4A93702046012127
:1030E000FFF76EFE66E04FF42C7303FB045393F876
:1030F0009D32002B57D04FF42C7303FB045393F8ED
:103100009E320BBB4FF42C7303FB04F6A919404607
:1031100001F5217104F0A2F8064B1B680693069B8B
:103120002E44C6F8A03245E0249FFF1FB4AEFF1F17
:103130007C9BFF1F20D6FF1F4DBAFF1FF8BBFF1F50
:103140006CC2FF1F00BBFF1F4FF42C7303FB045323
:1031500093F89F220132D2B283F89F2203F526739F
:103160009B79934211D94FF42C7303FB04F6A919F0
:10317000404601F5217104F071F8134B1B68079369
:10318000079B2E44C6F8A03214E04FF42C7303FBC7
:103190000453002283F89C2283F89D2283F89E2208
:1031A00083F89F2206E04FF42C7303FB04560023A0
:1031B00086F89C320134E4B2044B1B78A3423FF6FC
:1031C00046AE09B0BDE8F08320D6FF1F249FFF1F45
:1031D000F8B50746094D0024E6B22B7E33B12846E8
:1031E00039460BF00FFC08B9F0B205E0013405F5E3
:1031F0002C75042CF0D1FF2040B2F8BD38B1FF1F70
:1032000008B5022808D003280BD001280DD10748A3
:103210000921FFF7A9FD08BD05480A21FFF7A4FD14
:1032200008BD04480B21FFF79FFD08BD2C9DFF1F23
:10323000449DFF1F5C9DFF1F08B50248FFF788FDF6
:1032400008BD00BF749DFF1F08B50248FFF780FD51
:1032500008BD00BF8C9DFF1F08B50248FFF778FD31
:1032600008BD00BFA49DFF1F08B50248FFF770FD11
:1032700008BD00BFBC9DFF1F08B5022807D003286A
:1032800009D001280AD10648FFF762FD08BD0548AC
:10329000FFF75EFD08BD0448FFF75AFD08BD00BFFB
:1032A000D49DFF1FEC9DFF1F049EFF1F08B5014624
:1032B000012803D10348FFF74BFD08BD0148FFF784
:1032C0005FFD08BD349EFF1F08B50248FFF740FDB3
:1032D00008BD00BF4C9EFF1F08B518B10348FFF79B
:1032E00037FD08BD0248FFF733FD08BD649EFF1F90
:1032F0007C9EFF1F2DE9F04383B0F8B13E4B1B7855
:10330000002B76D13D4B93F8E5304BB13C483D491D
:103310000322FFF74BFD68B10122374B1A7009E019
:103320003948384900221346FFF736FD10B1012213
:10333000314B1A700022354B1A705AE02E4B1B7815
:10334000002B56D0314B1B78002B52D12B4B93F8CE
:103350001531002B43D02B4B9A784FF42C702C490D
:1033600000FB0211B1F8AA121B88994204D1284B24
:1033700000FB023003F046FF4FF0010C234B83F8B3
:1033800000C0DFF8809099F802E0214F4FF42C78CC
:1033900008FB0EFE07EB0E0606F521741D4D0FCD42
:1033A0000FC495E8030084E8030086F89CC200225D
:1033B00086F89D22042386F8AE32304606F5217148
:1033C00003F04CFF99F80200134B1B680193019B1B
:1033D00008FB0077C7F8A032FDF78EFA09E0094B29
:1033E00098780021FFF7ECFC0023034A1370074A8A
:1033F000137003B0BDE8F0836CC2FF1F7C9BFF1FFE
:10340000549CFF1F7CB9FF1F6C9CFF1F00BBFF1F5C
:10341000B4AEFF1F849CFF1F20D6FF1F2DE9F04391
:1034200083B0F8B13E4B5B78002B76D13D4B93F8DF
:103430002D314BB13C483D490522FFF7B7FC68B13F
:103440000122374B5A7009E03948384900221346A7
:10345000FFF7A2FC10B10122314B5A700022354B0C
:103460005A705AE02E4B5B78002B56D0314B5B786C
:10347000002B52D12B4B93F85D31002B43D02B4BBB
:103480009A784FF42C702C4900FB0211B1F8AA1263
:103490001B88994204D1284B00FB023003F0B2FE96
:1034A0004FF0010C234B83F801C0DFF8809099F8AE
:1034B00002E0214F4FF42C7808FB0EFE07EB0E06BE
:1034C00006F521741D4D0FCD0FC495E8030084E867
:1034D000030086F89CC2002286F89D22062386F807
:1034E000AE32304606F5217103F0B8FE99F80200BD
:1034F000134B1B680193019B08FB0077C7F8A032B0
:10350000FDF7FAF909E0094B98780021FFF758FC1C
:103510000023034A5370074A537003B0BDE8F08399
:103520006CC2FF1F7C9BFF1F9C9CFF1F80C4FF1F62
:10353000B49CFF1F00BBFF1FB4AEFF1FCC9CFF1F3E
:1035400020D6FF1F2DE9F04383B0F8B13E4B9B78A6
:10355000002B76D13D4B93F875314BB13C483D493A
:103560000722FFF723FC68B10122374B9A7009E06C
:103570003948384900221346FFF70EFC10B10122EA
:10358000314B9A700022354B9A705AE02E4B9B7843
:10359000002B56D0314B9B78002B52D12B4B93F8FC
:1035A000A531002B43D02B4B9A784FF42C702C492B
:1035B00000FB0211B1F8AA121B88994204D1284BD2
:1035C00000FB023003F01EFE4FF0010C234B83F88A
:1035D00002C0DFF8809099F802E0214F4FF42C7878
:1035E00008FB0EFE07EB0E0606F521741D4D0FCDF0
:1035F0000FC495E8030084E8030086F89CC200220B
:1036000086F89D22082386F8AE32304606F52171F1
:1036100003F024FE99F80200134B1B680193019BF1
:1036200008FB0077C7F8A032FDF766F909E0094BFF
:1036300098780021FFF7C4FB0023034A9370074AE0
:10364000937003B0BDE8F0836CC2FF1F7C9BFF1F2B
:10365000E49CFF1F38BAFF1FFC9CFF1F00BBFF1F2D
:10366000B4AEFF1F149DFF1F20D6FF1F08B5022810
:1036700007D0032809D001280AD10846FFF73AFEEF
:1036800008BD0846FFF7CAFE08BD0846FFF75AFF07
:1036900008BD00BFF0B583B0002844D0614B1B7853
:1036A000002B40F0BC80604B1B78002B40F0AB80BF
:1036B0005E4B93F85530002B00F0AB805C485D49C1
:1036C0000122FFF773FB002800F0A9800122554B6F
:1036D0001A70A4E0554857490122FFF767FB0028FC
:1036E00000F09D8001224F4B1A7098E04F4B93F8E9
:1036F0006D3063B150484F4900221346FFF74CFB31
:10370000002800F08C800122464B1A7087E04B485D
:10371000484900221346FFF73FFB00287FD00122D3
:10372000404B1A707BE03F4B1B78002B77D03E4B11
:103730001B781BB93D4B93F8853023B93B4B93F86D
:103740003D30002B56D03B4B9A784FF42C703C49BF
:1037500000FB0211B1F8AA121B88994204D1384B20
:1037600000FB023003F04EFD2F4B1B7883B1314B31
:103770009A784FF42C74324B04FB023404F5217414
:10378000304D0FCD0FC495E8030084E803000FE02F
:10379000284B9A784FF42C74294B04FB023404F51F
:1037A0002174294D0FCD0FC495E8030084E8030070
:1037B000204FBB78224D4FF42C7606FB03F3E8181C
:1037C000012180F89C12002480F89D4280F8AE42CE
:1037D00000F5217103F042FDB8781C4B1B68019382
:1037E000019B06FB0055C5F8A0320E4B1C70FDF77F
:1037F00083F814E00F4B98780121FFF7E1FA0022DB
:10380000084B1A700BE0094B5B7B002B3FF47FAF3A
:1038100060E7064B5B7B002B3FF468AF5AE703B0D1
:10382000F0BD00BF38ADFF1F4DBAFF1F7C9BFF1FCF
:10383000C49BFF1F94BBFF1FDC9BFF1F949BFF1FBC
:10384000B4AEFF1FAC9BFF1FF49BFF1F20D6FF1FD2
:103850002DE9F04383B0F0B1394B1B78002B6CD1CC
:10386000384B93F89D3053B1374838490222FFF75F
:103870009DFA002861D00122314B1A705DE0344876
:10388000324900221346FFF787FA002855D001225B
:103890002B4B1A7051E02A4B1B78002B4DD0294B33
:1038A00093F8CD30002B40D0284B9A784FF42C70F1
:1038B000284900FB0211B1F8AA121B88994204D1D1
:1038C000244B00FB023003F09DFCDFF8809099F858
:1038D00002E0204F4FF42C7808FB0EFE07EB0E069B
:1038E00006F521741C4D0FCD0FC495E8030084E844
:1038F0000300012286F89C22002486F89D4286F867
:10390000AE42304606F5217103F0A8FC99F802009A
:10391000124B1B680193019B08FB0077C7F8A0328C
:10392000074B1C70FCF7E8FF07E0084B9878012173
:10393000FFF746FA0022024B1A7003B0BDE8F0838D
:10394000FAC5FF1F7C9BFF1F0C9CFF1F78B9FF1F50
:10395000249CFF1FB4AEFF1F3C9CFF1F20D6FF1FFF
:1039600008B568B10C4B1B786BB90C480C490022A8
:103970001346FFF711FA70B10122074B1A7008BD08
:10398000054B1B783BB1064B98780121FFF718FADD
:103990000022014B1A7008BDFCC5FF1F1C9EFF1FB3
:1039A0005CBBFF1FF8B50D461746162824D8013812
:1039B000C4B204EB4406114B03EBC6063046FFF7D6
:1039C00007FC9DB1002817DA47B130460C4901EBDE
:1039D000840100221346FFF7DFF9F8BD304608499D
:1039E00001EB84010022FFF7E1F9F8BD002803DBB9
:1039F000C0B20121FFF7E4F9F8BD00BF5098FF1FE6
:103A000004BBFF1F0139C9B2052909D8090100EB20
:103A1000800000EB8000400000F5FA70014B585226
:103A2000704700BF8CC5FF1F0139C9B205290AD8EC
:103A3000054B03EB011100EB800000EB8000400020
:103A400000F5FA70488070478CC5FF1F0139C9B274
:103A5000052909D8054B03EB0111003018BF0120DF
:103A600008710122024B1A70704700BF8CC5FF1FFE
:103A70008DBBFF1F08B5074B1B7853B9064840F6AE
:103A8000B831064A03F042F8054B18600122014B99
:103A90001A7008BD04ACFF1F88ADFF1F4D3B00002E
:103AA00080B9FF1F10B5154A00235371537582F872
:103AB000253082F8353082F8453082F85530104A8A
:103AC00013701048104B196803F0BEF820B10D4870
:103AD0000D4B196803F034F80C4B1B7863B10C4B99
:103AE0001B784BB10B4C23685B6820460A490C22BB
:103AF0009847204607F06CFE10BD00BF8CC5FF1F25
:103B000004ACFF1F88ADFF1F80B9FF1F639AFF1F22
:103B10008DBBFF1FE4D7FF1F78FB000010B582B0FC
:103B2000084B1B6801930199074A0001131803F120
:103B300008049960105A598807F0D4FFA08002B099
:103B400010BD00BF20D6FF1F8CC5FF1F2DE9F0411F
:103B5000164B1B783BB3164E00242546154F4FF0ED
:103B60000108E8B23B191A7942B15A7932B996F88C
:103B700025231AB183F80580FFF7D0FF01351034F3
:103B80001836602CEDD10C4B1B7863B10B4B1B78B6
:103B90004BB10B4C23685B6820460A490D229847BD
:103BA000204607F015FEBDE8F08100BF04ACFF1F02
:103BB0007C9BFF1F8CC5FF1F639AFF1F8DBBFF1FE0
:103BC000E4D7FF1F88FB000010B50446094B03EB48
:103BD00000135B796BB1213000EB4000064B03EB27
:103BE000C000FFF7B5F82046FFF798FF2046FCF726
:103BF0002FFF10BD8CC5FF1F7C9BFF1F70B582B0CF
:103C00000B4D00240B4EE0B22B785BB1336801936F
:103C1000019AD5F80330D31AB5F80720934201D39F
:103C2000FFF7D2FF01341035062CECD102B070BD85
:103C300091C5FF1F20D6FF1FF0B583B00446234B6C
:103C40001B78652B06D8591C204A1170204A42F86F
:103C5000230009E01F4D2B685B6828461E493C2263
:103C60009847284607F0B4FD204604F02FFC20B307
:103C70001A4D284603F0C6FA2846214603F0EEFA0C
:103C8000174B1B680093009F154E284603F070FDEC
:103C900018B1284603F082FD206123698BB933688F
:103CA0000193019BDB1B052BEFD908E00125657310
:103CB0000A4803F0A7FA284606E0002004E00020A6
:103CC00002E0322BF2D8002003B0F0BD7CC5FF1F0C
:103CD000A4C2FF1FE4D7FF1F98FB0000B4AEFF1F74
:103CE00020D6FF1F08B5FFF79BF8FEF76FFE08BD53
:103CF00070B406460B7800250133DBB25CB2944207
:103D0000A8BF00235CB204EB440406EBC404607B50
:103D100020B90135ECB29442EED300E00B7070BCD8
:103D2000704700BF08B55C4B1B78013B072B00F2C6
:103D3000B280DFE803F004B054B0B03477A9574B39
:103D40001B78002B40F0A780FEF740FE544B1B78F9
:103D50007BB1544B5B7B23B152480121FEF718FE27
:103D600016E0514B5B7B9BB14F480121FEF710FEE3
:103D70000EE04D4B5B7B23B14B480121FEF708FE63
:103D800006E0484B5B7B1BB146480121FEF700FE75
:103D90000022434B1A700122404B1A7008BD434B5E
:103DA0001B783BB1424B5B7B23B141480021FEF7BE
:103DB000E7FD10E03F4840490522FFF799FF50B169
:103DC0003D4B93F9003003EB43033A4800EBC3004B
:103DD0000021FEF7D5FD0220FEF752FE08BD374850
:103DE00037490522FFF784FF70B1354B93F9003056
:103DF00003EB4303314800EBC3000221FEF7B8FD9B
:103E00000420FEF73DFE08BDFEF7CAFD00EB4000B2
:103E10002C4B03EBC0000321FEF7B2FD0520FEF79B
:103E20002FFE08BD284829490522FFF761FF58B138
:103E3000264B93F9003003EB4303234800EBC30008
:103E40000121FEF795FD1BE0184B1B783BB1184B89
:103E50005B7B23B116480021FEF792FD10E0154868
:103E600015490522FFF744FF50B1134B93F9003079
:103E700003EB43030F4800EBC3000021FEF780FD76
:103E80000220FEF7FDFD08BD11480421FEF770FD7C
:103E90000020FEF7F5FD08BD81C5FF1F4DBAFF1FCD
:103EA000619AFF1F68A0FF1F649AFF1F10BCFF1FCD
:103EB00050A0FF1F98A0FF1F11A1FF1F809AFF1F96
:103EC00008A2FF1F589FFF1F009BFF1F13A1FF1F8A
:103ED00080A0FF1F2DE9F04F87B0754D05F52174C7
:103EE00005F2E476DFF8E481DFF8E4A1DFF8E4919D
:103EF0002746237E002B00F0D18094F82A30042B33
:103F000000F2CC80DFE803F098033858860028469A
:103F100003F02EFC002800F0C180284603F030FC9E
:103F20002369A3F5C8739842C0F0B880614B1B7831
:103F300053B1614B5B7B3BB15F480021FEF720FD35
:103F40000220FEF79DFDA9E05C485D490522FFF7D0
:103F5000CFFE70B15A4B93F9003003EB430357483F
:103F600000EBC3000021FEF70BFD0220FEF788FDE9
:103F700094E0FEF73DFD91E0284603F0F9FB0028B0
:103F800000F08C80284603F0FBFB2369A3F5C8737F
:103F90009842C0F08380FEF703FD074600EB400027
:103FA000484B03EBC0000321FEF7EAFC464B1F70B1
:103FB0000520FEF765FD71E099F80030052B6DD105
:103FC000FEF7EEFC8346404B1B7883420BD000EBA0
:103FD00040003C4B03EBC0000321FEF7D1FC3A4B01
:103FE00083F800B05AE0284603F0C2FB002855D100
:103FF000D8F800300093009AE369D31A042B4DD906
:104000002846214603F02AF9D8F800300193019B95
:10401000E36143E0284603F0ABFB00283ED1D8F82B
:1040200000300293029AE369D31A042B36D9002395
:1040300023768AF8003031E0AB46284603F098FB3F
:10404000A8B9D8F800300393039AE369D31A042B74
:104050000DD9637E4BB12846214603F0FFF8D8F80E
:1040600000300493049BE36101E00023237658466B
:1040700003F07EFB90B13B7E83B197F824306BB1A7
:10408000D8F800300593059A3B6A934206D058460B
:1040900003F0B8F800233B7687F8243005F52C753B
:1040A00004F52C74B4427FF423AF07B0BDE8F08F61
:1040B00068BCFF1F10BCFF1F50A0FF1F98A0FF1F70
:1040C000FE9AFF1F589FFF1F5CBAFF1F20D6FF1FDD
:1040D0004DBAFF1F81C5FF1F044B1B78022B0CBF7D
:1040E00003220222014B1A70704700BF12A1FF1F6A
:1040F0002DE9F04F83B00546894617469846467B22
:10410000002E00F08980464B1878DFF82CB18BF830
:104110000000444C4FF42C7A0AFB004003F072F884
:104120009BF800C00AFB0C4E0EF521740FCD0FC496
:1041300095E8030084E8030001228EF89C228EF8A3
:104140009D928EF8AE8257B1ACF1020C0CEB8C0C48
:10415000354800EBCC00354902F0EEFD0AE0ACF149
:10416000020C0CEB8C0C304800EBCC0030490122E7
:1041700002F0E2FDDFF8C08098F80000294C4FF40F
:104180002C7505FB00F02118084601F5217103F09C
:1041900065F898F80000274B1B680093009B05FB0F
:1041A0000044C4F8A032B4F8AA320133A4F8AA3209
:1041B00084F8AC02FCF7A0FBFFF78EFF67B3184B47
:1041C0001A78184B05FB023003F0D2FA054618B3F3
:1041D000134C2378023B03EB8303134800EBC3002B
:1041E0001249002202F0A8FD2378124A12680192B7
:1041F000019A4FF42C700B4900FB031302F5C872AF
:10420000C3F8A42203F52A71012283F8A822002210
:1042100083F89D228A712E46304603B0BDE8F08FA8
:1042200012A1FF1FB4AEFF1FA8BBFF1F16B70300EC
:104230005D74D10520D6FF1F609AFF1F08B50B469D
:1042400000210122FFF754FF08BD00BF08B50B464F
:1042500001210A46FFF74CFF08BD00BF08B50B4619
:1042600000210A46FFF744FF08BD00BF054B187048
:1042700018B10122044B1A7070470022024B1A70C9
:10428000704700BF5EBAFF1FA4B9FF1F00B583B01F
:10429000074B1878074B1B78013B00930021FF2246
:1042A0000B4607F029FCC0B203B05DF804FB00BF69
:1042B0005EBAFF1F05ACFF1F08B502200021FEF704
:1042C0007FFD03200021FEF77BFD0222014B1A70C7
:1042D00008BD00BF12A1FF1F08B51D4B1B78002BA6
:1042E00035D01C4B1B7873BB1B4B1B787BB3022256
:1042F0001A4B1A70FFF7E0FF194B5B7B23B118488C
:104300000121FFF7ABFF09E0FFF7C0FF00EB400022
:10431000144B03EBC0000221FFF798FF01220D4B65
:104320001A7010E0104B5B7B23B10F480321FFF79D
:1043300085FF04E0FFF7C0FF0422084B1A7000223B
:10434000044B1A7008BD044B1B78002BEAD008BD43
:104350008EBBFF1F70ADFF1FA4B9FF1F249FFF1F5F
:10436000409FFF1F18A1FF1F289FFF1F2DE9F04F3F
:1043700087B05C4B03F5AC6403F2E47503F52C677E
:10438000DFF86891DFF868A1DFF86881264694F8C5
:104390009C22002A00F09B8094F8AE32032B00F29E
:1043A0009680DFE803F05C021D48204603F0E0F948
:1043B000002800F08C80204603F0E2F9D4F8943213
:1043C000A3F5C8739842C0F08280FFF75FFF00EB4F
:1043D0004000454B03EBC0000221FFF737FF76E0BA
:1043E000FFF754FF834698F8003083420AD000EB71
:1043F00040003D4B03EBC0000221FFF727FF88F888
:1044000000B064E0204603F0B3F900285FD1D9F88A
:1044100000300093009AD4F8A032D31A042B56D956
:104420002046294602F01AFFD9F800300193019B7B
:10443000C4F8A0324BE0204603F09AF9002846D198
:10444000D9F800300293029AD4F8A032D31A042B80
:104450003DD9FFF731FF04238AF8003037E02046CA
:1044600003F086F9C8B9D9F800300393039AD4F859
:10447000A032D31A042B10D994F89D3253B12046A0
:10448000294602F0EBFED9F800300493049BC4F8EF
:10449000A03202E0002384F89C32304603F068F931
:1044A000A8B196F89C3293B196F8A8327BB1D9F8AE
:1044B00000300593059AD6F8A432934207D03046CF
:1044C00002F0A0FE002386F89C3286F8A83204F59C
:1044D0002C7405F52C75BC427FF458AF07B0BDE8CD
:1044E000F08F00BFB4AEFF1F18A1FF1F20D6FF1F23
:1044F000249FFF1F7CC4FF1F10B5114C23685B680D
:104500002046104900229847204607F061F9FCF741
:1045100041FB23685B6820460B49122298472046DE
:1045200007F056F9FCF736FB23685B68204607491D
:104530001B229847204607F04BF9FCF72BFB10BDD8
:10454000E4D7FF1F28FC0000D8FB0000ECFB0000B4
:1045500038B5114C2368114D5B682046294600226E
:104560009847204607F034F9FCF714FB23685B6892
:1045700020460B4910229847204607F029F9FCF7FE
:1045800009FB23685B68204629460022984720469D
:1045900007F01EF938BD00BFE4D7FF1F28FC00005C
:1045A00008FC000070B506460024174D2B681B68F8
:1045B0002846315D984701340D2CF7D10620FCF7D1
:1045C00063FB737B63B13069FCF788FA0620FCF764
:1045D0005BFB0D4803685B680C490C22984770BD73
:1045E000094C23685B6820460949012298470D2041
:1045F000FCF74AFB23685B68204606490922984776
:10460000204607F0E5F870BDE4D7FF1F1CFC000052
:1046100044F400002CFC000010B584B0404803F0C6
:10462000A7F8002844D13F4B1B78002B40D03E4BCD
:104630001B680093009A3D4B1B68D31A642B37D933
:104640003B4B1B781BB90122394B1A7011E0394BD7
:10465000B3F90020384B53F822305B7B4BB1374C19
:1046600023685B682046364904229847204607F0B5
:10467000AFF800222B4B1A702B4B1B680193019A49
:10468000304B1A602B4B1B8801339BB21AB2652A40
:1046900002DC284A13800BE00022264B1A80274CAC
:1046A000204607F095F8FCF775FA204607F090F8D9
:1046B0001B4803F05DF8002830D11A4B1B78002B03
:1046C0002CD1194B1B680293029A1E4B1B68D31AFC
:1046D000B3F5487F22D9174BB3F90020164B53F896
:1046E000220003F0F3FE70B1124BB3F900200C4826
:1046F000114B53F8221002F0B1FD0B4B1B680393D2
:10470000039A0A4B1A600122064B1A70094BB3F93F
:104710000020094B53F82200FFF744FF04B010BDFE
:10472000B4AEFF1F789BFF1F20D6FF1F74B9FF1F79
:10473000FEBBFF1FFC9AFF1FA4C2FF1FE4D7FF1F91
:1047400038FC000024C5FF1F38B505460D4B1B780B
:104750000D4A12789A420BD00B4A13700B4C236807
:104760005B6820460A491D229847204607F030F82A
:10477000284609F06FF8074909F078F9064B1860E8
:1047800038BD00BF4CA0FF1F5FBAFF1FE4D7FF1F5B
:1047900040FC00000000C84214BCFF1F10B50246D8
:1047A00043780F3B412B00F20A81DFE813F042000F
:1047B00008010801080108010801080108010801B1
:1047C00008010801080108010801080108010801A1
:1047D0000801080108010801080108010801080191
:1047E0000801080108010801460049004C0050007A
:1047F00058005C00600064006A006D0077009C0057
:104800009F00A300A700AB00AF00B700BD00C3002E
:10481000C900CC00CF00D400D900DE00E200E900DE
:10482000E60086008F005400ED00FB0067000201E7
:10483000B3008078FDF75EFA10BDFEF75BF910BD9E
:10484000FEF768F910BD8078FEF770F910BD002002
:10485000FEF76CF910BD8078FFF708FD10BD012050
:10486000FFF77EF810BD0020FFF77AF810BD012099
:10487000FEF7C6FC10BDFEF7DFFC10BDFEF7E4FC42
:1048800010BDFEF7F1FC10BD4D4B1B78002B40F026
:10489000968001200146FEF7E9FE10BD484B1B78CB
:1048A000002B00F08C80474B1B78002B40F087805A
:1048B00001200021FEF7DAFE10BD414B5B78002B92
:1048C0007DD102200121FEF7D1FE10BD3C4B5B786B
:1048D000002B74D03B4B5B78002B70D10220002161
:1048E000FEF7C4FE10BDFEF7B7FC10BD0120FEF7B9
:1048F000D1FE10BD0020FEF7CDFE10BD0120FEF759
:10490000A7FF10BD0020FEF7A3FF10BD0120FEF79A
:10491000B3FC10BD0220FEF7AFFC10BDC078012132
:104920000022FFF73FF810BDC07801210A46FFF7CB
:1049300039F810BDC07800210A46FFF733F810BDE2
:10494000FFF798F810BDFFF7ADF810BD8078D1786B
:10495000FFF758F810BD8078D178FFF765F810BDE3
:104960008078D178FFF772F810BD0120FEF79EFC29
:1049700010BD8078FEF79AFC10BDFEF7A5FC10BDB7
:104980008078FFF7E1FE10BDC47880786428A8BF66
:10499000642008F05FFF0C4909F068F80B4B43F8FE
:1049A000240010BD8078003018BF0120FEF794FC71
:1049B00010BD8278003218BF0122054B1A7010BD5D
:1049C0006CC2FF1F00BBFF1F0000C8424098FF1FC2
:1049D00010BCFF1F70B582B0244C254D254E13E04E
:1049E00005F0A6FDC0B2DA2805D101232370DA2232
:1049F00032702B7008E0237833B12A78531CDBB275
:104A00002B70B054042B03D805F082FD0028E7D1A9
:104A1000174B1B78042B25D91748164B1A780270B0
:104A20005A7842709A788270DA78C2701B79037172
:104A3000FDF750F968B1114B1B680193019A104BB7
:104A40001A60104801F002FE0B48FFF7A7FE012094
:104A500000E000200023074A1370044A1370044A40
:104A6000137000E0002002B070BD00BF8CBBFF1FC0
:104A700088C5FF1F08C5FF1FECC5FF1F20D6FF1FFD
:104A800088C2FF1F60BBFF1F38B505460D4B1B7862
:104A90000D4A12789A420BD00B4A13700B4C2368C4
:104AA0005B6820460A4919229847204606F090FE86
:104AB000284608F0CFFE074908F0D8FF064B1860DB
:104AC00038BD00BF09A2FF1F5FBAFF1FE4D7FF1F59
:104AD00060FC00000000C84214BCFF1F2DE9F04339
:104AE00083B00446064600EB4002B04B03EBC20322
:104AF0005B7D002B00F0DD80FDF71EF8C0B204EBFB
:104B00004403AA4A02EBC3039B7A834200F06F81FD
:104B100004EB440402EBC404A072A54B1B78002BE9
:104B200000F065810024A34D06EB460702EBC707A2
:104B3000A04604EB8403EA5C731C9A4240F0B18007
:104B400004EB84032B445A78BB7A9A4240F0A98044
:104B500004EB84032B4493F803909B78013B062BD2
:104B600000F29F80DFE803F004070A132A6E810039
:104B7000FDF7C0FF95E0FDF7CDFF92E08E4B1B786F
:104B800013B1FDF7C7FF8CE0FDF7B4FF89E009F131
:104B9000FF338A4AD25C002A40F083800121874A91
:104BA000D1544846FEF72CFB48460621FCF728FD69
:104BB000B9F1010F75D1FDF7C5F872E004EB840877
:104BC00005EB08031B79022B12D0032B23D0012BFA
:104BD00067D17B4B4B4413F8013C002B61D1484615
:104BE0000121FEF743FD48460421FCF709FD58E08A
:104BF00009F1FF33724AD25C002A52D0714AD35C69
:104C0000002B4ED148460021FEF730FD48460221D8
:104C1000FCF7F6FC45E06A4B4B4413F8013C43B10A
:104C200048460021FEF722FD48460221FCF7E8FC39
:104C300037E048460121FEF719FD48460421FCF7FC
:104C4000DFFC2EE004EB84032B441B79013B022B99
:104C500002D84846FEF710FB08EB880805EB08036E
:104C600048461979FCF7CCFC1BE004EB840805EB03
:104C700008031B79022B09D0032B0DD0012B10D177
:104C8000484601210022FEF78DFE0AE04846002139
:104C90000A46FEF787FE04E0484601210A46FEF771
:104CA00081FE0134E4B2424B1B78A3423FF640AF91
:104CB0009DE000EB40033D4A02EBC3035888B0F58A
:104CC0007A7F05DBB0F5FA6FA8BF4FF4FA6001E018
:104CD0004FF47A7004EB4403344A02EBC303588068
:104CE0009B7D012B22D0022B40F081806423009316
:104CF0004FF47A714FF4FA62002306F0FDFE04EBE4
:104D000044032A4A02EBC3031A7AC3B2D31A002B14
:104D1000B8BF5B42052B6ADDC0B204EB4404234BF1
:104D200003EBC4031872FFF7AFFE60E0264B1B785D
:104D30007BB1A0F2DC500028B8BF4042FF230093B3
:104D400000B200214FF4FA720B4606F0D5FEC0B255
:104D50001BE004EB4403154A02EBC303DB7953B1B8
:104D6000FF2300934FF47A714FF4FA62002306F0A8
:104D7000C3FEC0B209E0002300934FF47A714FF4F0
:104D8000FA62FF2306F0B8FEC0B204EB4403074A00
:104D900002EBC3031B7A1B1A002BB8BF5B42032B29
:104DA00016DC0A4B1B78834221D917E088C4FF1F09
:104DB00084C4FF1F68BAFF1F4DBAFF1FF8BBFF1F57
:104DC0006CC2FF1F00BBFF1FF89AFF1F4DA0FF1F03
:104DD000084B1B78834288BF002000E0002004EBD2
:104DE0004404054B03EBC4042072FDF79FFE03B09F
:104DF000BDE8F0834DA0FF1F88C4FF1F2DE9F047D9
:104E0000464CA61D0C340025A4F10C0808F16107DE
:104E1000DFF81C91E8B2A24614F8063C002B72D0D1
:104E200034F8083CA3F5487292B2B2F5AF6F1FD8C0
:104E300024F80A3CD6F80630636014F80B3C012BCA
:104E400003D05BB1022B03D02CE0FFF747FE29E033
:104E5000002304F80B3C0123237223E0237A01335F
:104E6000DBB22372042B1DD9012304F80B3C19E09B
:104E7000D6F806206368D31A29498B4212D9294BE8
:104E80001B7823B118B9002304F80B3C07E0264B2C
:104E90001B78012B14BF002302230AF80B3C0023CC
:104EA0008AF8083000210AF8061C08F101034FF0C7
:104EB000010C1A78187E904204BF0CF1010C5FFAC5
:104EC0008CFC012A08BF01211833BB42F1D198F8AC
:104ED0007930012B1ED0BCF1050F04D198F80130B8
:104EE00089F8003007E019B1012389F8003002E0A9
:104EF000022389F8003099F800200C4B1B789A4265
:104F000001D0FCF797FD013518361834052D81D1F5
:104F1000BDE8F087BCF1050FE6D1DFE788C4FF1FCD
:104F2000A086010084C2FF1F70C2FF1FFDBBFF1FD0
:104F300000C5FF1F70B5172004F06EFD0446164B28
:104F40001B78164A12789A4208D0154A1268821ABB
:104F5000002AB8BF52424B2A0CDC70BD204608F034
:104F60007DFC4FF06A5108F0CDFC0E4B18600C4BE5
:104F70001C6070BD094E33700B4D2B685B68284672
:104F80000A491B229847284606F022FC3278024B39
:104F90001B789A42E2D070BD4CBAFF1F5FBAFF1F68
:104FA00060BAFF1F14BCFF1FE4D7FF1F7CFC00008A
:104FB00008B5084B1B78012B02D0022B05D008BD89
:104FC0000520002104F0A4FE08BD0E20012104F0FC
:104FD0009FFE08BDFA9AFF1F08B5084B1B78012BEE
:104FE00002D0022B05D008BD0520012104F090FE5F
:104FF00008BD0E20002104F08BFE08BDFA9AFF1FA9
:105000002DE9F04F85B000238DF80C308DF80D3070
:105010008DF80E308DF80F30FFF78CFF8B4B93F827
:105020009C321BB9894B93F84C354BB101278DF855
:105030000C70874B1868002108F05CFB064601E005
:1050400000270026834B93F89C32019323B9814BB0
:1050500093F84C353BB943E07E4B93F84C352BB974
:105060004FF07E5904E04FF07E5901E04FF07C593B
:10507000794B93F80080794D0024DFF804A24FF0BB
:105080008F4BB8F1000F17D0032C1AD84846514661
:1050900008F0F4FD30B94846714908F0D1FD18B95F
:1050A000484602E0504600E06D48594608F02AFCA8
:1050B00008F0EEFDA86104E0032C9CBF4FF48033A0
:1050C000AB6101340435042CDBD101238DF80D30A4
:1050D00030465F4B596808F00DFB06460137FFB2BA
:1050E000604B1B7873B1604A12785AB13046584B06
:1050F000996808F0FFFA064601238DF80E301F4428
:10510000FFB25BE0534A92F8FC2722B9514A92F869
:10511000AC2A002A52D073B9019BABB14D4B93F826
:105120004C358BB130464A4B596808F0E3FA0646D5
:105130004FF07C5910E03046454B996808F0DAFA98
:1051400006464FF07E5907E03046414B596808F05B
:10515000D1FA06464FF07E593F4B93F80080434DFD
:105160000024DFF81CA14FF08F4BB8F1000F17D0CF
:10517000032C1AD84846514608F080FD30B94846FD
:10518000374908F05DFD18B9484602E0504600E096
:105190003348594608F0B6FB08F07AFDA86104E0F0
:1051A000032C9CBF4FF48033AB6101340435042CD5
:1051B000DBD101238DF80E301F44FFB22C4B93F846
:1051C000303013F0FF0F0AD03046214BD96808F079
:1051D00091FA064601238DF80F301F44FFB2254B8C
:1051E0001868254B196808F035FD10B1FFF7E0FE8F
:1051F00005E017B9FFF7DCFE03E0FFF7EDFE012F36
:1052000040D81C4B1E681D4D00241D4F4FF08F4889
:10521000DFF84C90032C14D83046394608F02EFDA8
:1052200030B93046494608F00BFD18B9304602E067
:10523000384600E04846414608F064FB08F028FD87
:10524000A86101340435042CE4D184E068BCFF1F5C
:105250004098FF1FB4AEFF1F54BAFF1F08ACFF1FDA
:1052600000FEFFC68EBBFF1F4DBAFF1F40ACFF1FE5
:10527000B4ACFF1F14BCFF1F10C5FF1F7CACFF1F89
:1052800000FEFF463046002108F0F8FC00285CD004
:1052900030464FF07E5108F0D3FC08B14FF07E56F7
:1052A0002E4B93F800B02E4BD3F800902D4D0024D8
:1052B000DFF8BC804FF08F4A03ABE35C002B3BD0A0
:1052C000BBF1000F20D04846274B53F8241008F0BC
:1052D00019FB314608F0CAFB0746032C30D841467B
:1052E00008F0CCFC28B93846204908F0A9FC10B9D0
:1052F00002E0474600E01D4F3846514608F002FBE9
:1053000008F0C6FCA8611BE0032C19D848464146AA
:1053100008F0B4FC30B94846144908F091FC18B9BB
:10532000484602E0404600E01048514608F0EAFADC
:1053300008F0AEFCA86103E0032C9CBF0023AB6126
:1053400001340435042CB7D105E0064B00229A61E4
:10535000DA611A625A6205B0BDE8F08F54BAFF1FD5
:1053600014BCFF1F7CACFF1F4098FF1F00FEFFC650
:1053700000FEFF4610B582B0594B1B78012B5FD061
:1053800013B1022B45D05FE0FFF724FBFFF736FD9A
:10539000544B1B78012B17D10122514B1A70524BE1
:1053A0001B78002B2ED0514C23685B682046504957
:1053B00015229847204606F00BFA204606F008FA18
:1053C000204606F005FA1AE04A4B1B68BBB10222E0
:1053D000434B1A70FCF7B8FA434B1B787BB1434C34
:1053E00023685B682046444919229847204606F006
:1053F000EFF9204606F0ECF9204606F0E9F9384BC3
:105400001B780BB33D4801F019F93D4801F01EF936
:105410001AE03C4B1B780BB9FFF7DCFA384801F077
:10542000DBF888B9384B1B680193019A314B1B6834
:10543000D31AB3F57A7F07D9314801F063F903E055
:10544000FFF7DCFCFCF71EFB304801F097FB2B4814
:1054500001F066F92A4801F063F92D4C204601F06D
:105460005FF904F12C0001F05BF904F1580001F040
:1054700057F9FFF7C5FD234B1B7893B1254B1B78DC
:1054800063B90122234B1A701C4801F0D7F81C485D
:1054900001F0D4F8FEF726FCFFF72EF8FFF7BCF872
:1054A0001CE01C4B1B786BB100221A4B1A701A4877
:1054B00001F0A8FEFFF74CF8094B1B7813B90F4811
:1054C00001F020F9FEF72EFCFEF704FDFEF704FFC5
:1054D000FEF74CFFFDF7B0FCFEF790FB02B010BDED
:1054E00070C2FF1F00C5FF1F639AFF1FE4D7FF1F95
:1054F00098FC000088C2FF1FB0FC00003CADFF1FFD
:1055000060BBFF1F84C2FF1F20D6FF1F88ADFF1F97
:10551000CCC1FF1FFCBBFF1FB4AEFF1F08B50022AC
:10552000024B1A60FFF76CFD08BD00BF14BCFF1FE3
:1055300070B5FFF7F3FFFFF73BFD4748FEF77CFB35
:105540004648FEF779FB464C04F178052046FEF705
:1055500073FB1834AC42F9D14248FEF76DFB424C64
:1055600004F178052046FEF767FB1834AC42F9D108
:105570003E4C04F1F0063E4D2046FEF75DFB10B1B7
:105580002B7801332B701834B442F5D1394C04F127
:1055900078052046FEF750FB1834AC42F9D1364866
:1055A000FEF74AFB3548FEF747FB354C04F1F006A1
:1055B000344D2046FEF740FB10B12B7801332B70A1
:1055C0001834B442F5D13048FEF736FB2F4C04F5C1
:1055D0006A752046FEF730FB1834AC42F9D12C4CEA
:1055E00004F504752046FEF727FB1834AC42F9D1C8
:1055F000284B00210A4683F89C2283F89D2283F8D9
:105600009E2283F89F22A3F8AA2283F8AC1283F883
:10561000AE2283F8A822013103F52C730429EAD1C4
:105620001D4B002283F89C2283F89D22A3F8AA2216
:1056300083F8AC2283F8AE2283F8A82283F84C25A5
:1056400083F84D25A3F85A25012183F85C1583F8CA
:105650005E2583F8582570BD68A0FF1F649AFF1F60
:1056600098A0FF1F50A0FF1F809AFF1F589FFF1F89
:1056700090BBFF1F009BFF1F80A0FF1F409FFF1FCD
:1056800018A1FF1F05ACFF1F289FFF1F7C9BFF1F5A
:105690005098FF1FB4AEFF1F68BCFF1F70B590B0DD
:1056A00041F2883004F0BAFC0620022104F062FBCB
:1056B0000A2004F041FC062004F04EFB60B10122F8
:1056C000AC4B1A70AC4AAD4B1A600E22AC4B1A7040
:1056D0000F22AC4B1A700BE00222A64B1A70AA4A9A
:1056E000A64B1A600F22A64B1A700A22A54B1A70FD
:1056F000A04B1B78012B12D1A448002101F00CFD16
:10570000322004F019FC0520012104F033FB0520B0
:10571000012104F0FDFA0A2004F00EFC10E0012B38
:105720000ED90E20012104F025FB0E20012104F0EA
:10573000EFFA0A2004F000FC9448022101F0ECFC8E
:1057400093480C2105F048FEFFF75AFC914B1322B9
:105750001A7012221A76112283F83020102283F850
:105760004820884A127883F86020FCF793F8FCF709
:10577000BFF889481521002200F010FF8748142146
:10578000002200F00BFF864C20460521002200F08D
:1057900005FF04F12C000421002200F0FFFE04F1BB
:1057A00058000321002200F0F9FE0820012104F036
:1057B000E1FA7C48082101F09BF81720022104F04F
:1057C000D9FA794B1B7803F0FE01784A126812F47B
:1057D000805F02D08B4240F06A81734A117003F0FF
:1057E000FC027248006810F4805F02D0914240F0E1
:1057F00068816D490A7003F0F8036C49096811F477
:10580000805F02D09A4240F06681674A13705C4C18
:105810002078012104F0AEFA2078012104F078FA12
:10582000207802F0F1FF10BB5B4828210A4600F007
:105830004FFF5F4B1B680093009D5D4C564E3046FA
:1058400000F06EFF23680193019B5B1BB3F57A7F29
:10585000F5D9584D2B685B6828465749362298473A
:10586000284605F0B5FF23680293029DE7E74FF451
:10587000FA7004F061FBFFF75BFE504B1B7833B10D
:10588000FBF7A2F94D4B1B780BB1FBF735FAFAF792
:105890006BFFFAF79FFF4A4B00221A705A709A70FA
:1058A000FCF710FB474B93F84130032B02D84648D6
:1058B00002F0A2FF434C03A82146A27E02F02AFD7B
:1058C0009DF8103084F82030059B63629DF81830F5
:1058D00084F82830079BE362089B2363099B63637A
:1058E0000A9BA3630B9BE3639DF8303084F8403040
:1058F0009DF8313084F8413010AB53F80E5D586894
:105900009968C4F84250C4F84600C4F84A101B7B9A
:1059100084F84E3003A802F05BFE94F84130032B6C
:1059200009D820460023E3762849502200F086FB60
:10593000002870D152E00122224BDA761D4C2368F8
:105940005B68204622490A229847224B1D68284658
:1059500009F0C4F9024623685B6820462946984747
:1059600023685B6820461C4910229847204605F0B2
:105970002FFF80E0FA9AFF1F0AD7A33C10C5FF1F34
:10598000FB9AFF1F259FFF1FA69BC43B50C2FF1F12
:105990000082FF1F88C4FF1F3CADFF1F60BBFF1FBD
:1059A000CCC1FF1F9CC2FF1FE0D7FF1F3C800440FB
:1059B00020D6FF1FE4D7FF1FCCFC0000639AFF1F17
:1059C0006CC2FF1F28C5FF1F44C5FF1F18BCFF1F67
:1059D00004FD000048A0FF1F10FD0000444C236898
:1059E0005B68204643490A229847434D284609F000
:1059F00075F9024623685B68204629469847236864
:105A00005B6820463D490D2298472846E97E0122E1
:105A100000F078FC2FE00122394B1A70FCF71AFBDA
:105A2000FBF7B8F8324C23685B68204635492222E0
:105A30009847204605F0CCFE23685B682046324933
:105A400016229847204605F0C3FEFBF7A3F8FBF7A4
:105A5000BFF9FBF71BFAFBF783FAFBF7CDFAFBF76D
:105A600067FBFBF7F1FCFBF7E9F8204605F0B0FE19
:105A7000204605F0ADFE254A4FF480339361D36193
:105A800013625362224A9361D36113625362214AC3
:105A90009361D361136253620E2003F0BDFF05F0E2
:105AA000DFFF1D4800F02EFEFAF75EFD1DE04FF40B
:105AB000A2701A4A10604FF41070A2F57F62106055
:105AC0008BE64FF4A270164908604FF40070A1F500
:105AD0007F6108608DE64FF4A271124A11604FF4A5
:105AE0001071A2F57F6211608FE610B070BD00BF2B
:105AF000E4D7FF1F04FD000028C5FF1F24FD0000A0
:105B000068ADFF1F34FD000058FD000008C6FF1FF0
:105B100008ACFF1F40ACFF1F3CADFF1F08C0044096
:105B20000CC0044004C004402DE9F04F89B0BB48CC
:105B300000F07CFFBA4C2046BA4B1968002213468D
:105B400000F0F6F92046B849B84A08F0E7F8B84C32
:105B500004F52C652046FAF7DFFD04F52C74AC4201
:105B6000F8D1B24C0020B349224608F0D7F8B24F22
:105B70003846FAF7D1FD07F52C7B5846FAF7CCFDED
:105B80000020AE49224608F0C9F8AD4800210A4677
:105B9000FAF76EFDAB4BAA4A1360002494611046DD
:105BA00001F01CFFA84E3046012106F12402FAF74D
:105BB0005FFDDFF81493C6F800904FF0FF38C6F889
:105BC000188006F1280A5046012106F14C02FAF726
:105BD0004FFDC6F82890C6F840809C4D284601210C
:105BE00005F12402FAF744FDC5F80090C5F81880C5
:105BF00005F12800012105F14C02FAF739FDC5F83D
:105C00002890C5F840809248FAF756FDDFF8BC921C
:105C10004846FAF751FD8F48FAF74EFDDFF8B0829B
:105C20004046FAF749FD8C48012100F11802FAF7C5
:105C30001FFD8A4B884A1360104601F0B1F988486D
:105C40000760466004724472C46005F0B7FC854882
:105C500007604660012707724472C46005F0AEFC1D
:105C60008148C0F800B0C0F804A004724472C46057
:105C700005F0A4FC7D48C0F800B0C0F804A007728D
:105C80004472C46005F09AFC79480660704B43602A
:105C900004724472C46005F091FC7648C0F800A01C
:105CA0006B4A426004724772C46005F087FC724818
:105CB0005F4E0660C0F8049004724472C46005F040
:105CC0007DFC6E480660C0F8049007724772C4609D
:105CD00005F074FC6A4806F52C7AC0F800A0C0F8FC
:105CE000049004724FF002034372C46005F066FC36
:105CF0006448C0F800A0C0F8049007724FF0030B8E
:105D000080F809B0C46005F059FC5F4806F5AC6A3C
:105D1000C0F800A0456004724472C46005F04EFCF7
:105D20005A48C0F800A0456007724472C46005F08C
:105D300045FC574806F50166066005F128024260F9
:105D400004724472C46005F039FC5248066005F1E3
:105D50002803436007724472C46005F02FFC4E486C
:105D600005603C4A426004724472C46005F026FC3F
:105D70004A4805F128030360364A426004724772BC
:105D8000C46005F01BFC4648314B0360C0F804803A
:105D900004724472C46005F011FC4248C0F80090DF
:105DA000C0F8048004724772C46005F007FC3E48E6
:105DB000284A0260C0F8048004724FF00203437264
:105DC000C46005F0FBFB39481D4A0260C0F804803E
:105DD000047280F809B0C46005F0F0FB3448C0F8E4
:105DE00000801D4B436004724472C46005F0E6FB02
:105DF000304B1A78304B1A70304B1A68079207995B
:105E00002F4A116019680691069951601A68059227
:105E100005992C4A11601B685CE000BF88ADFF1F2C
:105E200028C5FF1F48A0FF1F655F00003C98FF1FAB
:105E3000B4AEFF1F8D04000068BCFF1F65040000A6
:105E4000B4ACFF1FA0000100E8ACFF1FA8BBFF1F00
:105E500008C6FF1F40ACFF1F50C2FF1F800001009B
:105E600084B9FF1F94B9FF1F98BBFF1FA8B9FF1F7C
:105E7000B8B9FF1FC8B9FF1FD8B9FF1FE8B9FF1F86
:105E8000F8B9FF1F3CC4FF1F4CC4FF1F08BAFF1F17
:105E90006CC4FF1F18BAFF1F28BAFF1F00BCFF1FEA
:105EA0005CC4FF1F14C5FF1F3CBAFF1F74C2FF1F55
:105EB0008CC2FF1F4CBAFF1F5FBAFF1F20D6FF1F07
:105EC0003CADFF1F60BBFF1F6000010008ACFF1F5F
:105ED0007CACFF1F0493049B5360114D05F12C0310
:105EE0002E46B0350F4AA3F1280411680391039997
:105EF00043F82C1C116802910298991B214441F827
:105F00002C0C2C33AB42F0D1074800F06FFC054B52
:105F10001B680193019A054B1A6009B0BDE8F08F28
:105F2000CCC1FF1F20D6FF1F9CC2FF1F84C5FF1FCF
:105F3000F8B504460D4617461E461C3002F038FBE5
:105F4000284608F0CBFE1A2804D82046294608F037
:105F500067FE01E000232370A77684F85060204696
:105F6000F8BD00BF10B504461C3002F031FB2046DE
:105F700010BD00BF2DE9F04104460F4615461E46F0
:105F800090F82500032848D8022A49D920461968E4
:105F900002F006FC002846D0204639462A4602F088
:105FA00023FB804638B1013D27D03B780A2B41D0F6
:105FB0000D2B1BD13AE000233B700720BDE8F08198
:105FC000104612F8011B0A2936D00D2910D12FE0F6
:105FD000002202705A1CB85C884218BF1A46336807
:105FE00001331A4432600020BDE8F0817A1C00239E
:105FF0000133984501D0AB42E2D123689B6820462B
:10600000984728B9002307F808300720BDE8F08139
:1060100000237B550320BDE8F0810220BDE8F0811C
:106020000320BDE8F0810420BDE8F081384600235C
:106030000A21CDE7384600230D21C9E72DE9F041BB
:1060400082B080460F46164602AC002344F8043D59
:1060500000F11C052846394632462346FFF78AFFE1
:106060000028F7D0072804D1002388F81B3001202E
:1060700002E088F81B00002002B0BDE8F08100BFFC
:106080003B2804D0232814BF0020012070470120A2
:10609000704700BF38B5044625460134287807F01C
:1060A0007DFE0028F8D1284638BD00BF70B50546F2
:1060B00008F014FE01382C180AD2002602E066709F
:1060C000A54205D814F8010907F068FE0028F6D1AA
:1060D00070BD00BF2DE9F041054614460F4619B9C1
:1060E0000523C376012445E01C3011461A46069B61
:1060F000FFF740FF064690B3072830D0E87601242A
:1061000038E05B2C22D108F10100FFF7C3FF804685
:106110005D2108F0FDFB0346C0B10022027040463D
:10612000FFF7C4FF95F850403CB14046394608F0AF
:1061300069FC58B90023EB761CE04046394608F06C
:10614000C5FB18B90023EB76012413E0072E03BF2B
:106150000523EB76012400240CE000240AE020460D
:10616000FFF798FF804604782046FFF789FF002854
:10617000F3D1C6E72046BDE8F08100BF2DE9F84322
:1061800005460F461C4616460AB112781AB9062370
:10619000EB7601245DE01C301946089A0A9BFFF754
:1061A000E9FE804600283ED0072847D0E876012443
:1061B0004FE00623EB7601244BE02FB15B2C03D19B
:1061C0000623EB76012444E048463D2108F0A0FB7D
:1061D0000746F0B1002303704846FFF767FF95F8C4
:1061E000504054B14846314608F00CFC88B901379C
:1061F000099B1F600023EB762BE04846314608F0F0
:1062000065FB30B90137099B1F600023EB76012441
:106210001FE0B8F1070F03BF0623EB76012400242B
:1062200017E0002415E02046FFF734FF814604788C
:106230002046FFF725FF0028F3D1BEE72046FFF7F1
:1062400029FF814604782046FFF71AFF0028B0D1C5
:10625000B3E72046BDE8F88370B586B004461E4615
:106260000B9D90F84100032803D90223E376012017
:1062700045E0287901280BD010B1022815D035E06F
:10628000002914BF012302232B710020286036E06F
:10629000009520461A460A9BFFF71CFF50B3E37E89
:1062A00063BB02232B71002029E00A9B009305ABFE
:1062B0000193029520463346FFF760FFE0B1E37E8D
:1062C000E3B90598FFF7E6FE0590FFF7EFFE059AA4
:1062D000137843B1531C0593127806F8012B1A4624
:1062E0001B78002BF6D10023337007E00823E376F8
:1062F000012004E0002002E0002000E0012006B0C0
:1063000070BD00BF10B51446082945D8DFE801F07C
:10631000050C131A21282F363D00254803685B68B9
:106320002449082298473DE0214803685B682249D8
:106330000E22984736E01E4803685B681F490D220D
:1063400098472FE01A4803685B681D491022984758
:1063500028E0174803685B681A490A22984721E039
:10636000134803685B681849112298471AE01048DF
:1063700003685B6815490D22984713E00C480368D1
:106380005B6813490B2298470CE0094803685B6877
:1063900010490D22984705E0054803685B680E49DF
:1063A0001322984714B1024805F012FA10BD00BF3D
:1063B000E4D7FF1F94FD0000A0FD0000B0FD000029
:1063C000C0FD0000D4FD0000E0FD0000F4FD000071
:1063D00004FE000010FE000020FE0000002202600B
:1063E000027170472DE9F04385B004468946904616
:1063F0001F460C9E02A8FFF7F1FF02AD0096019523
:106400002046494642463B46FFF726FF0028F5D086
:10641000E07ED0F1010038BF002005B0BDE8F08378
:1064200030B583B01C46069D0095FFF7DBFF05469F
:1064300030B32046144908F049FA48B120461349C0
:1064400008F044FA20B12046114908F03FFA18B983
:106450000123079A137013E020460E4908F036FA1C
:1064600048B120460C4908F031FA20B120460B49CA
:1064700008F02CFA18B90023079A137000E00025E1
:10648000284603B030BD00BF34FE00003CFE0000D3
:1064900040FE000044FE00004CFE000050FE0000E4
:1064A00030B583B01D46069C0094FFF79BFF044661
:1064B00020B1284607F038FC079B1870204603B02F
:1064C00030BD00BF30B583B01D46069C0094FFF779
:1064D00089FF044620B1284607F02AFC079B186074
:1064E000204603B030BD00BF10B584B0069C0094B8
:1064F00003AC0194FFF7E6FF034610B10399079A36
:106500001180184604B010BD30B585B01D46089CFA
:106510000094FFF767FF044678B1284603A90A22D2
:1065200008F064FD039BAB4204D01B7823B9099BA0
:10653000186002E0002400E00024204605B030BDD1
:1065400008B5C37A3BB1807A03F006FCD0F10100B4
:1065500038BF002008BD807A03F0FEFB003018BF72
:10656000012008BD08B5C37A23B1807A002103F069
:10657000CFFB08BD807A012103F0CAFB08BD00BF34
:1065800008B5C37A23B1807A012103F0C1FB08BDAD
:10659000807A002103F0BCFB08BD00BF10B50446A3
:1065A0008172C2720846012103F0E4FB2046FFF726
:1065B000E7FF00232373637310BD00BF10B5847A17
:1065C000204603F0C9FBD0F1010138BF002120466D
:1065D00003F09EFB10BD00BF007B704782B000231C
:1065E0000373437383730382034A12680192019A0F
:1065F0000260038102B0704720D6FF1FF0B583B060
:1066000004460E461746FFF7E9FF0125A5742782C9
:10661000AE40013EA6732046FFF7A4FF034B1B6864
:106620000193019B2360257303B0F0BD20D6FF1FAB
:1066300008B50A460121FFF7E1FF08BD10B5044681
:10664000FFF79EFF2046FFF7C9FF10BD10B50446B7
:10665000037B0BB1FFF7F2FF2046FFF783FF10BD6E
:1066600010B50446037B0BB1FFF7E8FF2046FFF7A8
:1066700087FF10BD84B070B582B0054607AE86E8CE
:106680000E00FFF7ABFF0023AB7405F114040FCE2F
:106690000FC496E8030044F8040B2180AB8A2B82D8
:1066A0009DF834300A2B28BF0A23AB732846FFF726
:1066B00059FF064B1B680193019B2B6001232B7331
:1066C00002B0BDE8704004B0704700BF20D6FF1F85
:1066D00030B58BB00446ADF81010ADF81220012390
:1066E0008DF82430022303936B460AAD15E90700A9
:1066F00003C31A8004AB0ECB2046FFF7BBFF0BB0E1
:1067000030BD00BF08B540F2EE210A46FFF7E0FFBA
:1067100008BD00BF08B528210A46FFF7D9FF08BD0C
:1067200010B586B0044603896BB12F4A12680192F6
:10673000019942688A1A934205D2FFF721FF204649
:10674000FFF74CFF4DE0238A002B4AD0264A1268FF
:106750000292029922688A1A934242D2637B0133E1
:10676000DBB26373A27B9A4225D913F0010F03D0E9
:106770002046FFF705FF02E02046FFF7F3FEA37C6B
:106780009BB9637B0A2B06D92046FFF7F9FE20460A
:10679000FFF724FF25E004EB43039B8A2382124B7F
:1067A0001B680393039B23601BE00F4B1B68049340
:1067B000049B236015E094F8283063B1A38A2382F8
:1067C000002363732046FFF7CDFE074B1B6805933C
:1067D000059B236005E02046FFF7D2FE2046FFF729
:1067E000FDFE06B010BD00BF20D6FF1F00230371C1
:1067F000114B198811F0010F18D102E00B420AD198
:1068000000E0012319430C4A11800C4A118821EA47
:106810000303138070470279013202715B009BB25F
:10682000B3F5805FEAD3FF2303717047012303713F
:10683000014B19880223E1E74AC6FF1F40C6FF1F2C
:106840002DE9F041044617461E4605790B2D3BD82D
:106850005FFA81F84046012103F08CFA25791C4B40
:1068600003F8058042F6E0621A4B23F815201A4B14
:10687000012202FA05F51A8815431D80FF002780C2
:10688000F6006680154B1B6813F0010F18D1134BEF
:106890001A6842F001021A60114B1A7842F0800225
:1068A0001A70A3F5143300221A6003210D4A1160F7
:1068B00001210432116045221A6020220A4B1A700D
:1068C0004FF40012094B1A602079BDE8F08100BF37
:1068D00064C6FF1F4CC6FF1F40C6FF1F3880044020
:1068E000005006400400044055E400E008E100E0E8
:1068F00008B54FF408724FF41663FFF7A1FF08BD07
:10690000C9000388994203DB43889942B8BF0B460C
:1069100002790B2A9CBF024921F81230704700BF50
:106920004CC6FF1F08B5384B93F90030374A128820
:106930001A4112F0010F07D0354AD05C002103F054
:10694000E7F90C22304B1A70324B1B785AB20B2AE3
:1069500035DC2E4A10885AB240FA02F111F0010FCC
:1069600026D009E05AB240FA02F111F0010F01D12C
:10697000DBB21DE027490B70254B985C012103F029
:10698000C7F9244B1A7820490A7052B2224931F8CB
:106990001210224A106808441060214A106801440D
:1069A0001160C521083A11601A7801321A7008BDC9
:1069B0000133DBB25AB20C2AD4D1164A1370174BEA
:1069C0001968C1F51C3303F58073B3F5487F05DB07
:1069D0004EF660229342A8BF134601E04FF448737D
:1069E0000E4A194411600E49086803440B60C52122
:1069F0000C4B196012680C4B9A4204D90023074AC9
:106A00001360044A137008BD0AA2FF1F40C6FF1F8F
:106A100064C6FF1F48C6FF1F4CC6FF1F44C6FF1FAA
:106A20000800044000000440FF70020030B482B04F
:106A30000E4B1B680193019D0123C0F824310346CE
:106A400000210A46441884F8C8209A621D60C3F8E1
:106A5000A020C3F8FC20013104330A29F2D100231D
:106A6000C0F8283102B030BC704700BF20D6FF1FED
:106A7000D0F82831092B09DC836A53B10123C26A9B
:106A80004AB1013304300A2BF9D106E04FF0FF3050
:106A9000704700207047184670474FF0FF3070472E
:106AA0002DE9F04182B00446884616461F46FFF79E
:106AB000DFFF002820DB16B304EB8005C5F850800B
:106AC000AE62AF672318012283F8C8200E4B1B6803
:106AD0000193019B44F82030D4F82401C5F8FC0050
:106AE000D4F828311344C4F828318318002BD8BFB8
:106AF0000123C4F8243104E04FF0FF3001E04FF0EF
:106B0000FF3002B0BDE8F08120D6FF1F08B5012399
:106B1000FFF7C6FF08BD00BFD0F8FC308B420AD09B
:106B200003460120D3F800218A4208D00130043303
:106B30000A28F7D101E0002070474FF0FF3070477E
:106B400038B50446D0F82851BDB1FFF7E5FFB0F1E4
:106B5000FF3F12D004EB80039A6A72B100229A625E
:106B6000204480F8C820C3F8D4201A65C3F8A020B8
:106B7000C3F8FC20013DC4F8285138BD2DE9F0438D
:106B800083B00546264B1B680193DDF804C000F175
:106B90002403002217464FF001084FF00209C3F802
:106BA000B07004331968E9B153F8281C9C6AC1EB32
:106BB0000C06A64216D3214443F8281CA91891F8C4
:106BC000C81079B1196D11B9C3F8AC800AE09C6F97
:106BD000A14207DDC3F8AC8001349C67A142D8BF55
:106BE000C3F8AC9001320A2AD9D12C4605F1280706
:106BF000D4F8D430012B02D0022B03D009E0A36AD1
:106C0000984706E0A36A98472846D4F8FC10FFF797
:106C100097FF0434BC42EBD103B0BDE8F08300BF62
:106C200020D6FF1F10B582B00446FFF775FFB0F104
:106C3000FF3F05D0034B1B680193019B44F82030B4
:106C400002B010BD20D6FF1F10B50446FFF764FF49
:106C5000B0F1FF3F1ABF001990F8C800002010BD26
:106C60002DE9F04F83B0019084693CB9002104F014
:106C700075FC00285AD004F03BFC57E0B4F1FF3F0C
:106C80000FD10198002104F069FC044600284DD082
:106C900001982146002204F04BFC204604F028FC19
:106CA00044E00198002104F065FC804600283DD0B6
:106CB000019BD3F81CC093F8209000231D4F9B46E6
:106CC0004FF0FF3A4E46200EC4F30F2108EB0302AB
:106CD000B2F90450C1F5803E37F91090013037F910
:106CE000100001FB00F109FB0E11091401FB05F175
:106CF000C913918026B1E243944506D2644407E06B
:106D0000A44504D2CCEB040402E0544600E05C4607
:106D10000233B3F5807FD6D1019B9C611846414672
:106D2000002204F005FC404604F0E2FB03B0BDE89D
:106D3000F08F00BF54FE000072B6836913B90123BF
:106D4000836105E0B3F1FF3F04BF6FF0010383618E
:106D5000C16180F8202062B6704700BF10B50446BC
:106D600004F0F6FC204610BD08B503480349044A68
:106D700006F0D4FF08BD00BF70C6FF1F5D6D0000A8
:106D80003C98FF1F38B5064D064C07482946224659
:106D900006F0C4FF05482946224606F0BFFF38BD6D
:106DA0005D6D00003C98FF1F78C6FF1F80C6FF1F67
:106DB00008B503480349044A06F0B0FF08BD00BF08
:106DC00088C6FF1F5D6D00003C98FF1F08B5034893
:106DD0000349044A06F0A2FF08BD00BF90C6FF1F8A
:106DE0005D6D00003C98FF1F2DE9F8438146804609
:106DF00000263746F7B94846314604F0BBFB074644
:106E0000002853D0D8F81810B1F5803F4ED0031D9C
:106E100000F582741A6831FB02F031FB12F200F3C4
:106E20000F0002F30F02C0EA024243F8042B9C4217
:106E3000F0D83BE04846314604F090FB8446A8B3C6
:106E40003B1D051DD8F8184007F5827EB4F5803F3C
:106E500016D107F10C040C3054F8082C50F8081C1B
:106E600092FA11F244F8082C5A6850F8041C92FA6D
:106E700011F25A600833083408309E45ECD812E00D
:106E800055F8042B34FB02F034FB12F200F30F0030
:106E900002F30F02C0EA0242196892FA11F143F8B4
:106EA000041B9E45ECD8604604F022FB013608F135
:106EB0000408042E9ED13FB148463946002204F012
:106EC00037FB384604F014FBBDE8F88308B5002111
:106ED00004F044FB0246A0B172B60A4B186810B920
:106EE0001A6062B608BD084B1B681BB9064B1A60D6
:106EF00062B608BD03490B60034B1A6062B604F02A
:106F0000F7FA08BDA8C6FF1F98C6FF1F38B51C4B6F
:106F10001A68126819791B4B19701B4B9A4206D2DA
:106F2000A3F5807404F5807304F5007402E0174B38
:106F300003F58074164A106898B1021D47F6FF7574
:106F400032F9021B2944091123F8021B9C42F7D88D
:106F500004F0CEFA0F4B1A680D490A6000221A603D
:106F600005E040F2FF7223F8022B9C42FBD80A4B4B
:106F70001B781BB14FF08042084B1A6038BD00BF30
:106F80009CC6FF1F1F800040308FFF1F308EFF1FE9
:106F9000A8C6FF1F98C6FF1FA4C6FF1F08E200E097
:106FA00070B54F48012104F075FB4E4B1A6842F44E
:106FB00080521A60802203F5032303F6F5731A70DA
:106FC0000024494E01253480284602F0B5FF0834DC
:106FD000A4B223B2B3F5006FF5D1444B1B6813F490
:106FE000800F16D0424B1A6848F6A2731A409A4294
:106FF0000FD1404B1A6840F23F439A4209D13E4BB1
:107000001B68012B05D13D4B1A6840F201139A42CF
:1070100017D0364B1A6842F480021A600122A3F599
:107020009033303B1A6040F23F42083B1A60043B09
:1070300048F6A3721A60324A1A6040F20112103305
:107040001A60274C23681A6800222E4919602368A9
:10705000022119715A7101209871D87119725A72EE
:107060009A72DA721A736FF0010159734FF0FF319F
:107070009973D97319691C4919611A755A75D98A96
:107080004FF48071D9821A765A769A76DA76D88B4E
:10709000D983998B06219983237903F1804303F5E2
:1070A00004331A70B0221A7004F0A0FA164B18704C
:1070B0002279164B1A70227902F110011448154BEF
:1070C00043F8210053119B0003F1604303F5614332
:1070D00002F01F02012101FA02F21A6070BD00BF26
:1070E0009CC6FF1F2C80044000C00C403C80044024
:1070F00000600340046003400C60034010600340E4
:10710000A28F0100308EFF1FA4C6FF1F1B8000400E
:107110000D6F00000092FF1F0229044B1A780CBF6C
:1071200002F0BF0242F040021A70704721C00C40CA
:1071300008B503480349044A06F0F0FD08BD00BF46
:107140009CC6FF1F5D6D00003C98FF1F08B50348FB
:107150000349044A06F0E2FD08BD00BFACC6FF1FAC
:107160005D6D00003C98FF1F08B503480349044AC1
:1071700006F0D4FD08BD00BFB4C6FF1F5D6D000062
:107180003C98FF1F08B503480349044A06F0C6FDB2
:1071900008BD00BFBCC6FF1F5D6D00003C98FF1F0F
:1071A00008B503480349044A06F0B8FD08BD00BF0E
:1071B000C4C6FF1F5D6D00003C98FF1F08B5034863
:1071C0000349044A06F0AAFD08BD00BFCCC6FF1F54
:1071D0005D6D00003C98FF1F10B504460C2380F83D
:1071E0007F3280F8803200234366006F18B104F0CC
:1071F0007FF900232367606F18B104F079F9002349
:10720000636710BD38B5044672B690F87F320C2B18
:107210001FD0006F00232367656F63670C2384F81A
:107220007F3262B608B104F063F915B1284604F064
:107230005FF904F1180001F0DFFA074B1B8823B156
:10724000013B9BB2044A138023B95E2000F030FC5E
:1072500038BD62B638BD00BFD4C6FF1F30B58FB091
:1072600004460D46FFF7CEFF5E2000F007FC2E4BD4
:107270001A8801321A8072B601A82946002201F04C
:1072800049F89DF808302377039B23629DF810305E
:1072900084F82430059BA362069BE362079B23636B
:1072A000089B6363099BA3639DF8283084F83C30F6
:1072B0009DF8293084F83D300EAB53F80E5D5868C8
:1072C0009968C4F83E50C4F84200C4F846101B7BCD
:1072D00084F84A3001A801F07BF962B694F83D3099
:1072E000032B0DD9104B1B882BB1013B9BB20E4ACF
:1072F00013800020ABB95E2000F0DAFB002010E024
:107300000023A4F87C32A4F87A320C2284F880227C
:107310001422626684F87E32082384F87F320120CA
:10732000FFE70FB030BD00BFD4C6FF1FC36C9AB2D9
:10733000012A2AD1026D4AF644418A420AD045F216
:1073400022618A4209D042F611318A421FD1134983
:10735000042204E01249002201E0124904221B0C1D
:10736000012B04D0022B14D1490842F00102B0F8DD
:107370005A30082B04D0102B0DD1490842F00202DC
:10738000C16680F8802201207047002070470020ED
:107390007047002070470020704700BF34EE35175B
:1073A0008D7BCD051AF79A0B2DE9F84F0446B0F8FE
:1073B0007A6206447A360D46002900F0B4814FF017
:1073C00008090027DFF898B3DFF898A302E0002D42
:1073D00000F0AC8194F87F320C2B00F29C81DFE846
:1073E00013F0A801A801D8002601A801A801A8014E
:1073F000A8010D004F007F00BC00A801636E9D42F4
:1074000034BFA846984604F14C0094F87E321844E4
:107410003146424602F058F994F87E32434484F8EB
:107420007E32B4F87A324344A4F87A32636EC8EB01
:1074300003036366002B40F07F81E36C534540F00B
:107440006A81636DC54A934240F06581A36D02F184
:107450005B4202F5F11202F60F42934240F05B816B
:10746000E36DA3F11002082A00F255814644C8EBEF
:107470000505636684F87E72092384F87F32A6E7E7
:10748000636E9D4234BFA846984604F14C0094F8C0
:107490007E3218443146424602F016F994F87E32A4
:1074A000434484F87E32B4F87A324344A4F87A3202
:1074B000636EC8EB03036366002B40F040812046F7
:1074C000FFF734FF002800F026814644C8EB05058D
:1074D000C4F8649084F87E720A2384F87F3276E7D9
:1074E000636E9D4234BFA846984604F14C0094F860
:1074F0007E3218443146424602F0E6F894F87E3275
:10750000434484F87E32B4F87A324344A4F87A32A1
:10751000636EC8EB03036366002B40F0138146449F
:10752000C8EB0505236D6366E36C5B4511D184F8F8
:10753000817294F8803284F87F3213F0010F05D005
:1075400003F07AFF6067002800F0FF80636EA36697
:107550003DE70B2384F87F3239E7636EAB4209D9EC
:107560005B1B6366B4F87A321D44A4F87A5200209B
:10757000BDE8F88F1E44ED1AB4F87A221344A4F83B
:107580007A32C4F8649084F87E720A2384F87F32D9
:107590001DE7636E9D4228BF1D465B1B6366023676
:1075A00016F8021C16F8010C023D226FB4F8783070
:1075B00003F1010CA4F878C002EB430341EA002276
:1075C0009A80B4F878307F2B24D92046216F00228E
:1075D00003F0AEFF2046216F012203F0A9FF206FC8
:1075E00003F086FF00232367636E1D44656604F184
:1075F0007A03F71AA4F87A72606F08B103F078FF83
:10760000636E002B40F0A4800C2384F87F320120AD
:10761000BDE8F88F0236002DC2D1636E002B40F01A
:107620009A800C2384F87F320020BDE8F88F636EC7
:107630009D4228BF1D465B1B636694F881325BB197
:10764000236FB4F8782003EB4202E36C93800023AD
:1076500084F8813219E03E4633787278023D0BD1CE
:10766000616E002951D043EA0223E364022384F8C7
:1076700081320020BDE8F88F0236216FB4F878001F
:1076800001EB400143EA02238B80374617F8021BC7
:107690007078023D626FB4F878305E1CA4F87860B0
:1076A00002EB430341EA00229A80B4F878307F2B42
:1076B00022D92046216F002203F03AFF206F03F009
:1076C00017FF002626672046616F012203F030FF76
:1076D000606F03F00DFF6667636E1D44656604F11D
:1076E0007A03FF1AA4F87A72002D3DD10C2384F896
:1076F0007F320120BDE8F88F002DACD1636E23B13D
:10770000002084F88102BDE8F88F0C2384F87F32D2
:107710000020BDE8F88F0C2384F8803284F87F3293
:107720000020BDE8F88F0020BDE8F88F0020BDE8FC
:10773000F88F0020BDE8F88F0020BDE8F88F00200A
:10774000BDE8F88F0020BDE8F88F0020BDE8F88F75
:107750000120BDE8F88F0020BDE8F88F574156455D
:1077600064617461524946460120BDE8F88F00BF4C
:1077700090F87F0207288CBF00200120704700BFCF
:1077800090F87F32072B07D8826E436ED21AC16EF3
:10779000A2FB0123184670470020704790F87F3203
:1077A000072B05D8C36E826EA2FB032318467047D1
:1077B000002070472DE9D847044690F87F320C2B03
:1077C00000F0AD8003F038FE2067002800F0A780AD
:1077D00094F87F32072B0BD813F0010F08D003F079
:1077E0002BFE606730B9206F03F082FEBDE8D887BA
:1077F000002363670023A4F87830B4F87C12B4F84F
:107800007A32C91A002905DD2046FFF7CDFD002890
:1078100040F0858094F87F320C2B2CD004F11806B0
:10782000304600F0B5FE30B304F17A084FF400772B
:107830004FF00009304641463A4600F0D5FE83B28B
:10784000A4F87C32BBB1A4F87A9294F87FA22046C7
:107850001946FFF7A9FD20B194F87F320C2B5ED1B9
:1078600009E094F87F320C2B05D0BAF1070F16D936
:10787000072BDFD913E004F1180000F0BDFF294BFE
:107880001B8823B1013B9BB2264A138013B95E20AB
:1078900000F00EF90C2384F8803284F87F32236FD5
:1078A0001BB3B4F87820DAB113467F2A07D8002139
:1078B000226F02EB430291800133802BF8D12046E6
:1078C000216F002203F034FE94F87F32072B07D893
:1078D00013F0010F04D12046216F012203F028FE8E
:1078E000206F03F005FE00232367636FBBB1B4F87C
:1078F00078207AB113467F2A07D80021626F02EB05
:10790000430291800133802BF8D12046616F012220
:1079100003F00EFE606F03F0EBFD00236367BDE82C
:10792000D88700BFD4C6FF1F70B5054690F8303029
:1079300013F0FF0F4FD003F07FFD064600284AD01A
:10794000296AEB6999421FD201F58072934232D2C3
:107950005C1AA8690844311D224601F0D7FA2B6A47
:1079600023442B62EB6A2344EB6263087F2B1DD90F
:1079700004E022F8024F01337F2BFAD92846314622
:10798000002203F0D5FD0DE0134B1B8823B1013B12
:107990009BB2114A138013B95E2000F089F80023CE
:1079A00085F83030304603F0A3FD70BD06EB43028E
:1079B00002320024DDE7A8690844311D4FF48072CB
:1079C00001F0A4FA2B6A03F580732B62EB6A03F5CE
:1079D0008073EB62D2E770BDD4C6FF1F002380F82E
:1079E0003030C36283627047184B1A6842F4805289
:1079F0001A60174B174A1A60174ADA6002F1804280
:107A00001A61164A1A60164B1B7813F0010F07BF54
:107A10004FF41072134B4FF40072134B1A60104B5B
:107A20001B7813F0020F4FF400720CBF0F4B104B7A
:107A30001A600B4B1B7813F0040F07BF4FF4107242
:107A40000C4B4FF400720C4B1A6070473C800440A2
:107A500000C0024001401F000110003800001F80DC
:107A6000E0D7FF1F18B0044008C004401CB0044019
:107A70000CC0044014B0044004C0044030B45E287C
:107A800010D84309084A012101FA03F514782C4360
:107A90001470064A00F01F00814052F823400C4346
:107AA00042F8234030BC7047F0C6FF1FD8C6FF1F06
:107AB0005E2815D8430900F01F00012202FA00F0E9
:107AC000084A52F8231021EA000042F8230038B98E
:107AD000054A012101FA03F3117821EA0303137027
:107AE000704700BFD8C6FF1FF0C6FF1F72B60D4B10
:107AF0004FF0FF30002203F65461C3F8000283F810
:107B0000082283F8092203F5037343F8083C8B42EB
:107B1000F3D3002243F8082C024A034B1A6062B6E2
:107B2000704700BFF8C6FF1FF4C6FF1F03684BB1C4
:107B300072B6036893F80822013A83F8082262B605
:107B400000230360704700BF2DE9F84380460F46CD
:107B500091462C4B1B680BB9FFF7C8FFD8F8000003
:107B600030B1D0F80032BB424AD04046FFF7DEFFCA
:107B700072B6244B1868034600252E462A46D3F8D1
:107B80000012B94214D119463AB1D3F80442C2F8EE
:107B90000442C3F804021B4A136091F80822013220
:107BA00081F8082262B6C8F800101846BDE8F883CC
:107BB00093F80842002C08BF1546002C08BF1E464B
:107BC000D3F8044214B11A462346D8E7B9F1000F9E
:107BD00013D096B13DB1D6F80432C5F80432C6F8D8
:107BE0000402084B1E60012386F80832C6F80072B2
:107BF000002386F80932C8F8006062B6D8F80000A1
:107C0000BDE8F883F4C6FF1FF8B50D4617463D4B97
:107C10001B78002B28D072B63A4B1B7813F0010F5B
:107C200007D0394B1968394A12680A4038490A6046
:107C30001A60344B1B7813F0020F07D0354B1968CC
:107C4000324A52680A4032494A601A602D4B1B780A
:107C500013F0040F07D0304B19682C4A92680A4081
:107C60002B498A601A6062B62C4BDB68B3F1384F3F
:107C70000AD02A4B2A4A1A604FF03842DA604FF095
:107C800078421A61274A1A6029460122FFF75CFFF1
:107C90000446A8B190F8093213F0010F01D006464E
:107CA00011E006462846214600F0BCF950B11FB944
:107CB000012384F8093206E0052384F8093202E042
:107CC000002600E000260F4B1B78C3B113F0010F14
:107CD00003D00F4B1A68144B1A600A4B1B7813F031
:107CE000020F03D00A4B5A68104B1A60054B1B78E1
:107CF00013F0040F03D0064B9A680D4B1A60304600
:107D0000F8BD00BFF0C6FF1F80E100E0D8C6FF1F2E
:107D1000E4C6FF1F84E100E088E100E000C002400B
:107D200001401F0000001F8000E100E004E100E0CE
:107D300008E100E0F8B505460E461746414B1B78B2
:107D4000002B28D072B63F4B1B7813F0010F07D0E1
:107D50003D4B19683D4A12680A403D490A601A6065
:107D6000384B1B7813F0020F07D03A4B1968374A8B
:107D700052680A4036494A601A60324B1B7813F049
:107D8000040F07D0344B1968304A92680A403049D2
:107D90008A601A6062B6314BDB68B3F1384F0AD0A3
:107DA0002E4B2F4A1A604FF03842DA604FF078427B
:107DB0001A612C4A1A60284631460022FFF7C4FE99
:107DC000044620B190F8093213F0010F05D1304676
:107DD000394600F027F9064600E00126194B1B78CA
:107DE000C3B113F0010F03D0194B1A681E4B1A6070
:107DF000144B1B7813F0020F03D0154B5A681B4B22
:107E00001A60104B1B7813F0040F03D0104B9A68C4
:107E1000174B1A60A4B194F8093213F0010F0AD07D
:107E2000384621464FF4007201F04EFC2846FFF719
:107E30007DFE0120F8BD2846FFF778FE3046F8BDEC
:107E40003046F8BDF0C6FF1F80E100E0D8C6FF1F36
:107E5000E4C6FF1F84E100E088E100E000C00240CA
:107E600001401F0000001F8000E100E004E100E08D
:107E700008E100E01B4B1B68012283F800211A4B2C
:107E80004FF00042DA62020A5A631A46D36A002BA4
:107E9000FCDA154B9A6B4FF00042DA620A0C42F0A2
:107EA00080525A631A46D36A002BFCDA0E4B9A6B47
:107EB0004FF00042DA6289B241F0805159631A46AC
:107EC000D36A002BFCDA084B9A6B4FF00042DA625F
:107ED000C0B258631A46D36A002BFCDA024B9B6B84
:107EE000704700BF4CD5FF1F00C0024030B40921CD
:107EF000094A4FF00045FF24D5625463D36A002B32
:107F0000FCDA906B10F0800F03D04B1E13F0FF01D2
:107F1000F2D1C0B230BC704700C002400D4B4FF0F0
:107F20000042DA620C4A5A631A46D36A002BFCDA22
:107F3000084B986B00044FF00042DA62064A5A631D
:107F40001A46D36A002BFCDA024B9B6B9BB2184398
:107F5000704700BF00C00240FFFF0010084B1B68C5
:107F6000012283F88020074B4FF00042DA62FF22A3
:107F70005A631A46D36A002BFCDA024B9B6B70479C
:107F80004CD5FF1F00C0024010B544F295000021FF
:107F9000FFF770FFFFF7AAFF0446FFF7DFFF204659
:107FA00010BD00BF10B544F687004FF4D571FFF740
:107FB00061FFFFF79BFF012818BF4FF0004403D17A
:107FC000FFF7ACFF0446FFE7FFF7C8FF204610BDF0
:107FD00010B5044647F2FF700021FFF74BFFFFF793
:107FE00085FFFFF7BBFF46F6FF102146FFF742FF74
:107FF000FFF77CFF0446FFF7B1FF204610BD00BF2E
:1080000010B547F6FF200021FFF734FFFFF76EFFA2
:1080100018B9FFF783FF044600E00024FFF79EFF36
:10802000204610BD70B503460D46324A1278012A2B
:1080300098BF430245F2FF101946FFF71BFFFFF7F9
:1080400055FF18B1FFF78AFF002070BD2A4A4FF094
:108050000044FF20D4625063D36A002BFCDA936B98
:10806000DBB2FE2B05D0FF2BF4D0FFF777FF00200B
:1080700070BD05F5FF76204B204A5A635A63B5421E
:1080800013D2A81C05F500751A461C4CD36A13F0D0
:10809000F00FFBD05463936B190A00F8021C00F830
:1080A000013C0230A842F1D100E02E46124AD36AC8
:1080B00013F0F00FFBD0104B9B6B1A0A32707370E9
:1080C0000D4AD36A13F0F00FFBD00B4B9A6B0C4A9E
:1080D0001268012182F880104FF00042DA62FF221C
:1080E0005A631A46D36A002BFCDA034B9B6B0120C0
:1080F00070BD00BF50D5FF1F00C00240FFFF001041
:108100004CD5FF1F10B400230361CB6943618A8AF9
:108110004B8B43EA02438361C361CB7A03F01003C4
:10812000DBB2002B0CBF0023022380F825300A7835
:10813000202A08BF00F1260308D020E014F8012F00
:10814000202A03D003F8012B8342F7D10A7A202A90
:1081500012D02E221A700A7A5A704A7A202A02D134
:10816000981C093102E0D81C0A319A700A78202A3A
:108170001ABF431C0270034600221A7006E000F189
:10818000270380F826200C462E30D7E75DF8044BF5
:10819000704700BF2DE9F04F87B0064691460B7837
:1081A000002B00F0A3802F2B0DD1A5E011F8013F8B
:1081B000002B00F0A2802F2B0CD19EE002F8011BB7
:1081C0009A42FBD321E003AA05A820240DF1150C47
:1081D0000DF117052E2B0BD1824214D2134603F852
:1081E000014B8342FBD1531CC3EB0C031A440AE03E
:1081F0007E2B08D8A3F16107FFB2192F9CBF203B4B
:10820000DBB213700132AA42D0D396F82530032B8B
:1082100005D1D6F818B073695B0A01930EE0022B02
:1082200066D1B269F261394B1B78023A02FA03FB5C
:10823000374A1268934401229A400192002100912A
:1082400001278A4639E006A840F810AD5946524643
:10825000FFF7DAFC044648B355464FF00B082046BA
:1082600003A9424606F050F828B948462146FFF7D0
:1082700049FF01241DE023783FB10BB1E52B05D167
:10828000C9F820B089F8245057468BB133692033A0
:10829000336120340135102DE1D10BF1010B02A81F
:1082A000FFF744FC009A0132009206E0002400E04F
:1082B000002402A8FFF73AFC23E0009B01998B42BF
:1082C000C1D396F82530032B14D0304600F012F9B4
:1082D0000446B0B1F369023B0C490A7803FA02FB89
:1082E0000B4A13689B44CDF800A0E6E7002408E0A1
:1082F000002406E0002404E003AA20210DF1170366
:108300005CE7204607B0BDE8F08F00BF5CD5FF1FDB
:1083100058D5FF1F30B59BB005460C4600F048F914
:10832000684B1A798DF804209A6802921A7B8DF8AE
:108330000C20654A00921A6904925A6905929A695A
:108340000692DA6907921A6A089293F824208DF847
:10835000242093F825208DF8252053F8260F5968FE
:108360009A68CDF82600CDF82A10CDF82E201B7B78
:108370008DF8323000E0013423782F2BFBD043BB43
:108380009DF804302B71029BAB609DF80C302B7371
:10839000049B2B61059B6B61069BAB61079BEB61AB
:1083A000089B2B629DF8243085F824309DF82530F9
:1083B00085F825301AAB53F8424D58689968C5F8CE
:1083C0002640C5F82A00C5F82E101B7B85F83230F0
:1083D00071E00DA800F0ECF8684621460DAAFFF701
:1083E000D9FE631C1C4613F8012B2F2A5DD0002AEE
:1083F000F8D15DE09DF838302B710F9BAB609DF894
:1084000040302B73119B2B61129B6B61139BAB61F3
:10841000149BEB61159B2B629DF8583085F8243036
:108420009DF8593085F825301AAB53F80E4D586831
:108430009968C5F82640C5F82A00C5F82E101B7BA0
:1084400085F832302DE09DF838308DF804300F9BE0
:1084500002939DF840308DF80C30119B0493129BD1
:108460000593139B0693149B0793159B08939DF804
:1084700058308DF824309DF859308DF825301AABDE
:1084800053F80E0D59689A68CDF82600CDF82A10D9
:10849000CDF82E201B7B8DF832300DA800F098F817
:1084A0006AE70DA800F094F805E00028CBD1F8E7C2
:1084B00000289FD1F5E7684600F08AF828461BB0EF
:1084C00030BD00BF60D5FF1FB000010010B58EB0F9
:1084D000014601A80022FFF71DFF9DF82940032C4B
:1084E0008CBF0024012401A800F072F820460EB0D1
:1084F00010BD00BF30B583B0044600230193174B75
:108500001968C569164B1B78102B0AD101A801EB1D
:1085100015210122FFF778FBB0B1EDB230F815302C
:108520000AE001A801EBD5110122FFF76DFB68B14C
:1085300005F07F0550F82530E3610A4A1468A3422C
:108540008CBF0024012402E0002400E0002401A8E4
:10855000FFF7ECFA204603B030BD00BF94D5FF1FF3
:1085600098D5FF1F9CD5FF1F10B582B002AB03F852
:10857000011D0268546819460122A04702B010BDCF
:1085800090F82530012B1CBF012303710020704798
:1085900090F82530012B07D803694069C01A0028DC
:1085A000B8BF6FF00040704700207047704700BFB1
:1085B000002202714FF47A718160027303490160F5
:1085C000042180F8251080F826207047B0000100B3
:1085D000044A0260042280F82520002280F8262028
:1085E000704700BFB00001002DE9F04F83B0064690
:1085F000884690F82530012B00F2A3800369416979
:10860000C91A8A4234BF91468946B9F1000F00F079
:108610009A804F4A127802F10901012000FA01F113
:1086200001390B40F1698C1E94404A4A1068044499
:1086300004EB5324C3F30805002D3CD0002202A80C
:1086400040F8042D2146FFF7DFFA014610B3C5F5C7
:10865000007BCB4509D9404629444A4601F034F80D
:1086600033694B4433614D4615E0404629445A4630
:1086700001F02AF833695B44336101A8FFF756FA29
:108680000134334B1B78012202FA03F3013B1C42F5
:108690000BD104E0002501A8FFF748FA54E030466A
:1086A000FFF728FF08B95D464EE0CB4501D2D8441C
:1086B00003E05D4648E04FF0000BCBEB09075D4659
:1086C000CBEB080BDFF888A00BEB05080023019328
:1086D000B7F5007F0FD201A821461A46FFF794FA9A
:1086E000014608B340463A4600F0EEFF33693B448A
:1086F00033614D4618E001A821464246FFF71AFBB8
:1087000090B1336903F50073336105F5007501A875
:10871000FFF70CFA01349AF80030012202FA03F351
:10872000013B1C4208D103E001A8FFF7FFF90BE071
:108730003046FFF7DFFE38B1A7F50077A945C3D86B
:1087400002E0002500E00025284603B0BDE8F08FD8
:108750005CD5FF1F58D5FF1F00B583B00DF1070191
:108760000122FFF741FF01280CBF9DF807004FF0E1
:10877000FF3003B05DF804FB70B582B004460669B3
:10878000C5690DF107010122FFF72EFF012803BF84
:108790002661E5619DF807004FF0FF3002B070BD23
:1087A000F8B505460E4690F82530012B1DD84369D3
:1087B0008B421CD3C7690F4B1B78093321FA03F492
:1087C000026922FA03F3E31A52BF1C468369C361AC
:1087D00044B12846FFF78EFE034608B9EF6107E073
:1087E000013CF6D12E61012302E0002300E00023CA
:1087F0001846F8BD5CD5FF1F042380F82530002300
:1088000080F82630704700BF2DE9F04F87B07D4DCE
:108810007D4B53F830302B6001247C4B1C7021467B
:1088200001F0A8FA2B6883F88040FFF7DDF8784B59
:108830001B78002B28D072B6754B1B7813F0010FF4
:1088400007D0744B1968744A12680A4073490A6069
:108850001A606F4B1B7813F0020F07D0704B19682A
:108860006D4A52680A406D494A601A60684B1B782D
:1088700013F0040F07D06B4B1968674A92680A40DF
:1088800066498A601A6062B6674BDB68B3F1384F9D
:108890000AD0654B654A1A604FF03842DA604FF0F3
:1088A00078421A61624A1A6005215F4A4FF000441B
:1088B0006048D4625063D36A002BFCDA936B4B1E82
:1088C00013F0FF01F5D15C4B1B680293029D504CE5
:1088D000DFF87491DFF86CA1DFF84881504F4D4EFE
:1088E000FFF752FB012858D02378B3B113F0010FE2
:1088F00003D04A4B1A68514B1A60237813F0020FC9
:1089000003D0464B5B68CAF80030237813F0040F9D
:1089100003D0424B9B68C9F80030474B1B68039358
:10892000039B5B1BFA2B00F2C181237823B372B641
:10893000237813F0010F06D03268374B1B681340C1
:10894000364A13603360237813F0020F06D03A687A
:10895000314B5B681340314A53603B60237813F01E
:10896000040F08D0D8F800202B4B9B6813402B4AEB
:108970009360C8F8003062B62B4BDB68B3F1384F18
:10898000AED0294B294A1A604FF03842DA604FF0D6
:1089900078421A61264A1A60A2E7FFF703FBB0F19A
:1089A000004F04D10122264B1A7000254EE0B0F58D
:1089B000D57F05D10222224B1A704FF0804545E049
:1089C000134B1B78002B00F0738113F0010F03D0C1
:1089D000124B1A68194B1A600D4B1B7813F0020FDB
:1089E00003D00E4B5A68174B1A60094B1B7813F0D3
:1089F000040F00F05F81094B9A68134B1A60002442
:108A00005DE100BF4CD5FF1F1401010051D5FF1FD0
:108A1000F0C6FF1F80E100E0D8C6FF1FE4C6FF1FBD
:108A200084E100E088E100E000C0024001401F0056
:108A300000001F80FFFF001020D6FF1F00E100E0B4
:108A400050D5FF1F04E100E008E100E09E4B1B68E9
:108A50000493049E9D4CDFF89CA2DFF894B2DFF8EB
:108A6000B492DFF8B4829A4F2846FFF7B1FA024673
:108A700000285FD02378B3B113F0010F03D0954BDA
:108A80001968954B1960237813F0020F03D0914BAE
:108A90005B68CBF80030237813F0040F03D08D4BC4
:108AA0009B68CAF80030012A00F20681864B1B68D9
:108AB0000593059A921B40F2DC539A4200F2FE8025
:108AC000237833B372B6237813F0010F06D03A68D7
:108AD000824B1B6813407F4A13603B60237813F07E
:108AE000020F08D0D8F800207C4B5B681340794A0D
:108AF0005360C8F80030237813F0040F08D0D9F879
:108B00000020764B9B681340724A9360C9F800308E
:108B100062B6734BDB68B3F1384FA5D0704B714A26
:108B20001A604FF03842DA604FF078421A616E4AAC
:108B30001A6099E76D4B1B78022B07D1FFF760FA9B
:108B4000800F032802D10322684B1A705F4B1B78F9
:108B5000C3B113F0010F03D05E4B1A685E4B1A606D
:108B60005A4B1B7813F0020F03D05A4B5A68604BD4
:108B70001A60564B1B7813F0040F03D0554B9A68BC
:108B80005C4B1A60002206A840F8142D1146FFF72E
:108B90003BF8B0F8FE214AF655239A4277D190F877
:108BA000C231062B03D00B3BDBB2012B02D8D0F82D
:108BB000C64100E0002401A8FEF7B8FF01A8214645
:108BC0000022FFF721F8B0F8FE214AF655239A4219
:108BD0005FD1B0F80B30B3F5007F5CD1037C022B82
:108BE0005BD1C589002D5AD0427BB2FA82F2C2F124
:108BF0001F02414B1A70C38A03B9436AB0F811705F
:108C000007F10F0E4FEA1E1EB0F8136006B9066A90
:108C100061193A4C21601944394C216003EB0E0C68
:108C20008C44384CC4F800C0741BCEEB0404A4EB95
:108C3000430424FA02F2551C334C256040F6F474C8
:108C4000A2422ED94FF6F474A2420BD810202F4A1C
:108C500010702F4A7F0157610B449361032382F800
:108C600025300AE02022294B1A70294B00225A6134
:108C7000C26A9A61022283F82520254B9A69DA613B
:108C800000221A6101A8FEF751FF01240AE0002426
:108C900008E0002406E0002404E0002402E00024B0
:108CA00000E0002401A8FEF741FF08E0002406E0F0
:108CB000002404E0002402E0002400E00024204618
:108CC00007B0BDE8F08F00BF20D6FF1FF0C6FF1F22
:108CD00080E100E0E4C6FF1F00E100E0D8C6FF1F0E
:108CE00000C0024001401F0000001F8050D5FF1F40
:108CF00004E100E008E100E05CD5FF1F94D5FF1F10
:108D000054D5FF1F58D5FF1F9CD5FF1F98D5FF1FB7
:108D100060D5FF1F88E100E084E100E010B5054C5C
:108D20002046FFF745FC20460349044A04F0F6FFBD
:108D300010BD00BF60D5FF1FD18500003C98FF1F0C
:108D4000014A024B1A60704701100138A0D5FF1F7D
:108D50002DE9F0075E495F4E5F48604D604C614B06
:108D6000DFF8A0A1DFF8A0C10A782AB372B60A78AA
:108D700012F0010F07D0226807683A40DFF87881C7
:108D8000C8F8002022600A7812F0020F07D02A6883
:108D900047683A40DFF86081C8F804202A600A7802
:108DA00012F0040F07D0326887683A40DFF8488134
:108DB000C8F80820326062B6DA68B2F1384F09D0DC
:108DC000494A1A604FF03842DA604FF078421A612F
:108DD000464A1A60464AD2F80080012288F80021EB
:108DE000444A127812F0020F35D04FF00042DA6296
:108DF00070225A63DA6A002AFCDA9A6B4FF000425A
:108E0000DA6200225A63DA6A002AFCDA9A6B5FFAA5
:108E100082F9012288F880200A78C2B112F0010F8D
:108E200005D0354AD2F80080344AC2F800800A786A
:108E300012F0020F03D0304A5268CCF800200A78B2
:108E400012F0040F03D02C4A9268CAF8002019F0DF
:108E5000800F89D035E04FF00042DA6205225A6374
:108E6000DA6A002AFCDA9A6B4FF00042DA620022DA
:108E70005A63DA6A002AFCDA9A6B5FFA82F90122F5
:108E800088F880200A78C2B112F0010F05D01A4A82
:108E9000D2F80080194AC2F800800A7812F0020F56
:108EA00003D0154A5268CCF800200A7812F0040F5B
:108EB00003D0114A9268CAF8002019F0010F7FF41C
:108EC00053AF00220E4B1A70BDE8F007704700BF89
:108ED000F0C6FF1F88E100E0D8C6FF1F84E100E074
:108EE00080E100E000C0024001401F0000001F8040
:108EF000A8D5FF1FA4D5FF1FE4C6FF1F00E100E0B7
:108F0000A5D5FF1F08E100E004E100E02DE9F04FE6
:108F100085B080468A4691460846002105F088FAC9
:108F20007D4B1B7803937D4B1B78002B28D072B6AA
:108F30007A4B1B7813F0010F07D0794B1968794AE7
:108F400012680A4078490A601A60744B1B7813F063
:108F5000020F07D0754B1968724A52680A4072496D
:108F60004A601A606D4B1B7813F0040F07D0704BEA
:108F700019686C4A92680A406B498A601A6062B646
:108F80006C4BDB68B3F1384F0AD06A4B6A4A1A60FF
:108F90004FF03842DA604FF078421A61674A1A603F
:108FA000674B1B780293002B00F02B81654B1B68ED
:108FB000012283F80021584B1B7813F0020F1BD0BD
:108FC0005C4B4FF00042DA6270225A631A46D36A51
:108FD000002BFCDA574B9A6B4FF00042DA6200220A
:108FE0005A631A46D36A002BFCDA524B9B6B13F080
:108FF000800F00F0D681F9E14E4B4FF00042DA626B
:1090000005225A631A46D36A002BFCDA494B9A6B45
:109010004FF00042DA6200225A631A46D36A002BEC
:10902000FCDA444B9B6B13F0010F00F0DF81B8E1D9
:10903000012381F800313F4B4FF00042DA620622F3
:109040005A631A46D36A002BFCDA3A4B9B6B012316
:1090500081F880302023013B7FF4FDAF039A12F0AA
:10906000040F05D0029B012B0CBF8522752200E066
:109070007522012381F800312E4B4FF00040D86259
:109080005A631A46D36A002BFCDA2A4B9B6B0123E6
:1090900081F88030039A12F0020F1DD081F8003160
:1090A000244B4FF00042DA6270225A63DA6A002AD7
:1090B000FCDA204B9B6B1F4A4FF000440020D46227
:1090C0005063D36A002BFCDA936B13F0800FF6D059
:1090D000012381F8803094E0012381F80031154BA1
:1090E0004FF00042DA6205225A63DA6A002AFCDA9B
:1090F000104B9B6B0F4A4FF000440020D46250632A
:10910000D36A002BFCDA936B13F0010FF6D1012325
:1091100081F8803075E000BFA4D5FF1FF0C6FF1FA7
:1091200080E100E0D8C6FF1FE4C6FF1F84E100E035
:1091300088E100E000C0024001401F0000001F80E5
:10914000A5D5FF1FA8D5FF1F9B4B1B78C3B113F0FC
:10915000010F03D0994B1A68994B1A60964B1B78F4
:1091600013F0020F03D0954B5A68964B1A60924B3E
:109170001B7813F0040F03D0904B9A68924B1A603F
:10918000FFF7E6FD8C4B1B78002B28D072B68A4B7C
:109190001B7813F0010F07D08C4B19688C4A1268AA
:1091A0000A4086490A601A60834B1B7813F0020F4D
:1091B00007D0884B1968864A52680A407F494A603E
:1091C0001A607D4B1B7813F0040F07D0824B19688F
:1091D0007F4A92680A4079498A601A6062B67F4B7A
:1091E000DB68B3F1384F0AD07C4B7D4A1A604FF0F0
:1091F0003842DA604FF078421A617A4A1A600023E6
:109200000293039901F00803DBB20093DFF8D8C1A1
:10921000012001EA00020192704B4FF000420099D8
:1092200061B108EB0901013981EA080111F07E4FB3
:1092300006D028F07E4BCBF1007B02E0CB4600E06D
:10924000CB46DCF8001081F800010199D9B1DA624F
:1092500003215963D96A0029FCDA996BDA624FEA73
:10926000184141F080515963D96A0029FCDA996BA1
:10927000DA621FFA88F141F080515963D96A0029F6
:10928000FCDA996B15E0DA62C8F3074141F08051CE
:1092900041F440715963D96A0029FCDA996BDA62AA
:1092A0001FFA88F141F080515963D96A0029FCDA2C
:1092B000996BBBF1000F18D09AF800101C6844F4A9
:1092C00080641C60DA625963BBF1010707D0574420
:1092D00051464D78DC6A002CC0F29280FAE757467E
:1092E000D96A0029C0F29980FAE7DCF8004084F8D6
:1092F0008000DA44D844B9EB0B0990D1029A002AD5
:1093000031D0012384F80031344B4FF00042DA624F
:1093100006225A631A46D36A002BFCDA2F4B9B6B4A
:10932000012384F880302023013B7FF4FDAF039BB1
:1093300013F0040F05D0029901290CBF8A227A226A
:1093400000E07A22012384F80031244B4FF00041E1
:10935000D9625A631A46D36A002BFCDA1F4B9B6B07
:10936000012384F88030144B1B78002B58D013F065
:10937000010F03D0114B1A68114B1A600E4B1B786A
:1093800013F0020F03D00D4B5A680E4B1A600A4BB4
:109390001B7813F0040F43D0084B9A680A4B1A60ED
:1093A0003EE0114B1968012381F88030029A022AAD
:1093B0007FF63EAEC8E600BFF0C6FF1FE4C6FF1F43
:1093C00000E100E004E100E008E100E080E100E00D
:1093D000D8C6FF1F84E100E088E100E000C0024041
:1093E00001401F0000001F80A8D5FF1F0E4B1B6807
:1093F000012283F8802000230C4A1370029300E7B7
:109400009C6B1E6846F480661E60DA625D6301F83C
:10941000014BB9427FF45DAF62E7996B397064E745
:1094200005B0BDE8F08F00BFA8D5FF1FA5D5FF1F71
:109430000B4B1B7813B90B4B1B7873B10A4B1B7882
:10944000202B03D90123037100207047581C064AC2
:109450001070064AD154012070470020704700BFA9
:1094600016D6FF1FD8D5FF1F17D6FF1FB4D5FF1F75
:10947000704700BF024B1878024B1B78C01A704728
:1094800015D6FF1F14D6FF1F074B1B78074A12780B
:109490009A4205D9591C044A1170054AD05C70479C
:1094A0004FF0FF30704700BF14D6FF1F15D6FF1FC7
:1094B000DCD5FF1F054B1B78054A12789A4286BF00
:1094C000044AD05C4FF0FF30704700BF14D6FF1F36
:1094D00015D6FF1FDCD5FF1F08B5104BDB7813F046
:1094E000200F0CD1122000F0B9FB0D4B1B689BB173
:1094F00000210C4A11700C4A1078984708BD0B4A9D
:1095000013780133DBB21370012B02D8084B1B78A0
:1095100013B9122000F0A2FB08BD00BF0060064096
:10952000B0D5FF1F14D6FF1F15D6FF1F00D6FF1F93
:10953000D8D5FF1F38B514460D4B1B7813B90D4B0A
:109540001B7893B10C4B1D78C5F12103A34202D2C5
:10955000012202711C4609482844224600F0B4F852
:109560002544054B1D70204638BD002038BD00BF86
:1095700016D6FF1FD8D5FF1F17D6FF1FB4D5FF1F64
:10958000002202714FF47A7181600273014A026015
:10959000704700BFD000010008B53D4BDB78DBB25F
:1095A00013F0100F06D01021394AD17013F0400F7C
:1095B00003D108BD13F0400F2CD013F0040F1BD0C3
:1095C0000023344A1370344A1370344B1B681BB1A8
:1095D0009847314B1B782BB901222F4B1A70002270
:1095E0002F4B1A702A4BD0229A702D4A12781A717A
:1095F00001222C4B1A7009E00122264B1A7000221E
:10960000294B1A70224BC0229A701B790222204BE0
:10961000DA7008BD1E4A927812F0100F1CD013F0B9
:10962000010F14D11F4B1B781B4A12789A4207D99D
:10963000591C1C4A11701A4AD25C154B1A7102E06F
:109640000022134B1A71D022114B9A701BE0104B61
:10965000C0229A701B7916E00022144B1A70122057
:109660001349032200F0C6FB094B1B79DAB20E4BFB
:109670001B781F2B07D80749097821B1581C0A49C4
:1096800008700C49CA540222014BDA7008BD00BFB1
:1096900000600640ACD5FF1F17D6FF1FFCD5FF1F8B
:1096A000B4D5FF1F18D6FF1F15D6FF1F00D6FF1F0A
:1096B000D9940000DCD5FF1F08B50248FFF760FF12
:1096C00008BD00BF04D6FF1F844641EA000313F023
:1096D00003036DD1403A41D351F8043B40F8043BB9
:1096E00051F8043B40F8043B51F8043B40F8043B7C
:1096F00051F8043B40F8043B51F8043B40F8043B6C
:1097000051F8043B40F8043B51F8043B40F8043B5B
:1097100051F8043B40F8043B51F8043B40F8043B4B
:1097200051F8043B40F8043B51F8043B40F8043B3B
:1097300051F8043B40F8043B51F8043B40F8043B2B
:1097400051F8043B40F8043B51F8043B40F8043B1B
:1097500051F8043B40F8043B403ABDD2303211D3BB
:1097600051F8043B40F8043B51F8043B40F8043BFB
:1097700051F8043B40F8043B51F8043B40F8043BEB
:10978000103AEDD20C3205D351F8043B40F8043BBB
:10979000043AF9D2043208D0D2071CBF11F8013BB9
:1097A00000F8013B01D30B8803806046704700BF7F
:1097B000082A13D38B078DD010F003038AD0C3F18E
:1097C0000403D21ADB071CBF11F8013B00F8013B70
:1097D00080D331F8023B20F8023B7BE7043AD9D32F
:1097E000013A11F8013B00F8013BF9D20B78037004
:1097F0004B7843708B7883706046704730B4394A39
:109800003949136813F0800FFBD10B6813F0800FF8
:10981000F7D172B6354B1B78002B5FD0344B1C68E8
:1098200004331D68043318680433196804331A6854
:1098300004331B682C44204401440A441A44C2F3F4
:109840004E0242F400422B4B1A602C331C68043346
:109850001D68043318680433196804331A68043324
:109860001B682C44204401440A441A44C2F34E02AB
:1098700042F40042204B1A6003F108131C680433C1
:109880001D68043318680433196804331A680433F4
:109890001B682C44204401440A441A44C2F34E027B
:1098A00042F40042154B1A602C331C6804331D68C7
:1098B000043318680433196804331A6804331B68C6
:1098C0002C44204401440A441A44C2F34E0242F498
:1098D00000420B4B1A600022044B1A7062B630BC77
:1098E000704700BF24B0034024B00B401AD6FF1FBE
:1098F00038B003402CB0034030B003402CB00B40D4
:1099000030B00B4060223A4B1A70E12201331A70DA
:10991000384B1B78082B10D1012203F1804303F54B
:109920006C331A60132334490B6001F5FF2101F2F7
:10993000FC710A60314A13601FE00A2B0DD13922F5
:109940002F4B1A6013232C490B6001F5FF2101F204
:10995000FC710A60294A13600FE00C2B0CBF352202
:109960003D22274B1A60122323490B6001F5FF218A
:1099700001F2FC710A60214A1360224B1B7833B15B
:109980000123214A136002F50022136005E0002341
:109990001D4A136002F5002213601C4B1B78012B3B
:1099A00006D880231A4A136002F5002213601AE0D9
:1099B000042B06D88423164A136002F50022136094
:1099C00011E0082B06D88523114A136002F5002206
:1099D000136008E0102B94BF862387230C4A136082
:1099E00002F50022136001220A4B1A70704700BF73
:1099F000004007400BA2FF1F0CB003400CB00B400F
:109A000008B003401DD6FF1F20B003400CA2FF1F6B
:109A100024B003401AD6FF1F2DE9F843282873D835
:109A20003C4B1E5CFF2E72D03B4B1B780BB1FFF7FB
:109A3000E5FE16F0800F29D172B6384C384D4FF044
:109A4000010726602F7062B672B6236813F0800F8C
:109A500004D12B7813F0FF0F0FD1F2E7314B1868C8
:109A600000222F4B1A7062B62F4B1B781841BDE8AD
:109A7000F8832B7813F0FF0FE3D062B602F0FAF808
:109A800072B6236813F0800FF3D0E7E772B606F0E2
:109A900040095FFA89F9254F254C06F03F06254D10
:109AA0004FF00108B9F1000F04D03B6823F0100318
:109AB0003B6003E03B6843F010033B60266085F8A1
:109AC000008062B672B6236813F0800F04D12B7841
:109AD00013F0FF0F0FD1E5E7174B18680022154B65
:109AE0001A7062B6104B1B781841BDE8F8832B78CA
:109AF00013F0FF0FD6D062B602F0BCF872B623683E
:109B000013F0800FF3D0E7E70020BDE8F8830020D2
:109B1000BDE8F883E80001001AD6FF1F00B003403B
:109B20001CD6FF1F10B0034019D6FF1F0CB00B400E
:109B300000B00B401BD6FF1F10B00B40024B1A6841
:109B400001321A60704700BF20D6FF1F08B50D4CC8
:109B5000236813F4802F01D000F0D8FE236813F49B
:109B6000806F01D000F05EFD236813F4006F01D018
:109B700002F0C4FB236813F4805FE9D002F07CFE9E
:109B8000E6E700BF3480044008B5FFF7DFFF00BF01
:109B90001022014B1A80704700200540704700BF1B
:109BA000024A1368184410601846704710A2FF1F3D
:109BB000FEE700BFEFF31383ABB9EFF31083ABB94C
:109BC000EFF3058323B10F2B05D9094A985C03E015
:109BD0004FF4807000E00020EFF311833BB183422B
:109BE00038BF184670474FF0FF307047002070476D
:109BF000F0E300E030B40023B0FBF2F402FB140405
:109C00001D46092C94BF30343734E4B2CC54B0FB39
:109C1000F2F008B10133EFE70D4400226A7093427D
:109C200007DD885CCC5C8C54C8540132013B9A42FD
:109C3000F7DB084630BC704710B50C46002802DB45
:109C4000FFF7D8FF10BD2D2301F8013B4042FFF77D
:109C5000D1FF204610BD00BF704700BF1D4B03EB76
:109C6000C000436803F14042A2F592227C2A18D931
:109C700003F14042A2F594227C2A14D903F1404218
:109C8000A2F596227C2A10D903F14042A2F598222F
:109C90007C2A0CD903F14042A2F59A227C2A08D9E9
:109CA00070470D4906E00D4904E00D4902E00D49F9
:109CB00000E00D4972B61A6822F0877222F48032F1
:109CC00042F080721A60C3F38403084A41F82320EB
:109CD00062B670471401010014A2FF1F4CA2FF1FBF
:109CE0009CA2FF1FCCA2FF1FECA2FF1F599C0000EB
:109CF000044B00221A6004490A60044A10601022D2
:109D00001A60704714D0034004D0034000D00340D1
:109D100021281ED80F4B53F8303093F8802212F0D0
:109D2000FF0F08D019B1012283F88020704701226B
:109D300083F800217047074B03EBC000436821B153
:109D40001A6842F003021A6070471A6822F0020291
:109D50001A60704714010100212806D8044B53F8FB
:109D6000303093F80002C0B270470020704700BF47
:109D70001401010021283AD81D4B03EBC0035B6896
:109D8000012919D0042925D0194A52F83020002081
:109D900082F8800219B94FF480721A607047022964
:109DA00003D140F203121A60704703290CBF4FF42D
:109DB000817200221A6070470D4A52F8302001214A
:109DC00082F880124FF4A2721A601A6822F0200200
:109DD0001A607047064A52F83020012182F880123A
:109DE0004FF4A2721A601A6842F020021A6070479B
:109DF0001401010070B50D46212861D8042A5FD8EE
:109E0000DFE802F00709050B03000B2306E00A2335
:109E100004E0082302E00C2300E009231E04294B80
:109E200003EBC0035C68236813F4E06F02D10021E8
:109E3000FFF7A0FF244B254AC3F89C21244AC3F80E
:109E4000A021244AC3F8A421234AC3F8A821234A05
:109E5000C3F8AC2104F14043A3F592237C2B18D91D
:109E600004F14042A2F594227C2A14D904F1404323
:109E7000A3F596237C2B10D904F14043A3F5982336
:109E80007C2B0CD904F14043A3F59A237C2B08D9F1
:109E900070BD134906E0134904E0134902E0134979
:109EA00000E0134972B6236823F470232360C4F3DF
:109EB000840241F8225043F080731E43266062B64C
:109EC00070BD00BF140101000092FF1F1198FF1F19
:109ED000E597FF1FB997FF1F8D97FF1F6197FF1F22
:109EE00014A2FF1F4CA2FF1F9CA2FF1FCCA2FF1FAA
:109EF000ECA2FF1F72B60C4B1B680C4A12680C498F
:109F0000096862B611F0806F02D0322B88BF01322F
:109F1000C3F5BB33FF330749A1FB03039B094FF490
:109F20007A7000FB0230704718E000E020D6FF1F77
:109F300004ED00E0ABAAAAAA38B50546FFF7DAFFA0
:109F4000044625B938BD013D0AD004F57A74FFF7FF
:109F5000D1FF001BB0F57A7FF5D201F08BFEF6E75A
:109F600038BD00BF10B5264B4FF400021A604FF009
:109F700080721A604FF000721A604FF080621A60AF
:109F80004FF000621A6000201E4B18604BF6FF7104
:109F90000433196028231C4A136008321360083206
:109FA00013600832136008321360083213600832FD
:109FB0001360083213600922144C226004F58054A7
:109FC00004342060043421600434236008342360A6
:109FD000143C226004F5FE24043420600C48016027
:109FE0000C490B6008310B600B4B1A60FFF78AFCC1
:109FF0004FF4C870FFF7A0FF01F008F810BD00BFD4
:10A0000008E100E0048003400C800340008003402E
:10A0100008800B400C800B4000800B40254B1A68D9
:10A0200042F480621A600023234A1370234A13709B
:10A03000234A1370234A1370234A1370234B1B784F
:10A0400013B1152B05D008E040F21332204B1A60F3
:10A0500003E040F213321F4B1A601F4B1B78012B99
:10A0600002D0052B05D008E04FF451721B4B1A604B
:10A0700003E04FF451721A4B1A60C0F34432194B8B
:10A080001A70C0F347125A7000F01F009872042231
:10A090009A700221D9745A7588221A743C22DA7097
:10A0A0004022114B1A704FF40052A3F229331A6068
:10A0B000704700BF34800440B0D6FF1F29D6FF1F71
:10A0C000B8D6FF1FB1D6FF1F28D6FF1F6CD6FF1FC3
:10A0D00040A0044018C00440F4A2FF1F44A0044064
:10A0E0001CC0044000A006402DE400E0164B9B7805
:10A0F00003F0EC0300F00302134310F0040F18BF49
:10A1000043F01003104A937000F00F03042B04D1A6
:10A110001346927942F040029A710B4B5A7902F041
:10A12000EF0210F0100F18BF42F01002064B5A71E8
:10A130009B7903F0EF0310F0200F18BF43F01003DA
:10A14000014A9371704700BF00A0064010B5144B40
:10A150001B6813F4806F21D0124B1B7813F0FF0F94
:10A1600006D0104C01F086FD237813F0FF0FF9D1D3
:10A170004FF400520C4B1A6000230C4AD37040F28B
:10A1800003120B490A6004310A600A4A13700A4A32
:10A1900013700A4B1B680BB101221A7010BD00BF6F
:10A1A0003480044028D6FF1F84E100E000A0064070
:10A1B00040A00440B0D6FF1F29D6FF1F24D6FF1FA2
:10A1C00010B50446094A137813F0FF0FFBD120465F
:10A1D0000121FFF7CFFD20460021FFF799FD044B39
:10A1E00053F83420034B1A6010BD00BF28D6FF1F60
:10A1F00014010100B4D6FF1F10B40C4609B140F0A1
:10A200008000184B1B78984228D0174A126812F425
:10A21000806F21D003F07F03012B02D0052B04D0E7
:10A2200006E00022114B1A6002E00022104B1A6077
:10A23000002C0CBF4422602200F07F03012B02D0CF
:10A24000052B05D008E042F44072084B1A6003E089
:10A2500042F44072064B1A60024B18705DF8044BD2
:10A26000704700BFF4A2FF1F3480044044A00440A4
:10A270001CC00440114B1B7898421ED0104A126833
:10A2800012F4806F17D013B1152B04D006E0002212
:10A290000C4B1A6002E000220B4B1A6010B115281B
:10A2A00005D008E040F21332064B1A6003E040F29A
:10A2B0001332054B1A60014B187070476CD6FF1FA4
:10A2C0003480044040A0044018C0044010B50D4B39
:10A2D0001B6813F4806F12D021280CD80A4C0B4B4A
:10A2E00053F8303023600121FFF744FD236800223A
:10A2F0001A70012010BD0020034B186010BD002013
:10A3000010BD00BF3480044024D6FF1F140101009B
:10A31000114B1B6813F4806F1BD0122804D140F23C
:10A3200002320E4B1A600DE0142804D140F20232C2
:10A330000B4B1A6006E00B4B5A7B02F0FE025A737D
:10A3400000207047074B5A7B42F001025A730120EC
:10A3500070470020704700BF348004400CA00440C8
:10A3600014C0044000A006402DE9F04107461F4BF1
:10A370001B6813F4806F37D01D4B1B680BB1012293
:10A380001A701C4B1C780134402C28BF00241A4D35
:10A390001A4EDFF86C8017E0FFF70CFC40280FDC4A
:10A3A000337913F0800F0FD02B780133402B28BF67
:10A3B000002318F80320D2B2F271DBB22B7003E055
:10A3C000FF2801DD01F056FC2B78DBB29C42E3D084
:10A3D000FFB20B4B1F5501220A4B1A70E4B2054B1A
:10A3E0001C70BC22054BDA70BDE8F081348004405B
:10A3F000B4D6FF1FB8D6FF1FB1D6FF1F00A006407E
:10A400002CD6FF1F28D6FF1F2DE9F84F0746284BF3
:10A410001B6813F4806F49D0264B1B680BB10122D7
:10A420001A7007EB010B5F453DD2DFF89890224E82
:10A43000DFF88C80DFF890A099F800400134402CC0
:10A4400028BF00243578EDB2A54220D1BC2388F87E
:10A450000330FFF7AFFB402811DC98F8043013F00D
:10A46000800F10D033780133402B28BF00231AF817
:10A470000320D2B288F80720DBB2337003E0FF2854
:10A4800001DD01F0F7FB3378DBB29D42E1D017F834
:10A49000013B0AF804300122084B1A70E4B289F833
:10A4A00000405F45C8D1BC22054BDA70BDE8F88F8B
:10A4B00034800440B4D6FF1FB1D6FF1F28D6FF1F3B
:10A4C00000A00640B8D6FF1F2CD6FF1F10B5064BC4
:10A4D0001B7813F0FF0F06D0034C01F0CBFB237861
:10A4E00013F0FF0FF9D110BD28D6FF1F064B1B78C4
:10A4F000DBB2064A1278D2B293422CBF3F3202F14D
:10A50000FF32D01A704700BFB8D6FF1FB1D6FF1F69
:10A51000054B1878C0B2054B1B78DBB2984238BFA8
:10A520004030C01A704700BFB0D6FF1F29D6FF1FAA
:10A5300010B4184B1A78D2B2174B1B78DBB29A4280
:10A5400018D001333F2B18D81449C85CC0B2DCB214
:10A5500011490C7012490968C9B19A4203D300E04D
:10A560000023D31A01E04032D31A1A2B0FDC002348
:10A570000B700CE04FF0FF3009E0084B1878C0B2C8
:10A580000021054B1970064B19680029E8D15DF8C8
:10A59000044B7047B0D6FF1F29D6FF1F70D6FF1F90
:10A5A00024D6FF1F094B1A78D2B2094B1B78DBB2B5
:10A5B0009A4207D00133402B28BF0023054AD05CC4
:10A5C000C0B270474FF0FF30704700BFB0D6FF1FDA
:10A5D00029D6FF1F70D6FF1F0D4B1B6813F4806F29
:10A5E00014D00C4BDA7802F0CB02DA7040225A74A5
:10A5F000DA7842F03402DA70074B1A78D2B2074B9D
:10A600001A70074B1B680BB100221A70704700BF0D
:10A610003480044000A0064029D6FF1FB0D6FF1F9B
:10A6200024D6FF1F70B43D4B1B7913F0300F33D08D
:10A6300072B63A4B9B7D03F0FF022BB9374BDA79A8
:10A6400040225A7462B627E062B6354B1978C9B217
:10A65000344B1C78E4B2314D334EEB79D8B24B1CFD
:10A66000402B28BF0023A3421CBFF0541946531EA1
:10A6700013F0FF02F1D1CAB2294B1A702B4B1B68A1
:10A6800053B1A1422EBFC4EB0101C4F1400409192A
:10A690002729C4BF01221A70204BDA78D2B212F0F7
:10A6A000800F27D01B7913F0800F23D0204B1C780C
:10A6B000E4B2204B1B78DBB29C4210D017491E4DF0
:10A6C00001E0A3420BD00133402B28BF00230879BF
:10A6D000E85CC0B2C871087DC0B20728F1D9DBB20E
:10A6E00014490B700D4B1B7913F0800F02D07C21A5
:10A6F0000A4BD97012F0400F0ED0084B1B7913F0A3
:10A70000400F09D000220D4B1A700D4B1B6803B18E
:10A710001A703C22014BDA7070BC704700A00640F2
:10A72000B0D6FF1F29D6FF1F70D6FF1F24D6FF1FEC
:10A73000B8D6FF1FB1D6FF1F2CD6FF1F28D6FF1F8C
:10A74000B4D6FF1F30B40E4B1B7843F002020D4C01
:10A7500004EBC20460600C48007800280CBF882419
:10A76000C82444EA0141074D45F8321080F0010049
:10A77000054A107083F00103014A137030BC704722
:10A7800024D7FF1F0080FF1F9DD7FF1F10B4431E5B
:10A79000032B11D872B60A4A52F8230050B142680E
:10A7A000074941F82320074A32F813400188611A0B
:10A7B00022F8131062B600E000205DF8044B7047E9
:10A7C00014D7FF1F54D9FF1F013803280DD872B6C4
:10A7D000074B53F820302BB1002001305B68002B71
:10A7E000FBD100E0002062B670470020704700BF38
:10A7F00068D7FF1F38B572B601231B491B4C5A1886
:10A8000012F8012C12F0080F24D09A0054F832509C
:10A810006DB9164B03EBC20108304860144943F888
:10A820003210144B1A78013A1A7062B638BD42F0F1
:10A83000010254F832506DB90C4B03EBC2010830E1
:10A8400048600D4943F832100A4B1A78013A1A70E1
:10A8500062B638BD0133052BD1D162B60022054B5B
:10A860001A7000F037FC38BD600201000080FF1F45
:10A870008800400092D7FF1FC800400010B4431E5C
:10A88000032B37D8400140F010001C4A104472B628
:10A890001B4AD25C032A09D8DFE802F019021B0523
:10A8A0000830022216E00830042213E0154A52F85C
:10A8B00023201AB9134A42F8231003E0124A52F82F
:10A8C00023205160104A42F8231062B612E003229E
:10A8D00000E005220A4CE25401F10803436000F055
:10A8E0000803002B0CBF8823C8230A8843EA0243CD
:10A8F000036062B65DF8044B704700BF0080FF1F25
:10A90000D0D6FF1F68D7FF1F78D7FF1F2DE9F84F5C
:10A91000A34CDFF8E092DFF8E0A2DFF8E0B22578A0
:10A92000EDB215F0040F1DD09E4B1B7813F0FF0FF6
:10A9300016D09D4B1B7803F0FF022BB1531EDBB2E8
:10A94000994A137003B900BE984B1B7803F0FF02BD
:10A9500033B1531EDBB2954A13700BB900F018FDEA
:10A960000423237015F0080F00F0E48299F80030FA
:10A97000DBB21D0940F021828D4D9E0805EBC60318
:10A980005A6855F83630C3F38303013B0C2B00F2B1
:10A990001082DFE813F0CB01CB010E020E020E0293
:10A9A0000E020E020E02E8010E020E020E020D0051
:10A9B000804913680B6052684A607F4A45F8362028
:10A9C00000227E490A607A490A618A6101217C4A33
:10A9D00011709BB240F28162934218D8B3F5D06FE8
:10A9E0002ED2B3F5817F00F01E8106D8802B00F0B7
:10A9F000C980822B00F0CC8066E140F202329342A3
:10AA000000F02681B3F5A06F00F062815CE142F2B4
:10AA10002102934200F0868107D8B3F5086F00F059
:10AA2000AB80B3F5106F11D04EE142F22122934278
:10AA300000F0418142F22132934200F0498143E12A
:10AA4000604B5D68002D40F0188130E1594B9A78D9
:10AA5000544B1A70564D05F180062B6A13F0800F87
:10AA600003D0686A083800F035FB0835B542F4D1E8
:10AA7000DFF88C8100263746534AB05828B1456824
:10AA800000F028FB0DB12846F9E700234E4973502A
:10AA90004E4AB3504E4BF05828B1456800F01AFBAF
:10AAA0000DB12846F9E7002349497350494AB3508C
:10AAB00028F8023F484BFB5C023B032B0AD8DFE837
:10AAC00003F0020602060022434BDA5502E001229F
:10AAD000414BDA5501370436102ECDD100223F4BC1
:10AAE0001A7001253E4EDFF81C81314F05EB08033B
:10AAF00013F8013C06F8043B13F0080F2DD000F0CA
:10AB0000C9FA48B1A90007EB451200F108035360E8
:10AB1000344A47F8312007E0AB00002247F83320E1
:10AB20002E4B1A7801321A7000F0B4FA58B1AB000B
:10AB300043F0010307EBC30100F108024A601E4A1B
:10AB400047F8332009E0AB0043F00103002247F847
:10AB50003320224B1A7801321A70AA0042F0020107
:10AB6000002347F8313042F0030247F83230013514
:10AB70001D4B9E42BAD11EE20A4B1B781B4D2B7017
:10AB80000127AAE0194D00232B706B700227A4E067
:10AB9000084B9B88042B37D90F22154B1A70C1E044
:10ABA000802007409CD7FF1F25D7FF1F9ED7FF1F80
:10ABB0000080FF1F88D7FF1FC8004000BCD6FF1FC2
:10ABC0009DD7FF1F6402010014D7FF1FC0D6FF1FCF
:10ABD00068D7FF1F78D7FF1FD0D6FF1F92D7FF1F60
:10ABE000C420074088004000D420074094D7FF1FAE
:10ABF000C02007409020074094200740982007403D
:10AC000052D9FF1F60020100A04A0021117051704B
:10AC10009F4A12F8233013F0020F5CD09B4D0123A2
:10AC20002B70022759E09B4B9B8803F07F03042B7A
:10AC300002DC984A52881AB10F22954B1A7071E0C3
:10AC4000934A12F8231021F0020102F82310B2E116
:10AC5000904B9B8803F07F03042B02DC8D4A5288C3
:10AC60001AB10F228A4B1A705CE0894A12F823103D
:10AC700041F0020102F823109DE1864B5E889F8817
:10AC8000854BA3F10C02114633F80C0CB04209D1EC
:10AC900033F80A0CB84205D1360A032E0CBF2F78C0
:10ACA00017891AE00D690C330C32002DEBD10F22FD
:10ACB000774B1A7036E0794B1A68794B1A60754BEE
:10ACC0009A78784B1A7076E10F22714B1A7029E04E
:10ACD00000273D4601E002276C4D6E4BDB889F420A
:10ACE00028BF1F46402F34BF3E46402628463146E7
:10ACF000FFF728FD3544BF1B03D13F2E00F26081D2
:10AD000010E0402F34BF3E46402628463146FFF72C
:10AD100019FD3544BF1B01D13F2E03D9624B1D6085
:10AD2000624B1F8001238AF8003042E0594B19889A
:10AD300042F22103994212D15D4BD81D12F8011B3A
:10AD400003F8011F8342F9D15A4B1B68862B02D1AD
:10AD50000F22594B1A7000200146FFF7F3FC574BA6
:10AD600045F8363025E0504B1E68BEB14F4FB7F85E
:10AD70000080B8F1400F34BF454640253046294693
:10AD8000FFF7E0FCC5EB08039BB23B800BB9402DFD
:10AD900001D1354400E00025434B1D603D4B1B882D
:10ADA000B3F5A06F05D13B4B00225A709B788BF80E
:10ADB000003001238AF80030B9E0414E9F0806EBCD
:10ADC000C708D8F80420A2F10800013DEDB213F045
:10ADD000080F47D000F07EF93A4B53F825304BB3BB
:10ADE0005A68384941F8252003F10802C8F80420C0
:10ADF000354A525D032A12D8DFE802F002060A0E35
:10AE00000321314A51550AE002212F4A515506E0EB
:10AE100005212D4A515502E004212B4A515518F0C5
:10AE2000080F0CBF8822C8221B8842EA034346F859
:10AE300037307CE0244B5B5D032B0BD8DFE803F05D
:10AE4000777702060022204B5A5570E001221E4BF4
:10AE50005A556CE018F0080F0CBF022203221A4B5F
:10AE60005A5564E056F837301B0C22F8083C002B8A
:10AE700055D0002322F8063C42F8043C134B53F80B
:10AE800025302BBB114B43F8250025E094D7FF1F3D
:10AE9000C020074088D7FF1F7002010020D6FF1F87
:10AEA00064D9FF1FACD7FF1FBCD6FF1F90D7FF1F71
:10AEB0005BD9FF1F5CD9FF1F25D7FF1FC8004000CB
:10AEC0000080FF1F68D7FF1FD0D6FF1F14D7FF1FBA
:10AED0003F4B53F8253058603D4B43F825003D4B20
:10AEE00033F8151032F8082C0A4423F8152000F026
:10AEF000D1F860B100F10803C8F8043018F0080F69
:10AF0000354B364A08BF134646F837300FE000236A
:10AF100046F83730324B1A7801321A7007E018F0D1
:10AF2000080F2D4B2D4A08BF134646F8373008232B
:10AF30002370F4E415F0010F22D02A4902230B708C
:10AF40000022294B1A70294B24481860284C5C6059
:10AF500098602848D8601A619A610D20264B1870B5
:10AF6000FF23264803700838037018300270244A03
:10AF700013709F22234B1A7001230B70BDE8F88FCA
:10AF800015F0800F05D00D221B4B1A708022403B1C
:10AF90001A7015F0020F06D0184B1A78D2B21A7038
:10AFA0000222083B1A7015F0100F0ED01022164B1B
:10AFB0001A70BDE8F88F00200146FFF7C3FBB1E629
:10AFC00028460021FFF7BEFBACE6BDE8F88F00BFC6
:10AFD000C0D6FF1F54D9FF1FC800400088004000A2
:10AFE00092D7FF1F9420074024D7FF1F0080FF1F28
:10AFF000D4D6FF1F28D7FF1FC02007408820074056
:10B000008C200740842007408020074008B501F0CD
:10B01000A7FC00231B491A465A50C818426008333F
:10B02000882BF9D1184B1A6842F480221A60154B0C
:10B03000C3F30721154A1170C3F30741143211708D
:10B040001B0E04321370FF23343A1370083213704E
:10B05000783A137001238432137000216C3211701E
:10B060007C3A137070220A4B1A704FF40072A3F2EC
:10B0700041331A60102203F1C04303F5C8231A704C
:10B0800008BD00BF0080FF1F348004409C200740A3
:10B0900049E400E072B60D4B1A68B2FA82F30B2B4A
:10B0A00002D962B6002070474FF00041D94022EA31
:10B0B000010206490A6062B6054903EBC303DB00DF
:10B0C000C8180022CA504260704700BFF8A2FF1F94
:10B0D0000094FF1F08B50F4BC31A0F4AA2FB0313BE
:10B0E0001B090B2B14D80D4A12783AB10C4A12786E
:10B0F00012F0FF0F02D0FFF77DFB08BD72B6094AC0
:10B100004FF0004121FA03F311681943116062B650
:10B1100008BD00BF0094FF1F398EE33892D7FF1F90
:10B120009CD7FF1FF8A2FF1F10B5134B1B6853B924
:10B13000124B1B7813F0FF0F18D00320FFF726FBEC
:10B140000D4B1860A8B10C4B186843885A1C034477
:10B150001C7A03889A4206D3FFF7BCFF0022064BF5
:10B160001A60204610BD4280204610BD4FF0FF30CF
:10B1700010BD4FF0FF3010BDA8D7FF1F9CD7FF1F99
:10B1800008B50D4B1B6883B90C4B1B7813F0FF0FF0
:10B1900008D00320FFF7FAFA074B186028B94FF0E0
:10B1A000FF3008BD4FF0FF3008BD034B1B685A88C5
:10B1B0001344187A08BD00BFA8D7FF1F9CD7FF1FF4
:10B1C000044B9888044B1B681BB11A885B88D31A00
:10B1D0001844704754D9FF1FA8D7FF1F10B50B4B59
:10B1E0001B7813F0FF0F0FD0094B186820B1FFF741
:10B1F00071FF0022064B1A6003242046FFF7C6FAAF
:10B2000010B1FFF767FFF8E710BD00BF9CD7FF1F25
:10B21000A8D7FF1F2DE9F84F04460122384B1A70BA
:10B220008B46002965D00E46DFF8E080DFF8E0901D
:10B230009A46344FD8F8003083BB99F8003013F0A9
:10B24000FF0F06D100222E4B1A704FF0FF30BDE8E1
:10B25000F88F4AF2F9250420FFF7B6FA07280AD832
:10B2600001238AF80030FFF715FFC8F80000A8B9DD
:10B2700000238AF80030013D01D03B7833B1012230
:10B28000204B1A704FF0FF30BDE8F88F00F0F2FC51
:10B2900099F8003013F0FF0FDDD1D3E700233B70A6
:10B2A000D8F800104A88C2F14005AE4238BF354692
:10B2B00002F108030B442A444A80761B3DB1254421
:10B2C00014F8012B03F8012BAC42F9D100E025461C
:10B2D0004B883F2B07D940230B800420FFF7CEFA81
:10B2E0000023C8F800300522074B1A700EB12C4617
:10B2F000A0E70022024B1A705846BDE8F88F00BF45
:10B300009FD7FF1FA4D7FF1F9ED7FF1FA0D7FF1FE8
:10B310009CD7FF1F00B583B002AB03F8010D1846A0
:10B320000121FFF777FF03B05DF804FB10B5144B64
:10B330001B7813F0FF0F21D00122124B1A70124B11
:10B34000196851B10024114B1C704B880B800420EC
:10B35000FFF794FA0C4B1C600DE0FFF79BFE0146D3
:10B3600030B10022094B1A700420FFF787FA02E07F
:10B370000122064B1A700022024B1A7010BD00BF4A
:10B380009CD7FF1F9FD7FF1FA0D7FF1F9ED7FF1F70
:10B3900008B50E4B1B7813F0FF0F16D10C4B196834
:10B3A00041B14B880B800420FFF768FA0022084B5C
:10B3B0001A6008BDFFF76EFE014618B10420FFF7C2
:10B3C0005DFA08BD0122034B1A7008BD9FD7FF1F0D
:10B3D000A0D7FF1F9ED7FF1FF0B4C02928BFC021F0
:10B3E00072B6134B1860134B00221A605A609A60B1
:10B3F000DA601A615A61C1B113460E4C01275A092D
:10B4000003F01F0607FA06F654F82250354344F8B5
:10B41000225001338B42F2D100221346841863700C
:10B42000013302F582728B42F8D162B6F0BC7047EC
:10B43000B8D7FF1FC0D7FF1F10B472B6234B1B68CD
:10B440008BB9224B5B6883B9204B9B687BB91F4B40
:10B45000DB6873B91D4B1B696BB91C4B5B6963B926
:10B4600062B600202EE0194A08E0194A06E0194A9F
:10B4700004E0194A02E0194A00E0194AB3FA83F1DC
:10B480004FF00040C84023EA0003136015480378DA
:10B490000133DBB2037062B60C48121A9210C1EB92
:10B4A000421202EB821241F67C7101EB82020E49DC
:10B4B0000968881801248C540C4A12789A423CBFBF
:10B4C0000A4A13705DF8044B704700BFC0D7FF1FD6
:10B4D000C4D7FF1FC8D7FF1FCCD7FF1FD0D7FF1F70
:10B4E000D4D7FF1FBDD7FF1FB8D7FF1FB4D7FF1F8B
:10B4F000427872B60378012B02D9013B037011E048
:10B500005111094BD24302F01F024FF0004020FAC4
:10B5100002F253F82100104343F82100034B1A783C
:10B52000013A1A7062B67047C0D7FF1FBDD7FF1F20
:10B5300030B4C36883B1187A90420AD158685C7AF3
:10B54000006950F8245025B940F8241008780130DB
:10B550000870DB68002BEED130BC7047437A8B4219
:10B5600006D9036953F82100002243F821207047CF
:10B570000020704738B5437A8B4218D9036953F8D5
:10B580002140002243F821209CB12378012B12D9BD
:10B59000FFF752FF054628B10430211D4FF4807299
:10B5A000FEF792F82378013B2370284638BD00202F
:10B5B00038BD204638BD204638BD00BF4368427ABA
:10B5C0005B7A9A4210D872B60368DA680AB9D86012
:10B5D00004E0D3680BB11A46FBE7D0600268012390
:10B5E00013724268137262B6704700BF084B1B7833
:10B5F0005BB9D022074B1A704FF08042A3F256334A
:10B600001A600120024B187070470020704700BF7D
:10B61000BCD7FF1F5EE400E0F8B5184B1A6842F093
:10B6200080721A60164B1A6842F001021A600433E5
:10B630001F68144B1C689CB1134D237A6BB12E68A4
:10B6400023681B68204698472B689B1B1B099AB2EE
:10B65000A280E1888B4288BFE2806469002CECD133
:10B66000094B1B68DF1B3F09BBB2084A1380084A1D
:10B670001288974284BF064A1380F8BDFCED00E0B3
:10B68000001000E0B0D7FF1F041000E0D8D7FF1F64
:10B69000BED7FF1F30B472B699B902688AB1037978
:10B6A0000F2B0ED827490988194111F0010F08D036
:10B6B00003F1007303F59063B2EB431F01D162B64F
:10B6C0003EE0204B1D882946002341FA03F212F088
:10B6D000010F2DD1012202FA03F42543194A1580E6
:10B6E00062B6DAB2027118490C6844F002040C60C8
:10B6F00004390C6844F002040C60822413490C6085
:10B700001A310A7004310A7006390A7007310A705A
:10B7100003F1007303F590635B01036000221A607C
:10B720005A609A60DA601A615A619A61DA6107E0D8
:10B730000133102BC9D162B60023036010230371BB
:10B7400030BC7047DAD7FF1F4080044000800040C3
:10B7500003790F2B10D8094A137072B6084B02797F
:10B76000012101FA02F2198821EA02021A8062B666
:10B770001023037100230360704700BF1A8000404C
:10B78000DAD7FF1F2DE9F0438BB0074688468C6857
:10B79000C4B100252E464FF02109404601A94A4672
:10B7A0002B4600F017FA202C34BF224620221544E5
:10B7B000A41A3B685B68384601A998470644002CE8
:10B7C000EBD100E0002630460BB0BDE8F08300BFAF
:10B7D00000B583B0054B1B88ADF8043003685B6887
:10B7E00001A90222984703B05DF804FB240201007E
:10B7F000F0B58BB0164622B903681B68C9B29847EA
:10B800002FE0012A08BF0A2621B930228DF8252011
:10B81000212417E021243746B1FBF6F506FB151568
:10B82000EDB22246092D94BF30353735EDB20DF11A
:10B83000280E724402F8245CB1FBF7F111B1013C0F
:10B84000E4B2E9E733B1013CE4B20AAB23442D2270
:10B8500003F8242C03685B6801A92144C4F1220287
:10B8600098470BB0F0BD00BF08B50029BABF4942E8
:10B870002D2300230A22FFF7BBFF08BDFFFFFFFFB8
:10B880002DE9F04F85B0804614461D469DF838904E
:10B890001046194601F08EFA40B9D8F800305B68BE
:10B8A00040466749032298470746BEE0204629469E
:10B8B00001F080FA012808D1D8F800305B684046D2
:10B8C0006049032298470746AFE0204629464FF0DB
:10B8D00060425D4B01F0DEFE40B1D8F800305B689D
:10B8E00040465A490322984707469EE0204629468B
:10B8F0004FF06042564B01F0AFFE40B1D8F8003037
:10B900005B68404651490322984707468DE0204630
:10B9100029460022002301F09FFE28B105F10043D3
:10B920001D464FF0010A01E04FF0000AB9F1000F87
:10B930006CD04FF0000B0022464B3FA7D7E90067C1
:10B940001046194632463B4601F014FC02460B46AF
:10B950000BF1010B5FFA8BF18945F1D82CE04E46D3
:10B960002046294600223C4B01F004FC04460D46CB
:10B9700001F09AFEC0B206F101095FFA89F904AB41
:10B980001E4400F1300306F8103C01F08DFB024626
:10B990000B462046294601F039FA04460D46D145AA
:10B9A000DDD101E04FF0010AD8F800305B68404675
:10B9B00069465246984738E02046294601F028FA61
:10B9C00004460D4601F070FE064601F05DFB02469E
:10B9D0000B462046294601F019FA04460D4640461A
:10B9E00031460A225346FFF703FF07462E238DF800
:10B9F0000030B9F10F0F34BF4B460F23002BD1D0CD
:10BA000003F1010A5FFA8AFA0126A9E720462946CE
:10BA10000022104B01F0FCF901F046FE01464046C1
:10BA20000A225346FFF7E4FE0746384605B0BDE854
:10BA3000F08F00BFAFF30080000000A09999B93FDC
:10BA4000280201002C020100FFFFEF41300201003B
:10BA5000FFFFEFC10000E03F00002440AFF3008093
:10BA600008B1014A10607047DCD7FF1F10B4124BB9
:10BA70001968D9B1114C81FB0423CA18CB17C3EB49
:10BA800022420F4800FB121284FB01042144C3EB45
:10BA900021430C4800FB03F344F2A71000FB0230E3
:10BAA000002804DA00F10040013800E00648024BAB
:10BAB00018605DF8044B7047DCD7FF1F5F0B4E83A7
:10BAC0001DF30100ECF4FFFF42CE0C1F10B504463D
:10BAD00030B1FFF7CBFFB0FBF4F303FB140010BD54
:10BAE000002010BD10B50446884204DA081AFFF79A
:10BAF000EDFF204410BD10BD10B4401A019CE41AA3
:10BB000004FB00F4521A94FBF2F018445DF8044B65
:10BB1000704700BF10B50446006802F051F9204696
:10BB200010BD00BF38B504460D460068013102F073
:10BB3000CDFC18B120606560012038BD002038BD03
:10BB400010B5044643688B420AD2FFF7EBFF034669
:10BB500048B1A36833B9236800221A70012302E0B8
:10BB6000012300E00123184610BD00BF70B5044654
:10BB70000E4615462AB9036803B11A700023A36064
:10BB800012E01146FFF7DCFF48B9206818B102F057
:10BB900017F90023236000236360A36004E0A5601D
:10BBA0002068314603F03CF8204670BD38B50446A5
:10BBB000002303604360836003730D4639B1084678
:10BBC00003F08CF8024620462946FFF7CFFF2046B7
:10BBD00038BD00BF38B50C469AB191B18168994221
:10BBE00002D80023237038BD551EC91A8D4228BFC4
:10BBF0000D460168204619442A4603F09FF80023A9
:10BC0000635538BD08B5F9F749FDF9F7B3FB00F006
:10BC100031F8FAE708B5FFF7D3FA08BD08B5FFF722
:10BC200083FA08BD08B5FFF7ABFA08BD08B5FFF702
:10BC30007DFB08BD08B5FFF7D1FA08BD08B5084679
:10BC4000FFF768FB08BD00BF08B508461146FFF7BF
:10BC5000E1FA08BD704700BF044B00221A714FF48F
:10BC60007A7199601A73024A1A607047E4D7FF1F0D
:10BC70004002010008B50F4B1B78CBB901220D4BD8
:10BC80001A70FFF79DFA08B1FFF7E4FFFEF740FCDA
:10BC900008B100F03BFF00F0A7FA08B100F0D8FFB0
:10BCA00000F074FD08B101F075F80022014B1A7024
:10BCB00008BD00BFF4D7FF1F254B1A6842F400628D
:10BCC0001A600023234A1370234A1370234A137007
:10BCD000234A1370234A1370234B1B78092B02D07D
:10BCE0001A2B05D008E040F21332204B1A6003E013
:10BCF00040F213321E4B1A601E4B1B780A2B02D0E7
:10BD00001F2B05D008E04FF451721B4B1A6003E063
:10BD10004FF45172194B1A60C0F34432184B1A7029
:10BD2000C0F347125A7000F01F00987204229A70F4
:10BD30000221D9745A7588221A743C22DA70402282
:10BD4000104B1A704FF40042A3F22B331A60704765
:10BD50003480044068D8FF1FFDD7FF1F70D8FF1F35
:10BD600069D8FF1FFCD7FF1FFCA2FF1F0CB00440C7
:10BD700004D00440FDA2FF1F10B0044000D00440D6
:10BD800000B006402FE400E0164B9B7803F0EC0374
:10BD900000F00302134310F0040F18BF43F0100328
:10BDA000104A937000F00F03042B04D113469279CC
:10BDB00042F040029A710B4B5A7902F0EF0210F0F8
:10BDC000100F18BF42F01002064B5A719B7903F016
:10BDD000EF0310F0200F18BF43F01003014A9371D6
:10BDE000704700BF00B0064010B5224B1B6813F42B
:10BDF000006F3ED0204B1B7813F0FF0F06D01E4C77
:10BE0000FFF738FF237813F0FF0FF9D14FF400420A
:10BE10001A4B1A6000221A4BDA701A4B1B78092B46
:10BE200002D01A2B05D008E040F20312164B1A601C
:10BE300003E040F20312154B1A60154B1B7803F018
:10BE40007F030A2B02D01F2B05D008E040F203121B
:10BE5000104B1A6003E040F203120F4B1A600023EC
:10BE60000E4A13700E4A13700E4B1B680BB1012261
:10BE70001A7010BD34800440FCD7FF1F84E100E03D
:10BE800000B00640FCA2FF1F0CB0044004D00440E8
:10BE9000FDA2FF1F10B0044000D0044068D8FF1F6F
:10BEA000FDD7FF1FF8D7FF1F10B50446094A1378C6
:10BEB00013F0FF0FFBD120460121FDF75BFF204669
:10BEC0000021FDF725FF044B53F83420034B1A6083
:10BED00010BD00BFFCD7FF1F140101006CD8FF1F6D
:10BEE00010B40C4609B140F08000184B1B78984202
:10BEF00028D0174A126812F4006F21D003F07F0394
:10BF00000A2B02D01F2B04D006E00022114B1A602E
:10BF100002E00022104B1A60002C0CBF4422602269
:10BF200000F07F030A2B02D01F2B05D008E042F45B
:10BF30004072084B1A6003E042F44072064B1A60EC
:10BF4000024B18705DF8044B704700BFFDA2FF1F45
:10BF50003480044010B0044000D00440124B1B78E1
:10BF6000984220D0114A126812F4006F19D0092BA0
:10BF700002D01A2B04D006E000220D4B1A6002E01A
:10BF800000220C4B1A60092802D01A2805D008E0BC
:10BF900040F21332064B1A6003E040F21332054BB5
:10BFA0001A60014B18707047FCA2FF1F34800440D8
:10BFB0000CB0044004D0044010B50D4B1B6813F4C2
:10BFC000006F12D021280CD80A4C0B4B53F830309C
:10BFD00023600121FDF7CEFE236800221A700120A4
:10BFE00010BD0020034B186010BD002010BD00BF25
:10BFF00034800440F8D7FF1F140101000D4B1B686B
:10C0000013F4006F13D017280AD140F202320A4B02
:10C010001A600A4B5A7B42F001025A7301207047A2
:10C02000064B5A7B02F0FE025A7300207047002034
:10C03000704700BF3480044008B0044000B00640A0
:10C040002DE9F04107461F4B1B6813F4006F37D0F2
:10C050001D4B1B680BB101221A701C4B1C7801345C
:10C06000282C28BF00241A4D1A4EDFF86C8017E0E8
:10C07000FDF7A0FD40280FDC337913F0800F0FD0BF
:10C080002B780133282B28BF002318F80320D2B2C5
:10C09000F271DBB22B7003E0FF2801DDFFF7EAFD50
:10C0A0002B78DBB29C42E3D0FFB20B4B1F55012231
:10C0B0000A4B1A70E4B2054B1C70BC22054BDA70B7
:10C0C000BDE8F081348004406CD8FF1F70D8FF1F9A
:10C0D00069D8FF1F00B0064000D8FF1FFCD7FF1F24
:10C0E0002DE9F84F0746284B1B6813F4006F49D021
:10C0F000264B1B680BB101221A7007EB010B5F4541
:10C100003DD2DFF89890224EDFF88C80DFF890A0C7
:10C1100099F800400134282C28BF00243578EDB26E
:10C12000A54220D1BC2388F80330FDF743FD402809
:10C1300011DC98F8043013F0800F10D033780133FD
:10C14000282B28BF00231AF80320D2B288F8072032
:10C15000DBB2337003E0FF2801DDFFF78BFD33789E
:10C16000DBB29D42E1D017F8013B0AF8043001220E
:10C17000084B1A70E4B289F800405F45C8D1BC2270
:10C18000054BDA70BDE8F88F348004406CD8FF1F8F
:10C1900069D8FF1FFCD7FF1F00B0064070D8FF1FF3
:10C1A00000D8FF1F10B5064B1B7813F0FF0F06D009
:10C1B000034CFFF75FFD237813F0FF0FF9D110BD9B
:10C1C000FCD7FF1F064B1B78DBB2064A1278D2B2AF
:10C1D00093422CBF273202F1FF32D01A704700BFC2
:10C1E00070D8FF1F69D8FF1F054B1878C0B2054BE8
:10C1F0001B78DBB2984238BF4030C01A704700BF8E
:10C2000068D8FF1FFDD7FF1F10B4184B1A78D2B2A1
:10C21000174B1B78DBB29A4218D001333F2B18D84A
:10C220001449C85CC0B2DCB211490C7012490968EB
:10C23000C9B19A4203D300E00023D31A01E040328F
:10C24000D31A1A2B0FDC00230B700CE04FF0FF30D9
:10C2500009E0084B1878C0B20021054B1970064B55
:10C2600019680029E8D15DF8044B704768D8FF1FB2
:10C27000FDD7FF1F28D8FF1FF8D7FF1F094B1A78DB
:10C28000D2B2094B1B78DBB29A4207D00133402B64
:10C2900028BF0023054AD05CC0B270474FF0FF3082
:10C2A000704700BF68D8FF1FFDD7FF1F28D8FF1FAA
:10C2B0000D4B1B6813F4006F14D00C4BDA7802F0AE
:10C2C000CB02DA7040225A74DA7842F03402DA7023
:10C2D000074B1A78D2B2074B1A70074B1B680BB189
:10C2E00000221A70704700BF3480044000B006403E
:10C2F000FDD7FF1F68D8FF1FF8D7FF1F70B43D4B55
:10C300001B7913F0300F33D072B63A4B9B7D03F09C
:10C31000FF022BB9374BDA7940225A7462B627E014
:10C3200062B6354B1978C9B2344B1C78E4B2314D42
:10C33000334EEB79D8B24B1C402B28BF0023A342CD
:10C340001CBFF0541946531E13F0FF02F1D1CAB2BC
:10C35000294B1A702B4B1B6853B1A1422EBFC4EB63
:10C360000101C4F1400409192729C4BF01221A7030
:10C37000204BDA78D2B212F0800F27D01B7913F05D
:10C38000800F23D0204B1C78E4B2204B1B78DBB20B
:10C390009C4210D017491E4D01E0A3420BD001333F
:10C3A000282B28BF00230879E85CC0B2C871087D3B
:10C3B000C0B20728F1D9DBB214490B700D4B1B79C1
:10C3C00013F0800F02D07C210A4BD97012F0400F7D
:10C3D0000ED0084B1B7913F0400F09D000220D4BF3
:10C3E0001A700D4B1B6803B11A703C22014BDA70B6
:10C3F00070BC704700B0064068D8FF1FFDD7FF1F14
:10C4000028D8FF1FF8D7FF1F70D8FF1F69D8FF1F5C
:10C4100000D8FF1FFCD7FF1F6CD8FF1F174B1A68EF
:10C4200042F480521A600023154A1370154A1370A3
:10C43000154A1370154A1370154A137040F21331E0
:10C44000144A11604FF4517104321160C0F3443149
:10C45000114A1170C0F34711517000F01F00907223
:10C46000937013742C23D37040220C4B1A704FF42A
:10C470000032A3F22D331A60704700BF34800440AD
:10C48000E4D8FF1F79D8FF1FECD8FF1FE5D8FF1FA6
:10C4900078D8FF1F08C0044000C0064031E400E027
:10C4A000164B9B7803F0EC0300F00302134310F0EB
:10C4B000040F18BF43F01003104A937000F00F03ED
:10C4C000042B04D11346927942F040029A710B4B2F
:10C4D0005A7902F0EF0210F0100F18BF42F010026C
:10C4E000064B5A719B7903F0EF0310F0200F18BF31
:10C4F00043F01003014A9371704700BF00C006402B
:10C5000010B5144B1B6813F4805F21D0124B1B78BD
:10C5100013F0FF0F06D0104CFFF7ACFB237813F09D
:10C52000FF0FF9D14FF400320C4B1A6000230C4A74
:10C53000D37040F203120B490A6004310A600A4AC0
:10C5400013700A4A13700A4B1B680BB101221A7050
:10C5500010BD00BF3480044078D8FF1F84E100E0A4
:10C5600000C0064008C00440E4D8FF1F79D8FF1F70
:10C5700074D8FF1F10B50446094A137813F0FF0F53
:10C58000FBD120460121FDF7F5FB20460021FDF7F8
:10C59000BFFB044B53F83420034B1A6010BD00BF9F
:10C5A00078D8FF1F14010100E8D8FF1F10B40C4613
:10C5B00009B140F08000104B1B78984219D00F4A07
:10C5C000126812F4805F12D003F07F03082B02D1AF
:10C5D00000220B4B1A60002C0CBF4422602200F09A
:10C5E0007F03082B03D142F44072054B1A60024BC3
:10C5F00018705DF8044B7047FEA2FF1F34800440A2
:10C600000CC00440704700BF10B50D4B1B6813F4FD
:10C61000805F12D021280CD80A4C0B4B53F83030D5
:10C6200023600121FDF7A6FB236800221A70012078
:10C6300010BD0020034B186010BD002010BD00BFCE
:10C640003480044074D8FF1F140101000D4B1B6897
:10C6500013F4805F13D00E280AD140F202320A4B45
:10C660001A600A4B5A7B42F001025A73012070474C
:10C67000064B5A7B02F0FE025A73002070470020DE
:10C68000704700BF3480044004C0044000C006402E
:10C690002DE9F04107461F4B1B6813F4805F37D02C
:10C6A0001D4B1B680BB101221A701C4B1C78013406
:10C6B000282C28BF00241A4D1A4EDFF86C8017E092
:10C6C000FDF778FA40280FDC337913F0800F0FD094
:10C6D0002B780133282B28BF002318F80320D2B26F
:10C6E000F271DBB22B7003E0FF2801DDFFF7C2FA25
:10C6F0002B78DBB29C42E3D0FFB20B4B1F550122DB
:10C700000A4B1A70E4B2054B1C70AC22054BDA7070
:10C71000BDE8F08134800440E8D8FF1FECD8FF1F4B
:10C72000E5D8FF1F00C006407CD8FF1F78D8FF1F48
:10C7300038B505460C4629B115F8010BFFF7A8FFDF
:10C74000013CF9D138BD00BF10B5064B1B7813F082
:10C75000FF0F06D0034CFFF78DFA237813F0FF0F7D
:10C76000F9D110BD78D8FF1F064B1B78DBB2064A03
:10C770001278D2B293422CBF273202F1FF32D01A84
:10C78000704700BFECD8FF1FE5D8FF1F054B187896
:10C79000C0B2054B1B78DBB2984238BF4030C01A9C
:10C7A000704700BFE4D8FF1F79D8FF1F10B4184BA3
:10C7B0001A78D2B2174B1B78DBB29A4218D00133E9
:10C7C0003F2B18D81449C85CC0B2DCB211490C70B8
:10C7D00012490968C9B19A4203D300E00023D31A71
:10C7E00001E04032D31A1A2B0FDC00230B700CE04F
:10C7F0004FF0FF3009E0084B1878C0B20021054B1C
:10C800001970064B19680029E8D15DF8044B704790
:10C81000E4D8FF1F79D8FF1FA4D8FF1F74D8FF1FCB
:10C82000094B1A78D2B2094B1B78DBB29A4207D077
:10C830000133402B28BF0023054AD05CC0B27047AB
:10C840004FF0FF30704700BFE4D8FF1F79D8FF1FBB
:10C85000A4D8FF1F054B1A78D2B2054B1A70054BAE
:10C860001B680BB100221A70704700BF79D8FF1FF8
:10C87000E4D8FF1F74D8FF1F2F4B1B7913F0200F34
:10C8800023D02D4BDB79D9B22C4B1B780133402BB5
:10C8900028BF00232A4A1278D2B29A4204D0294AE9
:10C8A000D154D9B2254A1170274A116869B1274A73
:10C8B0001278D2B293422EBFC2EB0303C2F1400200
:10C8C0009B18272BC4BF01230B701B4BDB78DBB2FB
:10C8D00013F0800F1CD0184A127912F0800F17D075
:10C8E0001B4A1178C9B2194A1278D2B2914203D1C7
:10C8F0006C21114AD1700BE00132282A28BF002296
:10C900001449885CC0B20C49C871D2B20F490A7090
:10C9100013F0400F0ED0084B1B7913F0400F09D0D5
:10C9200000220D4B1A700D4B1B6803B11A702C229C
:10C93000014BDA70704700BF00C00640E4D8FF1F0B
:10C9400079D8FF1FA4D8FF1F74D8FF1FE5D8FF1F99
:10C95000ECD8FF1F7CD8FF1F78D8FF1FE8D8FF1F37
:10C9600000B585B072B61B4B70221A7041211A4A6D
:10C9700011700F21013A117080221A701A46137833
:10C9800013F0800FFBD0154B186862B6144B984219
:10C990009CBF00EB8000400001A90A22FDF72AF9A4
:10C9A0009DF804307BB908E001A9595C31B1918050
:10C9B000023201330A2BF7D100E0002301335B0080
:10C9C000084A137003E0074A53800123ECE705B0DF
:10C9D0005DF804FB0000024007000240080002402E
:10C9E0007F9698008CA3FF1F08B503681B68C9B227
:10C9F000984708BD08B503681B68C9B2984708BDC9
:10CA000008B503681B68C9B2984708BD08B5036834
:10CA10001B68C9B2984708BD08B54B0803F13760D9
:10CA200000F5D830B0FBF1F0FDF7F8FA08BD00BF13
:10CA300010B514464B0803F1376000F5D830B0FB51
:10CA4000F1F0FDF7EBFA2046FDF750FB10BD00BFFB
:10CA500008B5FDF77BFB08BD08B50846FDF7B0FB40
:10CA600008BD00BF08B50846FDF704FC08BD00BFBF
:10CA700008B508461146FDF7BFFB08BD08B50846D6
:10CA8000FDF724FC003018BF012008BD08B508469A
:10CA9000FDF73EFC003018BF012008BD08B5FDF7CA
:10CAA00037FD08BD08B5FDF77DFD08BD08B5FDF7EC
:10CAB0003FFD08BD08B5FDF709FD08BD08B5FDF748
:10CAC0008BFD08BD08B5FDF711FD08BD08B508468A
:10CAD000FDF74AFC012008BD08B50846FDF744FCF7
:10CAE000012008BD10B5144608461146FDF78CFC20
:10CAF000204610BD38B50D46084602F0EFF8044652
:10CB000028462146FDF780FC204638BD704700BF0F
:10CB1000044B00221A714FF47A7199601A73024A19
:10CB20001A607047F0D8FF1FC002010008B5036803
:10CB30001B68C9B2984708BD08B503681B68C9B22D
:10CB4000984708BD08B503681B68C9B2984708BD77
:10CB500008B503681B68C9B2984708BD08B54B08FB
:10CB600003F1376000F5D830B0FBF1F0FFF7A4F81F
:10CB700008BD00BF10B514464B0803F1376000F53F
:10CB8000D830B0FBF1F0FFF797F82046FFF7FCF83C
:10CB900010BD00BF08B5FFF727F908BD08B5084666
:10CBA000FFF782F908BD00BF08B50846FFF7D6F9C0
:10CBB00008BD00BF08B508461146FFF791F908BD4A
:10CBC00008B50846FFF7F8F9003018BF012008BD86
:10CBD00008B50846FFF712FA003018BF012008BD5B
:10CBE00008B5FFF701FB08BD08B5FFF747FB08BD17
:10CBF00008B5FFF709FB08BD08B5FFF7D3FA08BD74
:10CC000008B5FFF755FB08BD08B5FFF7DBFA08BD0F
:10CC100008B50846FFF714FA012008BD08B5084614
:10CC2000FFF70EFA012008BD10B51446084611465C
:10CC3000FFF756FA204610BD38B50D46084602F0FB
:10CC40004DF8044628462146FFF74AFA204638BDEB
:10CC5000704700BF044B00221A714FF47A7199603B
:10CC60001A73024A1A60704700D9FF1F200301009F
:10CC700008B503681B68C9B2984708BD08B50368C2
:10CC80001B68C9B2984708BD08B503681B68C9B2DC
:10CC9000984708BD08B503681B68C9B2984708BD26
:10CCA00008B54B0803F1B76000F55840B0FBF1F050
:10CCB000FFF7B4FB08BD00BF10B514464B0803F1E5
:10CCC000B76000F55840B0FBF1F0FFF7A7FB204636
:10CCD000FFF7E6FB10BD00BF08B5FFF711FC08BD6C
:10CCE00008B50846FFF746FC08BD00BF08B5084672
:10CCF000FFF788FC08BD00BF08B508461146FFF7DE
:10CD000055FC08BD08B50846FFF77EFC003018BF8B
:10CD1000012008BD08B50846FFF798FC003018BF91
:10CD2000012008BD08B5FFF731FD08BD08B5FFF7C4
:10CD300077FD08BD08B5FFF739FD08BD08B5FFF759
:10CD400003FD08BD08B5FFF785FD08BD08B5FFF771
:10CD50000BFD08BD08B50846FFF79AFC012008BD89
:10CD600008B50846FFF794FC012008BD10B514462D
:10CD700008461146FFF7DCFC204610BD38B50D46CD
:10CD8000084601F0ABFF044628462146FFF7D0FCD9
:10CD9000204638BD704700BF044B00221A714FF483
:10CDA0007A7199601A73024A1A60704710D9FF1F8E
:10CDB0008003010031F0004310B408D00F4AA3F5FE
:10CDC000801494420AD804205DF8044B7047002870
:10CDD0000CBF022003205DF8044B7047B3F5801FA1
:10CDE00001D20320F7E7064A934201D00020F2E780
:10CDF000D0F1010038BF0020EDE700BFFFFFDF7F6B
:10CE00000000F07F81F0004102E000BF83F00043AA
:10CE100030B54FEA41044FEA430594EA050F08BFD5
:10CE200090EA020F1FBF54EA000C55EA020C7FEA99
:10CE3000645C7FEA655C00F0E2804FEA5454D4EB16
:10CE40005555B8BF6D420CDD2C4480EA020281EAE0
:10CE5000030382EA000083EA010180EA020281EA18
:10CE60000303362D88BF30BD11F0004F4FEA01316A
:10CE70004FF4801C4CEA113102D0404261EB410179
:10CE800013F0004F4FEA03334CEA133302D05242FF
:10CE900063EB430394EA050F00F0A780A4F10104BB
:10CEA000D5F1200E0DDB02FA0EFC22FA05F28018F5
:10CEB00041F1000103FA0EF2801843FA05F35941DB
:10CEC0000EE0A5F120050EF1200E012A03FA0EFC5A
:10CED00028BF4CF0020C43FA05F3C01851EBE37184
:10CEE00001F0004507D54FF0000EDCF1000C7EEBA1
:10CEF00000006EEB0101B1F5801F1BD3B1F5001FDF
:10CF00000CD349085FEA30004FEA3C0C04F10104FD
:10CF10004FEA445212F5800F80F09A80BCF1004F26
:10CF200008BF5FEA500C50F1000041EB045141EAA8
:10CF3000050130BD5FEA4C0C404141EB010111F4A9
:10CF4000801FA4F10104E9D191F0000F04BF014654
:10CF50000020B1FA81F308BF2033A3F10B03B3F132
:10CF600020020CDA0C3208DD02F1140CC2F10C02C2
:10CF700001FA0CF021FA02F10CE002F11402D8BF20
:10CF8000C2F1200C01FA02F120FA0CFCDCBF41EAEC
:10CF90000C019040E41AA2BF01EB0451294330BDBB
:10CFA0006FEA04041F3C1CDA0C340EDC04F1140498
:10CFB000C4F1200220FA04F001FA02F340EA03006F
:10CFC00021FA04F345EA030130BDC4F10C04C4F1B5
:10CFD000200220FA02F001FA04F340EA0300294695
:10CFE00030BD21FA04F0294630BD94F0000F83F4DF
:10CFF000801306BF81F480110134013D4EE77FEAC2
:10D00000645C18BF7FEA655C29D094EA050F08BF0D
:10D0100090EA020F05D054EA000C04BF19461046EE
:10D0200030BD91EA030F1EBF0021002030BD5FEA32
:10D03000545C05D14000494128BF41F0004130BD5A
:10D0400014F580043CBF01F5801130BD01F00045AE
:10D0500045F0FE4141F470014FF0000030BD7FEA21
:10D06000645C1ABF194610467FEA655C1CBF0B461C
:10D07000024650EA013406BF52EA033591EA030F33
:10D0800041F4002130BD00BF90F0000F04BF00212B
:10D09000704730B54FF4806404F132044FF000055E
:10D0A0004FF0000150E700BF90F0000F04BF0021D7
:10D0B000704730B54FF4806404F1320410F000453D
:10D0C00048BF40424FF000013EE700BF42004FEA38
:10D0D000E2014FEA31014FEA02701FBF12F07F43B5
:10D0E00093F07F4F81F06051704792F0000F14BFB2
:10D0F00093F07F4F704730B54FF4607401F00045F6
:10D1000021F0004120E700BF50EA010208BF70474C
:10D1100030B54FF000050AE050EA010208BF704741
:10D1200030B511F0004502D5404261EB41014FF4AA
:10D13000806404F132045FEA915C3FF4DCAE4FF0AE
:10D1400003025FEADC0C18BF03325FEADC0C18BF95
:10D15000033202EBDC02C2F1200300FA03FC20FAE6
:10D1600002F001FA03FE40EA0E0021FA02F1144433
:10D17000C1E600BF70B54FF0FF0C4CF4E06C1CEA48
:10D1800011541DBF1CEA135594EA0C0F95EA0C0FBD
:10D1900000F0DEF82C4481EA030621EA4C5123EA30
:10D1A0004C5350EA013518BF52EA033541F480115F
:10D1B00043F4801338D0A0FB02CE4FF00005E1FB12
:10D1C00002E506F00042E0FB03E54FF00006E1FB5C
:10D1D00003569CF0000F18BF4EF0010EA4F1FF049F
:10D1E000B6F5007F64F5407404D25FEA4E0E6D41DF
:10D1F00046EB060642EAC62141EA55514FEAC520F0
:10D2000040EA5E504FEACE2EB4F1FD0C88BFBCF56B
:10D21000E06F1ED8BEF1004F08BF5FEA500E50F11C
:10D22000000041EB045170BD06F0004646EA0101E2
:10D2300040EA020081EA0301B4EB5C04C2BFD4EB14
:10D240000C0541EA045170BD41F480114FF0000E0D
:10D25000013C00F3AB8014F1360FDEBF002001F07B
:10D26000004170BDC4F10004203C35DA0C341BDCF5
:10D2700004F11404C4F1200500FA05F320FA04F0C7
:10D2800001FA05F240EA020001F0004221F00041FB
:10D2900010EBD37021FA04F642EB06015EEA430E6E
:10D2A00008BF20EAD37070BDC4F10C04C4F120059E
:10D2B00000FA04F320FA05F001FA04F240EA020051
:10D2C00001F0004110EBD37041F100015EEA430E22
:10D2D00008BF20EAD37070BDC4F1200500FA05F242
:10D2E0004EEA020E20FA04F301FA05F243EA0203C1
:10D2F00021FA04F001F0004121FA04F220EA0200D0
:10D3000000EBD3705EEA430E08BF20EAD37070BD15
:10D3100094F0000F0FD101F00046400041EB0101F5
:10D3200011F4801F08BF013CF7D041EA060195F0D7
:10D33000000F18BF704703F00046520043EB030391
:10D3400013F4801F08BF013DF7D043EA060370477E
:10D3500094EA0C0F0CEA135518BF95EA0C0F0CD089
:10D3600050EA410618BF52EA4306D1D181EA0301CF
:10D3700001F000414FF0000070BD50EA410606BFC9
:10D380001046194652EA430619D094EA0C0F02D10E
:10D3900050EA013613D195EA0C0F05D152EA033653
:10D3A0001CBF104619460AD181EA030101F0004171
:10D3B00041F0FE4141F470014FF0000070BD41F0BA
:10D3C000FE4141F4780170BD70B54FF0FF0C4CF494
:10D3D000E06C1CEA11541DBF1CEA135594EA0C0FB3
:10D3E00095EA0C0F00F0A7F8A4EB050481EA030E00
:10D3F00052EA03354FEA013100F088804FEA0333E7
:10D400004FF0805545EA131343EA12634FEA0222B4
:10D4100045EA111545EA10654FEA00260EF0004175
:10D420009D4208BF964244F1FD0404F5407402D2C7
:10D430005B084FEA3202B61A65EB03055B084FEA58
:10D4400032024FF480104FF4002CB6EB020E75EB55
:10D45000030E22BFB61A754640EA0C005B084FEA7D
:10D460003202B6EB020E75EB030E22BFB61A7546FA
:10D4700040EA5C005B084FEA3202B6EB020E75EB45
:10D48000030E22BFB61A754640EA9C005B084FEABD
:10D490003202B6EB020E75EB030E22BFB61A7546CA
:10D4A00040EADC0055EA060E18D04FEA051545EAB9
:10D4B00016754FEA06164FEAC30343EA52734FEA62
:10D4C000C2025FEA1C1CC0D111F4801F0BD141EADB
:10D4D00000014FF000004FF0004CB6E711F4801F40
:10D4E00004BF01430020B4F1FD0C88BFBCF5E06F20
:10D4F0003FF6AFAEB5EB030C04BFB6EB020C5FEA30
:10D50000500C50F1000041EB045170BD0EF0004E84
:10D510004EEA113114EB5C04C2BFD4EB0C0541EAB6
:10D52000045170BD41F480114FF0000E013C90E6B3
:10D5300045EA060E8DE60CEA135594EA0C0F08BF77
:10D5400095EA0C0F3FF43BAF94EA0C0F0AD150EA76
:10D5500001347FF434AF95EA0C0F7FF425AF104609
:10D5600019462CE795EA0C0F06D152EA03353FF431
:10D57000FDAE1046194622E750EA410618BF52EAAE
:10D5800043067FF4C5AE50EA41047FF40DAF52EA82
:10D5900043057FF4EBAE12E74FF0FF3C06E000BF1F
:10D5A0004FF0010C02E000BF4FF0010C4DF804CD2C
:10D5B0004FEA410C7FEA6C5C4FEA430C18BF7FEAEC
:10D5C0006C5C1BD001B050EA410C0CBF52EA430C1A
:10D5D00091EA030F02BF90EA020F0020704710F19A
:10D5E000000F91EA030F58BF994208BF90422CBF29
:10D5F000D8176FEAE37040F0010070474FEA410C22
:10D600007FEA6C5C02D150EA013C07D14FEA430C3F
:10D610007FEA6C5CD6D152EA033CD3D05DF8040BB0
:10D62000704700BF8446104662468C4619466346E2
:10D6300000E000BF01B5FFF7B7FF002848BF10F1B9
:10D64000000F01BD4DF808EDFFF7F4FF0CBF0120FE
:10D6500000205DF808FB00BF4DF808EDFFF7EAFF7A
:10D6600034BF012000205DF808FB00BF4DF808ED35
:10D67000FFF7E0FF94BF012000205DF808FB00BF2A
:10D680004DF808EDFFF7CEFF94BF012000205DF8B4
:10D6900008FB00BF4DF808EDFFF7C4FF34BF0120C1
:10D6A00000205DF808FB00BF4A0011D212F50012FD
:10D6B00011D20DD56FF47873B3EB62520ED44FEAEA
:10D6C000C12343F0004343EA505323FA02F070476A
:10D6D0004FF00000704750EA013002D14FF0FF30A8
:10D6E00070474FF00000704780F0004002E000BF3C
:10D6F00081F0004142001FBF5FEA410392EA030F3D
:10D700007FEA226C7FEA236C6AD04FEA1262D2EB86
:10D710001363C1BFD218414048404140B8BF5B428B
:10D72000192B88BF704710F0004F40F4000020F024
:10D730007F4018BF404211F0004F41F4000121F03A
:10D740007F4118BF494292EA030F3FD0A2F1010284
:10D7500041FA03FC10EB0C00C3F1200301FA03F1C2
:10D7600000F0004302D5494260EB4000B0F5000FE5
:10D7700013D3B0F1807F06D340084FEA310102F1A4
:10D780000102FE2A51D2B1F1004F40EBC25008BF56
:10D7900020F0010040EA03007047490040EB000020
:10D7A00010F4000FA2F10102EDD1B0FA80FCACF14F
:10D7B000080CB2EB0C0200FA0CF0AABF00EBC2504E
:10D7C00052421843BCBFD0401843704792F0000F3C
:10D7D00081F4000106BF80F400000132013BB5E78F
:10D7E0004FEA41037FEA226C18BF7FEA236C21D005
:10D7F00092EA030F04D092F0000F08BF084670476A
:10D8000090EA010F1CBF0020704712F07F4F04D137
:10D81000400028BF40F00040704712F100723CBF4A
:10D8200000F50000704700F0004343F0FE4040F474
:10D83000000070477FEA226216BF08467FEA236332
:10D840000146420206BF5FEA412390EA010F40F41D
:10D85000800070474FF0000304E000BF10F0004369
:10D8600048BF40425FEA000C08BF704743F0964350
:10D8700001464FF000001CE050EA010208BF70476B
:10D880004FF000030AE000BF50EA010208BF7047F2
:10D8900011F0004302D5404261EB41015FEA010C07
:10D8A00002BF84460146002043F0B64308BFA3F1FF
:10D8B0008053A3F50003BCFA8CF2083AA3EBC253E1
:10D8C00010DB01FA02FC634400FA02FCC2F1200200
:10D8D000BCF1004F20FA02F243EB020008BF20F037
:10D8E0000100704702F1200201FA02FCC2F120029D
:10D8F00050EA4C0021FA02F243EB020008BF20EA92
:10D90000DC7070474FF0FF0C1CEAD0521EBF1CEABF
:10D91000D15392EA0C0F93EA0C0F6FD01A4480EAAD
:10D92000010C400218BF5FEA41211ED04FF0006396
:10D9300043EA501043EA5111A0FB01310CF00040C2
:10D94000B1F5000F3EBF490041EAD3715B0040EAE8
:10D95000010062F17F02FD2A1DD8B3F1004F40EBB8
:10D96000C25008BF20F00100704790F0000F0CF08B
:10D97000004C08BF49024CEA502040EA51207F3A4F
:10D98000C2BFD2F1FF0340EAC250704740F400002A
:10D990004FF00003013A5DDC12F1190FDCBF00F01B
:10D9A00000407047C2F10002410021FA02F1C2F1C9
:10D9B000200200FA02FC5FEA310040F1000053EA65
:10D9C0004C0308BF20EADC70704792F0000F00F0B3
:10D9D000004C02BF400010F4000F013AF9D040EAB9
:10D9E0000C0093F0000F01F0004C02BF490011F44D
:10D9F000000F013BF9D041EA0C018FE70CEAD1534B
:10DA000092EA0C0F18BF93EA0C0F0AD030F0004CCA
:10DA100018BF31F0004CD8D180EA010000F000407E
:10DA2000704790F0000F17BF90F0004F084691F03C
:10DA3000000F91F0004F14D092EA0C0F01D1420276
:10DA40000FD193EA0C0F03D14B0218BF084608D13F
:10DA500080EA010000F0004040F0FE4040F4000089
:10DA6000704740F0FE4040F4400070474FF0FF0C1C
:10DA70001CEAD0521EBF1CEAD15392EA0C0F93EA63
:10DA80000C0F69D0A2EB030280EA010C49024FEAB5
:10DA9000402037D04FF0805343EA111143EA10136E
:10DAA0000CF000408B4238BF5B0042F17D024FF426
:10DAB000000C8B4224BF5B1A40EA0C00B3EB510F01
:10DAC00024BFA3EB510340EA5C00B3EB910F24BFEA
:10DAD000A3EB910340EA9C00B3EBD10F24BFA3EB6F
:10DAE000D10340EADC001B0118BF5FEA1C1CE0D137
:10DAF000FD2A3FF650AF8B4240EBC25008BF20F0EA
:10DB0000010070470CF0004C4CEA50207F32C2BF3D
:10DB1000D2F1FF0340EAC250704740F400004FF0DA
:10DB20000003013A37E792F0000F00F0004C02BF0B
:10DB3000400010F4000F013AF9D040EA0C0093F0D5
:10DB4000000F01F0004C02BF490011F4000F013B2F
:10DB5000F9D041EA0C0195E70CEAD15392EA0C0F97
:10DB600008D142027FF47DAF93EA0C0F7FF470AFCF
:10DB7000084676E793EA0C0F04D14B023FF44CAF12
:10DB800008466EE730F0004C18BF31F0004CCAD1A7
:10DB900030F000427FF45CAF31F000437FF43CAFE3
:10DBA0005FE700BF4FF0FF3C06E000BF4FF0010C05
:10DBB00002E000BF4FF0010C4DF804CD4FEA4002E7
:10DBC0004FEA41037FEA226C18BF7FEA236C11D031
:10DBD00001B052EA530C18BF90EA010F58BFB2EBE4
:10DBE000030088BFC81738BF6FEAE17018BF40F064
:10DBF000010070477FEA226C02D15FEA402C05D118
:10DC00007FEA236CE4D15FEA412CE1D05DF8040B9C
:10DC1000704700BF844608466146FFE70FB5FFF72F
:10DC2000C9FF002848BF10F1000F0FBD4DF808EDE7
:10DC3000FFF7F4FF0CBF012000205DF808FB00BFD8
:10DC40004DF808EDFFF7EAFF34BF012000205DF832
:10DC500008FB00BF4DF808EDFFF7E0FF94BF01207F
:10DC600000205DF808FB00BF4DF808EDFFF7D2FF7C
:10DC700094BF012000205DF808FB00BF4DF808EDBF
:10DC8000FFF7C8FF34BF012000205DF808FB00BF8C
:10DC90004FEA4002B2F1FE4F0FD34FF09E03B3EBB9
:10DCA00012620DD94FEA002343F0004310F0004FF9
:10DCB00023FA02F018BF404270474FF0000070474F
:10DCC00012F1610F01D1420205D110F0004008BFEE
:10DCD0006FF0004070474FF00000704742000ED2D6
:10DCE000B2F1FE4F0BD34FF09E03B3EB126209D497
:10DCF0004FEA002343F0004323FA02F070474FF04D
:10DD00000000704712F1610F01D1420202D14FF0C1
:10DD1000FF3070474FF00000704700BF03460846D1
:10DD2000194600F009B800BF00210A2201F0C2B86C
:10DD300000210A2201F0BEB810B40C461346014679
:10DD4000224602205DF8044B01F05CB970B50F4E1D
:10DD50000F4D761BB61007D0043D0024013455F852
:10DD6000043F9847A642F9D10A4E0B4D761B02F0AC
:10DD7000B7FBB61008D0043D0024013455F8043F29
:10DD80009847A642F9D170BD70BD00BFEC040100F8
:10DD9000EC0401003C050100EC040100034B1B688E
:10DDA0001844407800F00800704700BFE4ABFF1F44
:10DDB000024B0146186800F00BB800BFD0A7FF1F48
:10DDC000024B0146186801F0E7B900BFD0A7FF1F5A
:10DDD0002DE9F04F01F10B05162D83B0064627D92A
:10DDE00035F0070527D4A94225D8304600F06AFB54
:10DDF000B5F5FC7F26D2C14F4FEAD50C07EBCC031B
:10DE0000DC689C4200F0D2816368E268A16823F07C
:10DE10000303234430465D68CA6045F00105916004
:10DE20005D6000F051FB0834204603B0BDE8F08F80
:10DE30001025A942D9D900240C232046336003B011
:10DE4000BDE8F08F5FEA552C00F08A80BCF1040F2A
:10DE500000F260814FEA951C0CF1380C4FEA4C013E
:10DE6000A64F07EB8101CC68A14205D10CE0002B45
:10DE70007ADAE468A14207D0626822F00302531BF9
:10DE80000F2BF4DD0CF1FF3C0CF1010C9B4B3C69BA
:10DE900003F1080E744500F07E81616821F00301F2
:10DEA0004A1B0F2A00F36481002AC3F814E0C3F868
:10DEB00010E06ADAB1F5007F80F03A81C90803EB1F
:10DEC000C1004FEAA1085A688168A1604FF00109BA
:10DED00009FA08F848EA0202E0605A608460CC60FF
:10DEE0004FEAAC030120984090425BD8024206D131
:10DEF0002CF0030C400002420CF1040CFAD007EBAA
:10DF0000CC084446E146E3689C4207D145E1002A3B
:10DF100080F25681DB689C4200F03F81596821F015
:10DF200003014A1B0F2AF2DD1C46D3F80CC054F83B
:10DF3000088F591945F0010942F00105C3F8049012
:10DF40003046C8F80CC0CCF8088079613961C1F856
:10DF50000CE0C1F808E04D608A5000F0B5FA63E7C4
:10DF60007E214FF03F0C7BE72244E3685068A168B4
:10DF700040F00105CB6030469960556000F0A4FA8E
:10DF80000834204603B0BDE8F08F214430464B688A
:10DF900043F001034B6000F097FA0834204603B0C9
:10DFA000BDE8F08FBC68636823F00309A94504D37A
:10DFB000C5EB09030F2B00F39180514B514A1968AF
:10DFC0001368013305EB010A04EB090B00F06181D2
:10DFD0000AF5805A0AF10F0A2AF47F6A2AF00F0A1A
:10DFE00030465146019200F05FFCB0F1FF3F8046A1
:10DFF000019A00F00081834500F2FA80DFF810C139
:10E00000DCF80030C3455344CCF8003000F04A81BE
:10E0100012683C4901321BBFCBEB080B5B44C1F8D3
:10E020000080CCF8003018F0070300F01381C3F132
:10E030000802C3F5805390440833C244CAF30B0A64
:10E04000CAEB030A51463046CDF804C000F02CFC60
:10E05000431CDDF804C000F03581C8EB00025244D7
:10E0600042F00102DCF80030C7F808805344BC429B
:10E07000C8F80420CCF80030DFF894A015D0B9F12E
:10E080000F0F40F2EA806168A9F10C0222F007024A
:10E0900001F0010EA118052042EA0E0E0F2AC4F865
:10E0A00004E04860886000F21181174ABC6811687A
:10E0B0008B4288BF1360154A11688B4288BF13607A
:10E0C000626822F003029542C5EB020301D80F2BD0
:10E0D00004DC304600F0F8F90024A5E6621943F0AC
:10E0E000010345F0010565603046BA60536000F0F9
:10E0F000EBF90834204603B0BDE8F08FD4A7FF1F2A
:10E1000028D9FF1FE0ABFF1F24D9FF1F20D9FF1F15
:10E110002CD9FF1FBCF1140F61D9BCF1540F00F2D0
:10E120008F804FEA153C0CF16E0C4FEA4C0197E6DC
:10E130004B0A042B58D9142B00F2AE8003F15B027A
:10E14000500007EB8000DFF8BC818368834200F059
:10E150008A805A6822F00302914202D29B68984258
:10E16000F7D1D9687A68E160A3608C60DC60B7E6BB
:10E17000611942F0010745F00105656030465961BB
:10E180001961C1F80CE0C1F808E04F608A5008340A
:10E1900000F09AF948E65A68A2E609F1010919F077
:10E1A000030F04F108047FF4AEAE2DE004F1080380
:10E1B0006469A34208BF0CF1020C3FF467AE23E68A
:10E1C00019441C464868DB6854F8082F40F00105E4
:10E1D0004D603046D3609A6000F076F924E60CF189
:10E1E0005B0C4FEA4C013BE68A0938325000A8E745
:10E1F000BC423FF403AFBC68626822F0030262E7EE
:10E20000D8F8008098457BD11CF0030FA8F10803D3
:10E210000CF1FF3CF4D17B6823EA00037B604000F3
:10E2200098423FF6BFAE00283FF4BCAE0342CC4656
:10E230007FF465AE400003420CF1040CFAD05EE6B8
:10E24000BCF5AA7F1AD84FEAD53C0CF1770C4FEAFF
:10E250004C0105E64FF48053EFE60123C8F8043083
:10E26000444600222FE791100120D8F8042000FA3C
:10E2700001F10A43C8F80420194674E740F25453E8
:10E280009C451BD84FEA954C0CF17C0C4FEA4C0195
:10E29000E6E50AF1100AA3E6542B1FD80A0B6E32EA
:10E2A00050004EE7CBF30B0100297FF4B1AE0AEB2F
:10E2B0000901BA6841F001015160F6E6FC214FF016
:10E2C0007E0CCDE501224FF0000ACBE604F10801F7
:10E2D000304600F061FFDAF80030E6E6B3F5AA7FD9
:10E2E00003D8CA0B773250002BE740F254529342C6
:10E2F00003D88A0C7C32500023E7FC207E2220E7E2
:10E300007B688CE7D4A7FF1F032A70B428D940EAA2
:10E3100001039B0713D005780C78A54224D1013A5C
:10E32000002305E010F8015F11F8014FA5421BD151
:10E33000934203F10103F5D1002070BC70470C46F5
:10E34000034625681E68AE422146184604F10404BF
:10E3500003F1040304D1043A032A18462146F0D8F5
:10E36000002AD8D11046E8E7281B70BC704700BFD0
:10E370008842F0B410D98C18A0420DD28518531ED3
:10E3800042B121462A4611F8014D02F8014D013BE8
:10E390005C1CF8D1F0BC70470F2A3FD940EA01035A
:10E3A0009B073FD1A2F110073F0900EB071610367B
:10E3B0000C46034625681D6065685D60A5689D6024
:10E3C000E568DD601033B34204F11004F2D17B1C28
:10E3D00002F00F0C1B01BCF1030F1944034423D9B5
:10E3E0000E461D466446043C56F8047B45F8047B03
:10E3F000032CF8D8ACF1040424F00304043402F034
:10E40000030223442144002AC4D01A4411F8014BCA
:10E4100003F8014B9342F9D1F0BC70470346002A40
:10E42000F3D1B7E70346F0E76246002AEDD1B1E742
:10E43000F0B4840743D0541E002A3ED0CDB2034628
:10E4400003E0621E002C38D0144603F8015B9A07E3
:10E45000F7D1032C2AD9CDB245EA05250F2C45EA80
:10E46000054515D9A4F110073F0903F1100606EB85
:10E4700007161A46156055609560D5601032B24295
:10E48000F8D104F00F040137032C03EB07130DD967
:10E490001E462246043A032A46F8045BFAD8221F95
:10E4A00022F003020432134404F003042CB1C9B275
:10E4B0001C4403F8011BA342FBD1F0BC7047144677
:10E4C0000346C6E7704700BF704700BF024B0A46CD
:10E4D0000146186800F002B8D0A7FF1F2DE9F04FE1
:10E4E0000C4683B090468146002900F0E280FFF799
:10E4F000E9FF08F10B0654F8043C162E23F003053F
:10E50000A4F108074BD810210E46B0454CD88D42D7
:10E5100078DADFF890B3DBF808E07819864500F088
:10E52000CE80426822F0010C8444DCF804C01CF068
:10E53000010F7AD000221046DB0700F1928054F8D8
:10E54000083CC3EB070ADAF8043023F003032B443A
:10E5500088B3704500F0ED8002EB030E8E452ADB98
:10E56000C36882685746D3609A6057F8081FDAF884
:10E570000C30CB602A1F242A996000F22681132ACE
:10E5800040F2B3802368CAF808306368CAF80C30D8
:10E590001B2A00F2308108340AF11003A6E026F0AD
:10E5A0000706002E3146B0DA0C230020C9F80030EF
:10E5B00003B0BDE8F08F8B4253DB5746DAF80C10FE
:10E5C00057F8080F2A1F242AC160886000F20981C9
:10E5D000132A40F204812168CAF808106168CAF859
:10E5E0000C101B2A00F21C8108340AF11002216869
:10E5F000116061685160A16891601D46DAF80430CD
:10E600003C465746AA1B0F2A03F0010319D82B4397
:10E610003D447B606B6843F001036B604846FFF745
:10E6200053FF204603B0BDE8F08F22F0030202EB57
:10E63000050C8C4580DBC26881686546CA609160C4
:10E64000E0E7B91942F001001E430A447E604860C9
:10E65000536843F0010308315360484600F09CFDC5
:10E66000DCE741464846FFF7B3FB8046D0B154F89B
:10E67000043C23F001023A44A0F10801914200F069
:10E680009E802A1F242A50D8132A23D803462246C4
:10E69000116819605168596092689A60214648462D
:10E6A00000F07AFD4846FFF70FFF404603B0BDE893
:10E6B000F08F114603B0BDE8F04FFFF789BBDEF8DD
:10E6C000042022F00302501906F1100C604519DAFB
:10E6D000704631E723680360636843601B2A63D890
:10E6E00000F1080304F10802D2E73B4622681A60F1
:10E6F00062685A60A2689A603C467546DAF804304F
:10E7000057467FE73744831B43F00103CBF808707B
:10E710007B6054F8043C03F001031E43484644F870
:10E72000046CFFF7D1FE20467CE72146FFF720FE70
:10E73000B4E702EB030C06F110029445FFF63BAF81
:10E740005746DAF80C3057F8081F2A1F242ACB60E6
:10E75000996000F28780132A78D92368CAF80830B4
:10E760006368CAF80C301B2A00F2858008340AF16D
:10E77000100322681A6062685A60A2689A600AEB05
:10E780000603C6EB0C0242F00102CBF808305A60D7
:10E79000DAF8043003F001031E434846CAF8046067
:10E7A000FFF792FE38463DE7A3688360E368C360E5
:10E7B000242A2CD000F1100304F1100268E750F86D
:10E7C000042C22F0030215441CE721463846754606
:10E7D0003C46FFF7CDFD5746DAF8043012E73A46DB
:10E7E00005E7214638461D463C46FFF7C1FD574622
:10E7F000DAF8043006E7A368CAF81030E368CAF80C
:10E800001430242A18D010340AF118036EE7236953
:10E8100003616369436104F1180200F1180337E7EB
:10E82000A168CAF81010E168CAF81410242A0FD0A1
:10E8300010340AF11802DAE62369CAF8183063695D
:10E84000CAF81C3018340AF120034FE73B4690E722
:10E850002269CAF818206269CAF81C2018340AF123
:10E860002002C4E621463846CDF804C0FFF780FDFB
:10E87000DDF804C083E7A368CAF81030E368CAF87B
:10E880001430242A03D010340AF1180371E72369E5
:10E89000CAF818306369CAF81C3018340AF120032A
:10E8A00067E700BFD4A7FF1F38B5074C0023054614
:10E8B00008462360FBF774F9431C00D038BD236879
:10E8C000002BFBD02B6038BD68D9FF1F0F4B30B435
:10E8D0001C68054602E0D01A16D1ABB115F8013B11
:10E8E000E0181A46407800F00300012808BF03F141
:10E8F000200211F8013BE018407800F003000128E5
:10E90000E9D12033D01AE9D030BC7047E4ABFF1F07
:10E91000C9B2F0B4002947D085070FD00278002A89
:10E920003FD091423ED0431C05E013F8012B002A52
:10E9300037D0914236D09A071846F6D1036841EA9B
:10E94000012747EA074783EA0702A2F10135A3F14D
:10E95000013425EA020224EA0303134313F0803F43
:10E9600011D1021D104652F8043B83EA0704A4F1BA
:10E970000136A3F1013526EA040425EA0303234303
:10E9800013F0803FEED00378002B39D0994209D0A4
:10E99000431C01E0914205D0184613F8012B002AD0
:10E9A000F8D11046F0BC704784070BD00378002BD9
:10E9B000F8D0431C03E002780133002AF2D0990713
:10E9C0001846F8D10368A3F1013222EA030313F0D9
:10E9D000803F0AD1031D184653F8042BA2F10131E0
:10E9E00021EA020212F0803FF5D00378002BD9D043
:10E9F000431C184601330278002AFAD1F0BC704754
:10EA00001846CFE740EA010C1CF0070F23D1BDF1F7
:10EA1000100DCDE90245CDE900676FF000064FF01B
:10EA2000000700BFF0E80223F1E80245A24282FAA3
:10EA300046FCA7FA86FC08BFBCF1000F40F0D78067
:10EA4000AB4283FA46FCA7FA86FC08BFBCF1000F74
:10EA500040F0CA80E6E710F0030C21D020F003005C
:10EA600050F8042B5FEACC7C08D00FD211F801CB10
:10EA70005FFA92F3B3EB0C0C10D17BB111F801CB20
:10EA80005FFAA2F3B3EB0C0C08D13BB111F801CB48
:10EA90005FFAB2F3B3EB0C0C00D10BB960467047D0
:10EAA000BDF1100DCDE90245CDE900676FF000061C
:10EAB0004FF0000711F0030C2DD110F0040F0DD012
:10EAC00050F8042B51F8044BA24282FA46FCA7FAF4
:10EAD00086FC08BFBCF1000F40F0898011F0040FE4
:10EAE0009FD051F8045B00BFF0E80223AA4282FAEB
:10EAF00046FCA7FA86FC08BFBCF1000F71D1F1E813
:10EB00000245A34283FA46FCA7FA86FC08BFBCF183
:10EB1000000F63D1E8E721F00301BCF1020F1ED022
:10EB20003BDA51F8045B00BF50F8043B4FEA15256F
:10EB300083FA46FCA7FA86FCB7EB0C2F03EA1622F1
:10EB400008BFAA424DD151F8045BBCF1000F82EA24
:10EB500003034FEA056208BF93423CD1E4E751F852
:10EB6000045B00BF50F8043B4FEA154583FA46FCAE
:10EB7000A7FA86FCB7EB0C4F03EA164208BFAA427D
:10EB80002FD151F8045BBCF1000F82EA03034FEA76
:10EB9000054208BF93421ED1E4E751F8045B00BF71
:10EBA00050F8043B4FEA156583FA46FCA7FA86FC49
:10EBB000B7EB0C6F03EA166208BFAA4211D151F8F5
:10EBC000045BBCF1000F82EA03034FEA052208BF91
:10EBD000934200D1E4E719BA12BA0AE019BA22BA8C
:10EBE00007E011BA2ABA04E019BA2ABA01E011BA48
:10EBF00022BA9CFA8CF0DDE90067DDE902451DF1DF
:10EC0000100D38B1B0FA80F0C0F1180021FA00F10F
:10EC100022FA00F20120914298BF8041704700BF64
:10EC200080EA0102844612F0030F4FD111F0030F66
:10EC300032D14DF8044D11F0040F51F8043B0BD0C4
:10EC4000A3F101329A4312F0803F04BF4CF8043B19
:10EC500051F8043B16D100BF51F8044BA3F1013227
:10EC60009A4312F0803FA4F101320BD14CF8043BDF
:10EC7000A24312F0803F04BF51F8043B4CF8044B10
:10EC8000EAD023460CF8013B13F0FF0F4FEA332381
:10EC9000F8D15DF8044B704711F0010F06D011F860
:10ECA000012B0CF8012B002A08BF704711F0020F4E
:10ECB000BFD031F8022B12F0FF0F16BF2CF8022B39
:10ECC0008CF8002012F47F4FB3D1704711F8012B5C
:10ECD0000CF8012B002AF9D1704700BF20F0030186
:10ECE00010F00300C0F1000051F8043B00F1040CE7
:10ECF0004FEACC0C6FF000021CBF22FA0CF2134357
:10ED00004FF0010C4CEA0C2C4CEA0C4CA3EB0C021F
:10ED100022EA030212EACC1204BF51F8043B043089
:10ED2000F4D013F0FF0F1FBF013013F47F4F0130F9
:10ED300013F47F0F18BF0130704700BF40EA010392
:10ED40009B0770B42AD1032A28D90C4603462146D2
:10ED500054F8045BA5F1013626EA050616F0803F5B
:10ED600005D1043A032A43F8045B2146EFD89AB14F
:10ED70000C781C70013A01333CB16AB111F8014FB3
:10ED800003F8014B013A002CF7D12AB11A440021B3
:10ED900003F8011B9342FBD170BC70470346E6E7C2
:10EDA0002DE9F00F424C82B0D4F800C001900E461D
:10EDB00000E02646344614F8015B0CEB0500407871
:10EDC00000F0080000F0FF0A0028F2D12D2D5BD0E2
:10EDD0002B2D04BF7578B41C33F010003CD099463D
:10EDE000BAF1000F0CBF6FF0004B4FF0004BBBFBB4
:10EDF000F9F8002709FB18BB38460CE0303DAB4260
:10EE000019DD7E1C05D0404523D820D009FB0050D9
:10EE1000012714F8015B0CEB0506767816F0040F59
:10EE2000ECD116F0030606D0012E14BF5726372664
:10EE3000AD1BAB42E5DC7B1C15D0BAF1000F21D134
:10EE40000AB1EFB9116002B0BDE8F00F70475D453F
:10EE5000DCDD4FF0FF37DCE7302D1AD0002BBED1C0
:10EE60000A239946BCE70199BAF1000F4FF022033B
:10EE70000CBF6FF000404FF000400B60002AE2D062
:10EE8000611EDFE74042DBE7B41C75784FF0010AF2
:10EE9000A2E7207800F0DF00582803D0002B9ED195
:10EEA00008239CE7102365789946023498E700BF51
:10EEB000E4ABFF1F30B4044C0D46134601462A460E
:10EEC000206830BCFFF76CBFD0A7FF1F2DE9F00F03
:10EED000444C82B0D4F800C001900E4600E02646B3
:10EEE000344614F8015B0CEB0500407800F0080094
:10EEF00000F0FF070028F2D12D2D57D02B2D08BF91
:10EF00007578BA4608BFB41C33F0100039D04FF002
:10EF1000FF38B8FBF3F803FB08FB6FEA0B0B9946CD
:10EF2000002738460CE0303DAB4219DD002F25DBD1
:10EF3000404523D820D009FB0050012714F8015B7D
:10EF40000CEB0506767816F0040FECD116F00306EC
:10EF500006D0012E14BF57263726AD1BAB42E5DC89
:10EF6000002F1DDBBAF1000F18D10AB1A7B911604B
:10EF700002B0BDE8F00F70475D45DCDD4FF0FF37B4
:10EF8000DCE7302D17D0002BC1D10A2399464FF072
:10EF9000050BDFF85480C3E7611EE8E74042E4E771
:10EFA0000198222303604FF0FF30DEE7B41C757830
:10EFB0004FF0010AA8E7207800F0DF00582808D0B9
:10EFC000002BA4D1082399464FF0070B6FF060483F
:10EFD000A6E71023657899464FF00F0B02346FF0C7
:10EFE00070489DE7E4ABFF1F9999991930B4044C20
:10EFF0000D46134601462A46206830BCFFF766BF1F
:10F00000D0A7FF1FF0B5274C2668D6F8484185B039
:10F010000746002C41D065681F2D1EDD224818B917
:10F020004FF0FF3005B0F0BD4FF4C870039102926D
:10F030000193FEF7BDFE0399029A019B0446002846
:10F04000EED0D6F848512560002060600546C6F82D
:10F050004841C4F88801C4F88C013FB9AB1C0020BA
:10F060000135656044F8231005B0F0BD04EB850060
:10F070004FF0010CC0F88820D4F888610CFA05F232
:10F080001643022FC4F88861C0F80831E6D1D4F8DD
:10F090008C311A43C4F88C21E0E706F5A674C6F853
:10F0A0004841B8E7D8030100B1DD0000024B13B1BD
:10F0B000024800F005B8704700000000CDF00000E5
:10F0C0000146002002460346FFF79CBF38B5094DB4
:10F0D000094C641BA41018BF05EB840505D0013C46
:10F0E00055F8043D9847002CF9D1BDE8384001F0AF
:10F0F00025BA00BF0000000000000000F8B5234D55
:10F100000F460446FFF7DEF9AB685E6826F003069B
:10F11000F11B01F6EF7121F47F6121F00F01A1F5E0
:10F120008057B7F5805F07DB20460021FFF7BCFB67
:10F13000AB683344984204D02046FFF7C5F900205D
:10F14000F8BD20467942FFF7AFFB01300DD0104BE0
:10F15000AA681968F61B46F001062046C91B5660CE
:10F160001960FFF7B1F90120F8BD20460021FFF733
:10F170009BFBAB68C21A0F2ADEDD064D04492D68E1
:10F1800042F00102401B5A600860D5E7D4A7FF1F78
:10F190002CD9FF1FE0ABFF1F2DE9F0410D460646BD
:10F1A000002955D0FFF78EF955F8041CDFF874C11B
:10F1B00021F00103A5F10804E218DCF80800576803
:10F1C000904227F0030769D011F00101576032D057
:10F1D0000021D0194068C00706D43B44906800293C
:10F1E0004ED0D268C260906043F001026260E3508A
:10F1F000E1B9B3F5007F2DD35A0A042A6AD89809D9
:10F20000383041000CEB810C4649DCF8082062459F
:10F2100066D0516821F003018B4202D29268944576
:10F22000F7D1D368E360A2609C60D4603046BDE84B
:10F23000F041FFF749B955F8085C641B0CF1080868
:10F24000A06840452B4443D0E568C560A860C0E78E
:10F25000BDE8F081DB080CEBC3020125DCF80400FB
:10F260009168A1609B1005FA03F31843E260CCF8A3
:10F27000040094603046CC60BDE8F041FFF724B94B
:10F28000294DA842ADD143F00102CCF81440CCF88E
:10F290001040E060A0606260E350C7E71F44CB0706
:10F2A00007D455F8083CE41A1F44A268E368D36009
:10F2B0009A601E4B1B6847F001029F426260CCF8C7
:10F2C0000840B3D31A4B30461968FFF717FFADE774
:10F2D00001217EE7142A0CD802F15B00410091E77E
:10F2E0004B688010012505FA00F003434B6013467C
:10F2F00098E7542A03D8180B6E30410082E7B2F524
:10F30000AA7F03D8D80B773041007BE740F25451F5
:10F310008A4203D8980C7C30410073E7FC217E20A0
:10F3200070E700BFD4A7FF1FDCA7FF1FDCABFF1FE8
:10F3300028D9FF1FFFFFFFFF0000000000000000B2
:10F34000B19B000000000000E803D007E803DC05E3
:10F35000D0070000E803B004780540060807D0078E
:10F36000456E67696E6520736F756E64732064699E
:10F370007361626C6564202D2066696C6573206D15
:10F38000697373696E670000547261636B206F76F6
:10F3900065726C617920736F756E6473207072652D
:10F3A00073656E7400000000547261636B204F76C9
:10F3B00065726C617920736F756E64732064697314
:10F3C00061626C6564202D206E6F2066696C6573C8
:10F3D00020666F756E640000537461727420706CE7
:10F3E0006179696E6720000020696E20456E67694B
:10F3F0006E6520736C6F7420000000002028494463
:10F400003A2000002900000020696E204658207331
:10F410006C6F74200000000053746F702020706CBB
:10F420006179696E6720000053717565616B20001A
:10F4300020616761696E20696E200000206D5300B5
:10F440003A0000002D000000484152445741524507
:10F450002056455253494F4E3A2000004649524DDE
:10F46000574152452056455253494F4E3A200000CD
:10F47000302E39332E333000202D2000207C200008
:10F48000534F554E442046494C4520494E464F0067
:10F4900046696C656E616D6520202020202020204B
:10F4A0002020204D4D3A53533A6D532020202020E8
:10F4B0005072696F726974790000000054525545AA
:10F4C0000000000046414C534500000059657300A0
:10F4D0004E6F000048494748000000004C4F57005D
:10F4E00025000000566F6C756D657300456E676989
:10F4F0006E6520766F6C756D653A200045666665B1
:10F5000063747320766F6C756D653A20000000009F
:10F51000547261636B204F7665726C617920766FEF
:10F520006C756D653A20000053717565616B2053F1
:10F53000657474696E677300204D696E3D0000004C
:10F54000204D61783D00000020456E61626C65646D
:10F550003D00000053717565616B206D696E20730D
:10F56000706565643D0000004C69676874200000A8
:10F5700020466C6173682054696D653A2000000074
:10F5800020426C696E6B204F6E2054696D653A2085
:10F590000000000020426C696E6B204F66662054AC
:10F5A000696D653A200000005468726F74746C6570
:10F5B0002F456E67696E652053657474696E677355
:10F5C000000000004175746F20537461727420450F
:10F5D0006E67696E652077697468205468726F740D
:10F5E000746C653A200000004175746F2053746F8D
:10F5F0007020456E67696E6520416674657220549F
:10F60000696D652061742049646C653A20000000D2
:10F61000206D696E75746573000000004E2F410007
:10F620005468726F74746C6520537469636B2049FD
:10F63000646C652061743A200000000053746963B3
:10F640006B2043656E74657200000000537469633B
:10F650006B20456E6400000049646C652044656160
:10F660006462616E643A2000536572766F20536560
:10F670007474696E67730000536572766F2052650B
:10F680007665727365643A200000000054696D6508
:10F6900020746F207265636F696C3A20000000006F
:10F6A00054696D6520746F2072657475726E3A20AE
:10F6B00000000000456E6420706F696E74733A201C
:10F6C0000000000025207265636F696C6564202866
:10F6D00000000000207553292C20000025206261C5
:10F6E0007474657279202800207553290000000089
:10F6F000456E67696E652053746172740000000086
:10F70000456E67696E652053746F7000456E67695A
:10F710006E6520546F67676C6500000043616E6E14
:10F720006F6E200020466972650000004D616368BD
:10F73000696E652047756E200000000020537461DB
:10F74000727400002053746F7000000020546F67C3
:10F75000676C6500204F6E00204F66660000000059
:10F7600020537461727420626C696E6B696E6700FD
:10F7700020546F67676C6520626C696E6B696E6799
:10F780000000000020466C617368000055736572CC
:10F7900020536F756E64200020506C61790000006A
:10F7A00020526570656174004368616E6E656C20FF
:10F7B00054797065730000004368616E6E656C205B
:10F7C000000000005377697463682028000000007F
:10F7D00020706F736974696F6E7329005661726966
:10F7E00061626C6520496E707574202D20000000E8
:10F7F0004E756C6C00000000456E67696E652053A5
:10F8000070656564000000004D6173746572205678
:10F810006F6C756D65000000556E6B6E6F776E00D6
:10F8200020284368616E6E656C2052657665727340
:10F83000656429004368616E6E656C205472696767
:10F84000676572730000000020506F732000000095
:10F85000206F6E00206F66660000000020746F67E6
:10F86000676C65206F6E000020746F67676C6520A1
:10F870006F66660020737461727420626C696E6BCF
:10F88000696E67002073746F7020626C696E6B69BB
:10F890006E67000020666C61736800006368616ECB
:10F8A0006E656C5F66756E63000000006368315FB3
:10F8B00066756E63000000006368325F66756E6394
:10F8C000000000006368335F66756E63000000002F
:10F8D0006368345F66756E63000000006368355FBF
:10F8E00066756E63000000006368616E6E656C5F34
:10F8F0007265766572736564000000006368315F4D
:10F9000072657665727365006368325F72657665ED
:10F91000727365006368335F726576657273650044
:10F920006368345F72657665727365006368355F1E
:10F9300072657665727365006368616E6E656C5F93
:10F94000706F735F636F756E740000006368315F82
:10F95000706F73006368325F706F73006368335F4A
:10F96000706F73006368345F706F73006368355F36
:10F97000706F73006368616E6E656C5F706F735F4C
:10F980007472696767657273000000007371756552
:10F99000616B5F73657474696E67730073316D6951
:10F9A0006E00000073316D61780000007331656E88
:10F9B0000000000073326D696E00000073326D61EB
:10F9C000780000007332656E0000000073336D69CB
:10F9D0006E00000073336D61780000007333656E54
:10F9E0000000000073346D696E00000073346D61B7
:10F9F000780000007334656E0000000073356D6997
:10FA00006E00000073356D61780000007335656E1F
:10FA10000000000073366D696E00000073366D6182
:10FA2000780000007336656E000000006D696E732B
:10FA30007065656400000000766F6C756D6573001D
:10FA4000656E67696E650000656666656374730060
:10FA50006F7665726C6179006C6967687473000019
:10FA60006C315F666C617368000000006C315F622E
:10FA70006C696E6B6F6E00006C315F626C696E6BEF
:10FA80006F6666006C325F666C6173680000000030
:10FA90006C325F626C696E6B6F6E00006C325F621D
:10FAA0006C696E6B6F6666006C335F666C61736861
:10FAB000000000006C335F626C696E6B6F6E00005B
:10FAC0006C335F626C696E6B6F666600736572762D
:10FAD0006F000000736572766F5F72657665727392
:10FAE0006500000074696D655F7265636F696C0025
:10FAF00074696D655F72657475726E0065705F72B2
:10FB000065636F696C00000065705F6261747465A5
:10FB1000727900006175746F737461727400000013
:10FB20006175746F73746F70000000007468726F99
:10FB300074746C650000000063656E7465727468AF
:10FB4000726F74746C65000069646C6564656164EF
:10FB500062616E6400000000537461727420456E2F
:10FB600067696E650000000053687574646F776E96
:10FB700020456E67696E650053746F702053717510
:10FB800065616B73000000005374617274205371DF
:10FB90007565616B730000004552524F523A20590F
:10FBA0006F75206E65656420746F20757064617474
:10FBB000652074686520434F554E545F544F54413F
:10FBC0004C5F534F554E4446494C4553206E756D1E
:10FBD0006265722100000000535441525420544584
:10FBE000535420524F5554494E45000046696C65A8
:10FBF0006E616D6520202020202020202020204DB7
:10FC00004D3A53533A6D5300454E44205445535496
:10FC100020524F5554494E4500000000506C617908
:10FC2000696E672E2E2E2020000000004E6F74207B
:10FC3000666F756E64000000446F6E650000000022
:10FC4000566F6C756D6520436F6E74726F6C2053C8
:10FC50006F757263653A2053657269616C000000CC
:10FC6000566F6C756D6520436F6E74726F6C2053A8
:10FC70006F757263653A205243000000566F6C75D1
:10FC80006D6520436F6E74726F6C20536F75726375
:10FC9000653A204B6E6F6200446576696365206D3E
:10FCA0006F64653A20524320696E707574000000DD
:10FCB000446576696365206D6F64653A20536572AB
:10FCC00069616C20696E707574000000556E616228
:10FCD0006C6520746F20616363657373207468655D
:10FCE0002053442063617264202D20636865636B38
:10FCF00020616E64207265626F6F7420646576693E
:10FD000063650000496E692066696C652028000003
:10FD10002920646F6573206E6F7420657869737431
:10FD20000000000029206E6F742076616C69643ACF
:10FD300020000000496E692066696C65206578695D
:10FD4000737473202D2053657474696E6773204C2F
:10FD50006F616465643A0000284F6E6C792075739A
:10FD6000656420696E205243206D6F646529000030
:10FD70002F6F70736F756E642E696E6900FFFFFFE1
:10FD8000E803350583060807E803E204DC05D60628
:10FD9000080700006E6F206572726F72000000002D
:10FDA00066696C65206E6F7420666F756E64000006
:10FDB00066696C65206E6F74206F70656E00000060
:10FDC00062756666657220746F6F20736D616C6C0E
:10FDD000000000007365656B206572726F72000031
:10FDE00073656374696F6E206E6F7420666F756ED5
:10FDF000640000006B6579206E6F7420666F756E0D
:10FE000064000000656E64206F662066696C6500A2
:10FE1000756E6B6E6F776E206572726F7200000088
:10FE2000756E6B6E6F776E206572726F7220766181
:10FE30006C7565007472756500000000796573006B
:10FE40003100000066616C73650000006E6F000099
:10FE50003000FFFF0000010004000B0013001E0033
:10FE60002C003C004E0063007B009500B100D000E8
:10FE7000F10014013A0163018E01BB01EA011D0288
:10FE800051028802C102FC023A037B03BD03020453
:10FE900049049304DF042D057D05D00524067C0666
:10FEA000D50630078E07EE075008B4081A098309F3
:10FEB000ED095A0AC90A390BAC0B210C980C100D2C
:10FEC0008B0D080E860E070F890F0D1093101B1156
:10FED000A5113112BE124D13DE13701404159A15BC
:10FEE0003216CB16651701189F183E19DF19811AB3
:10FEF000251BCA1B711C181DC21D6C1E181FC51F97
:10FF000073202321D42186223923ED23A2245825CE
:10FF10000F26C82681273B28F628B2296F2A2D2BC9
:10FF2000EC2BAB2C6B2D2C2EED2EAF2F72303531F0
:10FF3000F931BD32823348340E35D4359B366237C1
:10FF40002938F138B939813A493B123CDB3CA43DB0
:10FF50006D3E363FFF3FC84091415A422343EB4339
:10FF6000B4447C4545460C47D4479C486349294ADC
:10FF7000F04AB64B7B4C404D044EC84E8C4F4E5011
:10FF80001051D251935253531254D0548E554B5654
:10FF90000757C2577C583659EE59A55A5C5B115C1D
:10FFA000C55C785D2A5EDB5E8A5F3960E6609161E0
:10FFB0003C62E5628D633364D9647C651E66BF660E
:10FFC0005F67FC6798683369CC69646AF96A8E6B0D
:10FFD000206CB16C406DCD6D596EE26E6A6FF06F42
:10FFE0007570F7707871F6717372EE726673DD7307
:10FFF0005274C5743675A47511767B76E4764A77AB
:020000021000EC
:10000000AE7710787078CE7829798379DA792F7A7B
:10001000817AD27A207B6C7BB57BFC7B417C847CB3
:10002000C47C027D3E7D777DAE7DE27D147E447E84
:10003000717E9C7EC47EEA7E0E7F2F7F4E7F6A7F1C
:10004000847F9B7FB07FC37FD37FE17FEC7FF47F92
:10005000FB7FFE7FFF7F000000000000000000002B
:10006000616C0000000000000000000000000000C3
:10007000E96D00000000000000000000000000002A
:10008000CD6E000000000000000000000000000035
:10009000B577000000000000000000000000000034
:1000A00029790000000000000000000000000000AE
:1000B0006985000081850000918500005987000056
:1000C00079870000AD8500000000000000000000FE
:1000D000319400003595000075940000899400006B
:1000E000B594000071940000050E08090D0C060778
:1000F0000F0400130393050E08090D0C06070F04E7
:10010000FFFFC585848687C4FFFF001303931A92FF
:10011000170000004008FE4340A004404408FE438E
:1001200044A004400018FE4300C004403000FE43D9
:10013000309004403400FE43349004401C18FE43C9
:100140001CC004401018FE4310C004400818FE43B1
:1001500008C004400C18FE430CC004400C10FE43C1
:100160000CB004401010FE4310B004401810FE43C1
:1001700018B004401C10FE431CB004401410FE4391
:1001800014B004400418FE4304C004400010FE43B1
:1001900000B004400008FE4300A004400408FE43F1
:1001A00004A004400C08FE430CA004400808FE43D1
:1001B00008A004401418FE4314C004401818FE435D
:1001C00018C004400410FE4304B004400810FE436D
:1001D00008B004401400FE43149004404C08FE4351
:1001E0004CA004400420FE4304D004402410FE43ED
:1001F00024B004402010FE4320B004402810FE43E9
:1002000028B004402C10FE432CB004400020FE43D4
:1002100000D004404808FE4348A004401000FE43BC
:10022000109004400D0A00006E616E00696E660059
:100230006F766600FFFFFFFF000000000000000077
:100240003DBC000049BC000015BC00001DBC000006
:1002500025BC00002DBC000035BC000000000000E3
:10026000001519150001000000A3FF1F1200000077
:10027000000200002CA3FF1F430000000003000049
:1002800088A3FF1F000000000103090414A3FF1F3F
:10029000000000000203090470A3FF1F000000001B
:1002A000030309048CA3FF1F0000000000000000EE
:1002B000000000000000000000000000000000003E
:1002C000CDCA0000E5CA00009DCA0000ADCA00000A
:1002D000A5CA0000B5CA000019CA000031CA000052
:1002E00051CA000059CA000065CA000071CA000066
:1002F0007DCA00008DCA0000BDCA0000C5CA00004A
:10030000E9C90000F5C9000001CA00000DCA0000DB
:10031000F5CA0000D9CA000000000000000000007B
:1003200011CC000029CC0000E1CB0000F1CB000093
:10033000E9CB0000F9CB00005DCB000075CB0000DD
:1003400095CB00009DCB0000A9CB0000B5CB0000F1
:10035000C1CB0000D1CB000001CC000009CC0000D3
:100360002DCB000039CB000045CB000051CB000065
:1003700039CC00001DCC000000000000000000008F
:1003800055CD00006DCD000025CD000035CD00001D
:100390002DCD00003DCD0000A1CC0000B9CC000067
:1003A000D9CC0000E1CC0000EDCC0000F9CC00007D
:1003B00005CD000015CD000045CD00004DCD00005D
:1003C00071CC00007DCC000089CC000095CC0000F1
:1003D0007DCD000061CD0000A8A3FF1F00202020DC
:1003E00020202020202028282828282020202020E5
:1003F00020202020202020202020202020881010B5
:100400001010101010101010101010101004040410
:1004100004040404040404101010101010104141CE
:1004200041414141010101010101010101010101BC
:1004300001010101010101011010101010104242D0
:10044000424242420202020202020202020202028C
:10045000020202020202020210101010200000002C
:10046000000000000000000000000000000000008C
:10047000000000000000000000000000000000007C
:10048000000000000000000000000000000000006C
:10049000000000000000000000000000000000005C
:1004A000000000000000000000000000000000004C
:1004B000000000000000000000000000000000003C
:1004C000000000000000000000000000000000002C
:1004D000000000000000000000000000000000001C
:1004E000F8B500BFF8BC08BC9E467047ADF00000F0
:1004F00035040000295B0000696D0000856D000077
:10050000B16D0000CD6D0000317100004D71000033
:100510006971000085710000A1710000BD710000CB
:100520001D8D0000418D0000B996000059BC0000EF
:0C05300011CB000055CC000099CD00005C
:04053C00F8B500BF4F
:1005400038B5084B1C681C6054B1074D94FAA4F3ED
:10055000B3FA83F355F823309847631E1C40F5D156
:1005600038BD00BFA0D00440ECA2FF1F38B5084B37
:100570001C681C6054B1074D94FAA4F3B3FA83F3DA
:1005800055F823309847631E1C40F5D138BD00BF95
:10059000A0C00440CCA2FF1F38B5084B1C681C60EB
:1005A00054B1074D94FAA4F3B3FA83F355F823300A
:1005B0009847631E1C40F5D138BD00BFA0B0044071
:1005C0009CA2FF1F38B5084B1C681C6054B1074D36
:1005D00094FAA4F3B3FA83F355F823309847631ED3
:1005E0001C40F5D138BD00BFA0A004404CA2FF1FA5
:1005F00038B5084B1C681C6054B1074D94FAA4F33D
:10060000B3FA83F355F823309847631E1C40F5D1A5
:1006100038BD00BFA090044014A2FF1F00000000DE
:100620000000803F0000803F0000803F000000008D
:1006300075736572312E776176000000000000004E
:10064000000000000100000075736572322E7761B2
:100650007600000000000000000000000100000023
:1006600075736572332E776176000000000000001C
:10067000000000000100000075736572342E776180
:1006800076000000000000000000000001000000F3
:1006900075736572352E77617600000000000000EA
:1006A000000000000100000075736572362E77614E
:1006B00076000000000000000000000001000000C3
:1006C00075736572372E77617600000000000000B8
:1006D000000000000100000075736572382E77611C
:1006E0007600000000000000000000000100000093
:1006F00075736572392E7761760000000000000086
:1007000000000000010000007573657231302E7723
:100710006176000000000000000000000100000001
:100720007573657231312E7761760000000000002C
:1007300000000000010000007573657231322E77F1
:1007400061760000000000000000000001000000D1
:100750007573657231332E776176000000000000FA
:1007600000000000010000007573657231342E77BF
:1007700061760000000000000000000001000000A1
:100780007573657231352E776176000000000000C8
:1007900000000000010000007573657231362E778D
:1007A0006176000000000000000000000100000071
:1007B0007573657231372E77617600000000000096
:1007C00000000000010000007573657231382E775B
:1007D0006176000000000000000000000100000041
:1007E0007573657231392E77617600000000000064
:1007F00000000000010000007573657232302E7732
:100800006176000000000000000000000100000010
:100810007573657232312E7761760000000000003A
:1008200000000000010000007573657232322E77FF
:1008300061760000000000000000000001000000E0
:1008400002016401656E7374617274322E77617691
:10085000000000000000000001000000D0070000C0
:10086000656E6163636C312E776176000000000075
:100870000000000001000000656E6163636C322EB1
:100880007761760000000000000000000100000019
:10089000656E6163636C332E776176000000000043
:1008A0000000000001000000656E6163636C342E7F
:1008B00077617600000000000000000001000000E9
:1008C000656E6163636C352E776176000000000011
:1008D00000000000010000000105020FFFFFFF19EA
:1008E000656E6465636C312E7761760000000000F0
:1008F0000000000001000000656E6465636C322E2C
:100900007761760000000000000000000100000098
:10091000656E6465636C332E7761760000000000BD
:100920000000000001000000656E6465636C342EF9
:100930007761760000000000000000000100000068
:10094000656E6465636C352E77617600000000008B
:1009500000000000010000000100000074725F73DD
:10096000746172742E776176000000000000000050
:10097000010000007475727265742E776176000054
:1009800000000000000000000100000074725F73AE
:10099000746F702E77617600000000000000000088
:1009A0000100000074725F737472746D2E7761764B
:1009B0000000000000000000010000007475727269
:1009C00065745F6D2E776176000000000000000006
:1009D0000100000074725F73746F706D2E77617622
:1009E00000000000000000000100000062725F7360
:1009F000746172742E7761760000000000000000C0
:100A00000100000062617272656C2E7761760000F1
:100A100000000000000000000100000062725F732F
:100A2000746F702E776176000000000000000000F7
:100A3000010000006D675F73746172742E776176D8
:100A40000000000000000000030000006D672E772A
:100A500061760000000000000000000000000000BF
:100A6000030000006D675F73746F702E776176000E
:100A70000000000000000000030000006D673273FA
:100A8000746172742E77617600000000000000002F
:100A9000030000006D67322E7761760000000000D1
:100AA0000000000000000000030000006D673273CA
:100AB000746F702E77617600000000000000000067
:100AC000030000006D673373746172742E77617672
:100AD0000000000000000000030000006D67332EDE
:100AE00077617600000000000000000000000000B8
:100AF000030000006D673373746F702E77617600AA
:100B000000000000000000000300000063616E6E42
:100B10006F6E662E77617600000000000000000016
:100B20000100000063616E6E6F6E66322E77617633
:100B300000000000000000000100000063616E6E14
:100B40006F6E66332E7761760000000000000000B3
:100B50000100000063616E6E6F6E682E7761760033
:100B600000000000000000000100000072656C6FD2
:100B7000616465642E77617600000000000000006B
:100B8000010000006D676869742E776176000000CF
:100B900000000000000000000100000064657374A4
:100BA000726F792E7761760000000000000000006F
:100BB000010000006C69676874312E77617600006F
:100BC0000000000000000000010000006C69676880
:100BD00074322E77617600000000000000000000F3
:100BE000010000006C69676874332E77617600003D
:100BF000000000000000000001000000726570614C
:100C000069722E776176000000000000000000008D
:100C100001000000626565702E77617600000000BB
:100C20000000000000000000090000006272616B1B
:100C3000652E7761760000000000000000000000D3
:100C4000010000007478656E676167652E776176D4
:100C500000000000000000000100000074786465DE
:100C6000676167652E776176000000000000000074
:100C70000100000073717565616B312E776176003C
:100C800000000000000000000100000073717565A5
:100C9000616B322E776176000000000000000000DA
:100CA0000100000073717565616B332E776176000A
:100CB0000000000000000000010000007371756575
:100CC000616B342E776176000000000000000000A8
:100CD0000100000073717565616B352E77617600D8
:100CE0000000000000000000010000007371756545
:100CF000616B362E77617600000000000000000076
:100D000001000000040A000074726B73746F702E8F
:100D10007761760000000000000000000200000083
:100D200074726B73746172742E77617600000000C8
:100D30000000000002000000656E72756E312E77B3
:100D400061760000000000000000000001000000CB
:100D5000656E72756E322E776176000000000000BD
:100D60000000000001000000656E72756E332E7782
:100D7000617600000000000000000000010000009B
:100D8000656E72756E342E7761760000000000008B
:100D90000000000001000000656E72756E352E7750
:100DA000617600000000000000000000010000006B
:100DB000656E72756E362E77617600000000000059
:100DC0000000000001000000656E72756E372E771E
:100DD000617600000000000000000000010000003B
:100DE000656E72756E382E77617600000000000027
:100DF0000000000001000000656E72756E392E77EC
:100E0000617600000000000000000000010000000A
:100E1000656E72756E31302E7761760000000000CD
:100E2000000000000100000070FD0000010D000046
:100E3000656E69646C655F642E7761760000000002
:100E40000000000001000000656E7374617274316F
:100E50002E77617600000000000000000100000015
:100E6000656E73746F702E7761760000000000006D
:100E70000000000001000000656E69646C65312EA1
:100E80007761760000000000000000000100000013
:100E9000656E69646C65322E776176000000000033
:100EA0000000000001000000656E69646C65332E6F
:100EB00077617600000000000000000001000000E3
:100EC000656E69646C65342E776176000000000001
:100ED0000000000001000000656E69646C65352E3D
:100EE00077617600000000000000000001000000B3
:100EF00064FF02FFE8030000747261636B73312EBC
:100F00007761760000000000000000000100000092
:100F1000747261636B73322E77617600000000009B
:100F20000000000001000000747261636B73332ED7
:100F30007761760000000000000000000100000062
:100F4000747261636B73342E776176000000000069
:100F50000000000001000000747261636B73352EA5
:100F60007761760000000000000000000100000032
:100F7000747261636B73362E776176000000000037
:100F80000000000001000000747261636B73372E73
:100F90007761760000000000000000000100000002
:100FA000747261636B73382E776176000000000005
:100FB0000000000001000000747261636B73392E41
:100FC00077617600000000000000000001000000D2
:100FD000747261636B7331302E77617600000000AC
:100FE0000000000001000000FF020C0A04000000E5
:100FF0006CD9FF1F599C0000599C0000599C0000AF
:10100000599C0000599C0000599C0000599C00000C
:10101000599C0000599C0000599C0000599C0000FC
:10102000599C0000599C0000599C0000599C0000EC
:10103000599C0000599C0000599C0000599C0000DC
:10104000599C0000599C0000599C0000599C0000CC
:10105000599C0000599C0000599C0000599C0000BC
:10106000599C0000599C0000599C0000599C0000AC
:10107000599C0000599C0000599C0000599C00009C
:10108000599C0000599C0000599C0000599C00008C
:10109000599C0000599C0000599C0000599C00007C
:1010A000599C0000599C0000599C0000599C00006C
:1010B000599C0000599C0000599C0000599C00005C
:1010C000599C0000599C0000599C0000599C00004C
:1010D000599C000001000000FFFFFFFF090A080003
:1010E0001201010102000040C01683040002010247
:1010F0000301000018035400650065006E007300D2
:1011000079006400750069006E006F0009024300F9
:10111000020100C03209040000010202010005249E
:101120000010010524010101042402060524060023
:10113000010705820310004009040100020A0000B3
:10114000000705030240000007058402400000007C
:101150001603550053004200200053006500720042
:10116000690061006C000000040309040C03000026
:10117000000000000000000000000000000000006F
:1011800000000000000000000000000094A6FF1F07
:10119000FCA6FF1F64A7FF1F000000000000000066
:1011A000000000000000000000000000000000003F
:1011B00000000000000000000000000078FC0000BB
:1011C000000000000000000000000000000000001F
:1011D000000000000000000000000000000000000F
:1011E00000000000000000000000000000000000FF
:1011F00000000000000000000000000000000000EF
:1012000000000000000000000000000000000000DE
:1012100000000000000000000000000000000000CE
:1012200000000000000000000000000000000000BE
:1012300001000000000000000E33CDAB34126DE65B
:10124000ECDE05000B0000000000000000000000C4
:10125000000000000000000000000000000000008E
:10126000000000000000000000000000000000007E
:10127000000000000000000000000000000000006E
:10128000000000000000000000000000000000005E
:1015B000A8A3FF1F0000000000000000D4A7FF1F29
:1015C000D4A7FF1FDCA7FF1FDCA7FF1FE4A7FF1F97
:1015D000E4A7FF1FECA7FF1FECA7FF1FF4A7FF1F47
:1015E000F4A7FF1FFCA7FF1FFCA7FF1F04A8FF1FF6
:1015F00004A8FF1F0CA8FF1F0CA8FF1F14A8FF1FA3
:1016000014A8FF1F1CA8FF1F1CA8FF1F24A8FF1F52
:1016100024A8FF1F2CA8FF1F2CA8FF1F34A8FF1F02
:1016200034A8FF1F3CA8FF1F3CA8FF1F44A8FF1FB2
:1016300044A8FF1F4CA8FF1F4CA8FF1F54A8FF1F62
:1016400054A8FF1F5CA8FF1F5CA8FF1F64A8FF1F12
:1016500064A8FF1F6CA8FF1F6CA8FF1F74A8FF1FC2
:1016600074A8FF1F7CA8FF1F7CA8FF1F84A8FF1F72
:1016700084A8FF1F8CA8FF1F8CA8FF1F94A8FF1F22
:1016800094A8FF1F9CA8FF1F9CA8FF1FA4A8FF1FD2
:10169000A4A8FF1FACA8FF1FACA8FF1FB4A8FF1F82
:1016A000B4A8FF1FBCA8FF1FBCA8FF1FC4A8FF1F32
:1016B000C4A8FF1FCCA8FF1FCCA8FF1FD4A8FF1FE2
:1016C000D4A8FF1FDCA8FF1FDCA8FF1FE4A8FF1F92
:1016D000E4A8FF1FECA8FF1FECA8FF1FF4A8FF1F42
:1016E000F4A8FF1FFCA8FF1FFCA8FF1F04A9FF1FF1
:1016F00004A9FF1F0CA9FF1F0CA9FF1F14A9FF1F9E
:1017000014A9FF1F1CA9FF1F1CA9FF1F24A9FF1F4D
:1017100024A9FF1F2CA9FF1F2CA9FF1F34A9FF1FFD
:1017200034A9FF1F3CA9FF1F3CA9FF1F44A9FF1FAD
:1017300044A9FF1F4CA9FF1F4CA9FF1F54A9FF1F5D
:1017400054A9FF1F5CA9FF1F5CA9FF1F64A9FF1F0D
:1017500064A9FF1F6CA9FF1F6CA9FF1F74A9FF1FBD
:1017600074A9FF1F7CA9FF1F7CA9FF1F84A9FF1F6D
:1017700084A9FF1F8CA9FF1F8CA9FF1F94A9FF1F1D
:1017800094A9FF1F9CA9FF1F9CA9FF1FA4A9FF1FCD
:10179000A4A9FF1FACA9FF1FACA9FF1FB4A9FF1F7D
:1017A000B4A9FF1FBCA9FF1FBCA9FF1FC4A9FF1F2D
:1017B000C4A9FF1FCCA9FF1FCCA9FF1FD4A9FF1FDD
:1017C000D4A9FF1FDCA9FF1FDCA9FF1FE4A9FF1F8D
:1017D000E4A9FF1FECA9FF1FECA9FF1FF4A9FF1F3D
:1017E000F4A9FF1FFCA9FF1FFCA9FF1F04AAFF1FEC
:1017F00004AAFF1F0CAAFF1F0CAAFF1F14AAFF1F99
:1018000014AAFF1F1CAAFF1F1CAAFF1F24AAFF1F48
:1018100024AAFF1F2CAAFF1F2CAAFF1F34AAFF1FF8
:1018200034AAFF1F3CAAFF1F3CAAFF1F44AAFF1FA8
:1018300044AAFF1F4CAAFF1F4CAAFF1F54AAFF1F58
:1018400054AAFF1F5CAAFF1F5CAAFF1F64AAFF1F08
:1018500064AAFF1F6CAAFF1F6CAAFF1F74AAFF1FB8
:1018600074AAFF1F7CAAFF1F7CAAFF1F84AAFF1F68
:1018700084AAFF1F8CAAFF1F8CAAFF1F94AAFF1F18
:1018800094AAFF1F9CAAFF1F9CAAFF1FA4AAFF1FC8
:10189000A4AAFF1FACAAFF1FACAAFF1FB4AAFF1F78
:1018A000B4AAFF1FBCAAFF1FBCAAFF1FC4AAFF1F28
:1018B000C4AAFF1FCCAAFF1FCCAAFF1FD4AAFF1FD8
:1018C000D4AAFF1FDCAAFF1FDCAAFF1FE4AAFF1F88
:1018D000E4AAFF1FECAAFF1FECAAFF1FF4AAFF1F38
:1018E000F4AAFF1FFCAAFF1FFCAAFF1F04ABFF1FE7
:1018F00004ABFF1F0CABFF1F0CABFF1F14ABFF1F94
:1019000014ABFF1F1CABFF1F1CABFF1F24ABFF1F43
:1019100024ABFF1F2CABFF1F2CABFF1F34ABFF1FF3
:1019200034ABFF1F3CABFF1F3CABFF1F44ABFF1FA3
:1019300044ABFF1F4CABFF1F4CABFF1F54ABFF1F53
:1019400054ABFF1F5CABFF1F5CABFF1F64ABFF1F03
:1019500064ABFF1F6CABFF1F6CABFF1F74ABFF1FB3
:1019600074ABFF1F7CABFF1F7CABFF1F84ABFF1F63
:1019700084ABFF1F8CABFF1F8CABFF1F94ABFF1F13
:1019800094ABFF1F9CABFF1F9CABFF1FA4ABFF1FC3
:10199000A4ABFF1FACABFF1FACABFF1FB4ABFF1F73
:1019A000B4ABFF1FBCABFF1FBCABFF1FC4ABFF1F23
:1019B000C4ABFF1FCCABFF1FCCABFF1F000002006E
:0819C000FFFFFFFFDC03010043
:00000001FF
